:020000040800F2
:100000005838002063050008AD040008650A02089E
:10001000B1040008B3040008B504000800000000A3
:10002000000000000000000000000000B70400080D
:10003000B904000800000000BB040008BD0400086B
:10004000BF040008C1040008C3040008C504000878
:10005000C7040008C9040008CB040008CD04000848
:10006000CF040008D1040008D3040008D504000818
:10007000D7040008D9040008DB040008DD040008E8
:10008000DF040008E1040008E3040008E5040008B8
:10009000E7040008E9040008EB040008ED04000888
:1000A000EF040008F1040008F3040008F504000858
:1000B000F7040008F9040008FB040008FD04000828
:1000C000FF040008010500080305000805050008F5
:1000D00007050008090500080B0500080D050008C4
:1000E0000F05000811050008130500081505000894
:1000F00017050008190500081B0500081D05000864
:100100001F05000821050008230500082505000833
:1001100027050008290500082B0500082D05000803
:100120002F050008310500083305000835050008D3
:1001300037050008390500083B0500083D050008A3
:100140003F05000841050008430500084505000873
:1001500047050008490500084B0500084D05000843
:100160004F05000851050008530500085505000813
:1001700057050008590500085B0500085D050008E3
:080180005F050008610500089D
:10020000DECEA5ED02003078463430370000000025
:1002100000000000000044433231365F3134313099
:100220000000000000004170706C69636174696FC8
:100230006E00000000000000000000000000000050
:100240000000000000000418BB00DAF7DECEA5EDC8
:100250000200307846343037000000000000000013
:10026000000053504C6174436F6E74726F6C6C6518
:1002700072004170706C69636174696F6E00000098
:10028000000000000000000000000000000000006E
:0802900000000000FE00DAF797
:1002980001000208100000002500020818000000F4
:1002A800790102081700000009060208170000007B
:1002B8000509020803000000410F020806000000BB
:1002C800E112020809000000811B02080200000078
:1002D8008D1C020811000000112102081000000006
:1002E800CD220208FF000000B12A02080C0000001D
:1002F800B92F020800000000F531020805000000CF
:1003080031580208120000002D5C02080A000000A3
:10031800056202080A000000C56C0208140000000B
:100328001D77020808000000D57E020807000000BB
:100338007D850208100000008D8902081300000066
:10034800359B02081300000025CA020816000000A9
:10035800A52E030816000000A930030817000000A6
:10036800B96803081600000089690308170000002F
:08037800397D030815000000A7
:100380002F49072291438D462E492F480A1A06D03D
:100390000722914381F30988022282F314882B48B3
:1003A0002B492C4A00F039F82B482C492C4A00F0F4
:1003B00034F82C482C492D4A00F02FF82C482D49B0
:1003C0002D4A00F02AF82D482D492E4A00F025F834
:1003D0002D482E492E4A00F020F82E482E490022A2
:1003E00000F026F82D482E49091A082903DB0022BF
:1003F0000260043001601F481F49884205D002682E
:10040000043003B4904703BCF7E700208646EC466F
:1004100000200021234A9047FEE7884207D0521A65
:1004200005D0037801300B700131013AF9D17047E2
:10043000884202D002700130FAE770471A487047CC
:1004400058380020584000205838002030EE03086B
:1004500088010020FC0100200000020800000208C2
:10046000F0BB030830EE030888010020880100205B
:10047000BC050008BC050008BC050008BC05000858
:10048000BC050008BC050008F0BB0308F0BB03086E
:1004900030EE0308FC0100200C3500205835002008
:1004A000583500202D400208FFFFFFFFFEE7FEE762
:1004B000FEE7FEE7FEE7FEE7FEE7FEE7FEE7FEE714
:1004C000FEE7FEE7FEE7FEE7FEE7FEE7FEE7FEE704
:1004D000FEE7FEE7FEE7FEE7FEE7FEE7FEE7FEE7F4
:1004E000FEE7FEE7FEE7FEE7FEE7FEE7FEE7FEE7E4
:1004F000FEE7FEE7FEE7FEE7FEE7FEE7FEE7FEE7D4
:10050000FEE7FEE7FEE7FEE7FEE7FEE7FEE7FEE7C3
:10051000FEE7FEE7FEE7FEE7FEE7FEE7FEE7FEE7B3
:10052000FEE7FEE7FEE7FEE7FEE7FEE7FEE7FEE7A3
:10053000FEE7FEE7FEE7FEE7FEE7FEE7FEE7FEE793
:10054000FEE7FEE7FEE7FEE7FEE7FEE7FEE7FEE783
:10055000FEE7FEE7FEE7FEE7FEE7FEE7FEE7FEE773
:10056000FEE71348854600F022F84EF68850CEF29A
:100570000000016851F47001016000BF00BF00BFBE
:10058000F1EE100A50F04070E1EE100A4FF000005A
:1005900080F314884EF63C71CEF20001086850F0EA
:1005A00040700860034804490160FFF7E9BE7047E6
:0C05B0000000022008ED00E00000000840
:020000040801F1
:1000000000000000000000000000000000000000F0
:1000100000000000000000000000000000000000E0
:10002000000000000000000000000000000004EAE2
:100030000F018600003D8601003D680120830042DB
:10004000F430F10B000E496E697469616C69736973
:100050006E672E2EF00400C000F411F40300790046
:100060000000F10A0006F10A0101F00201C085F169
:100070000A0001F00104C085095E8302A1F00001BD
:10008000C0008302DE8302C78304B5F10A0001F1D8
:100090000A0100F00200C000F10A0003F10A0101A8
:1000A000F00201C000F10500F00300C000F10B00F8
:1000B0000156F00400C0001E0000145D0B00CB4A86
:1000C000077108F42D00007D800085F419830387F3
:1000D000F00001C000F10B0010456E7465722059EC
:1000E0006561723A2020202020F00400C000F10B4E
:1000F00000023230F00400C0008F13028301B3818C
:100100000079830387F00001C000F10B000C456EFD
:10011000746572204D6F6E74683AF00400C0008FF1
:1001200013038301B38100CD830387F00001C00076
:10013000F10B000A456E746572204461793AF0044F
:1001400000C0008F13048301B3810102800154F4C5
:1001500019800128F41AF4114A00F420830387F06F
:100160000001C000F10B0010456E74657220486FED
:10017000757220283234293AF00400C0008F130031
:100180008301B381014F830387F00001C000F10BAD
:10019000000E456E746572204D696E757465733A14
:1001A000F00400C0008F13018301B381015CF412DD
:1001B0008000795E690020F10A0001F10A0100F077
:1001C0000200C000171301D001D801E001F502219F
:1001D000F41B83035780024AF41D83035780024AAD
:1001E000F10A0001F10A0102F00200C000F41B83D1
:1001F000035780024AF41DF303004783033EF41DB6
:10020000F10B00022028F00400C000F10200F00110
:1002100001C000F10B00022920F00400C0008002A0
:100220004AF41F83036FF10B00022028F00400C082
:1002300000F42FF423F303001583033EF10B0002B7
:100240002920F00400C00080024A830393F4028C4A
:100250000802658C0902805D0A029B5D0B029E68A4
:10026000002080024D17130271027602710276029D
:100270007BF4288001B7F4298001B7F42A8001B704
:100280001713028C0291028C02910296F4388001BD
:10029000B7F4398001B7F43A8001B74A00094A013E
:1002A00009F41300F41B870002B7F41D870002B79E
:1002B000F421877F02B7094A00F41C4A00F41E4A61
:1002C0007FF422F4140009F10A0001F10A0105F09B
:1002D0000200C000F411F416F00400C00009F10A95
:1002E0000000F10A0100F00200C000F419F423F349
:1002F00003001583033EF10B000120F00400C00051
:10030000F41F01890A0311F10B000120F00400C061
:1003100000F10200F00101C000F10B000120F00427
:1003200000C000F41DF303004783033EF10B0003FC
:10033000203230F00400C000F41B83035709F3118E
:1003400002F30BF30900F31103F30A0000F31F009B
:1003500000F00400C0000901890A0366F10B0001E6
:1003600030F00400C000F10200F00101C0000901FA
:10037000890A037EF10B000120F00400C000F102A5
:1003800000F00101C00009F40270084A0F52820314
:10039000875E09F40661002003A29948000084806A
:1003A00003A79920000082F40270084A0F528103CB
:1003B000BBF437F61C03A76900200968002009096F
:1003C000F00002C08509F10200F00100C08509F1CA
:1003D0000200F00101C08509F10A0000F00101C02E
:1003E0008509F10200F00104C08509F10200F00165
:1003F00005C08509F10200F00106C08509F102017E
:10040000F10200F00201C08509F10201F10200F0E1
:100410000202C085F10102F1010109F00500C08569
:10042000F1010009F00501C085F1010009F00502A4
:10043000C085F101004AFE525609F00503C085F15E
:10044000010009F00504C085F1010009F00600C0B3
:1004500085F10101F1010009F00601C085F10100FB
:10046000F1010109F00602C085F10101F101000965
:10047000F00608C085F10101F1010009F00603C092
:1004800085F10101F1010009F00606C085F10101C5
:10049000F1010009F10200F00607C085F10101F148
:1004A000010009F00702C085F1060009F00703C04A
:1004B00085F1060009F00704C085F1060009F0087F
:1004C00000C085F10103F10102F10101F101000910
:1004D000F00400C085F10102F1010109F00401C03E
:1004E00085F10103F10102F10101094D6F6E5475AF
:1004F0006557656454687246726953617453756ECA
:100500000000000300060009000C000F00124A6101
:100510006E4665624D61724170724D61794A756EC9
:100520004A756C4175675365704F63744E6F7644BE
:1005300065630000002300260029002C002F0032F4
:1005400000350038003B003E00410044FFFFFFFF44
:10055000FFFFFFFFFFFFFFFFFFFFFFFFFFFFFFFFAB
:10056000FFFFFFFFFFFFFFFFFFFFFFFFFFFFFFFF9B
:10057000FFFFFFFFFFFFFFFFFFFFFFFFFFFFFFFF8B
:10058000FFFFFFFFFFFFFFFFFFFFFFFFFFFFFFFF7B
:020000040802F0
:1000000000B583B04FF0000100914FF0F60301936B
:1000100008464FF007024FF0010303F067FB03B0FF
:1000200000BD00BF10B54FF002004FF0F80116F010
:1000300043FF40F2B104C0F602044FF003004FF05A
:100040000001224604F056FB4FF0010040F2A501EA
:10005000C0F60201224604F04DFB4FF000000146BD
:10006000224604F047FB4FF008004FF0090102461A
:1000700012F042FE4FF000004FF001014FF003027A
:1000800001F0F4FB4FF0010049F69A11C3F69961B3
:1000900002F092FA4BF62440C0F6030008F002FF8B
:1000A00010BD00BF08B54FF00A0001F01FFA08BDEF
:1000B00008B521B94FF0030017F008FE08BD01296B
:1000C00004D14FF0010017F001FE08BD022903D151
:1000D0004FF0000017F0FAFD08BD00BF11B1012973
:1000E00016D108E040F28811C2F200010B781370BB
:1000F0004FF00000704740F21000C4F202000168A7
:1001000081F01003C3F3001010704FF0000070472F
:100110004FF01400704700BF11B1012928D11AE037
:1001200042F63C01C4F200010B6813F4004F42F6A2
:100130003C00C4F2000001684FEAC1534FEAD350BB
:1001400008BF404207EE100AF8EEC70AC2ED000AE7
:100150004FF00000704740F2FC10C2F20000D0EDFA
:10016000007AB8EE670A82ED000A4FF0000070478F
:100170004FF01400704700BF30B585B04FF0010557
:1001800000954FF00304019402954FF000004FF0EA
:1001900005012246034601F0B9F800950194029545
:1001A0004FF0000021462246034601F0AFF84FF41D
:1001B00000504BF66441C0F6030140F20422C2F243
:1001C00000020BF015FB05B030BD00BF38B514467A
:1001D0004FF000031370002940F0838040F20020AC
:1001E000C2F20000016800297ED142F62402C4F266
:1001F00000024FF0CA0515604FF05303136042F63A
:100200000800C4F20000016841F40025056003689D
:1002100043F4000101604FF0FF00106043F6400519
:10022000C4F202052A6842F001032B604BF69841A4
:10023000C0F60301086840F20003C4F2000318602E
:100240004FF0000540F20402C4F2000215604BF6C4
:100250004841C0F60301086840F20802C4F20002F7
:10026000106040F22002C4F2000215604BF64441D7
:10027000C0F60301086840F21C01C4F200010860E6
:100280004BF64C40C0F603000168116040F22C02AE
:10029000C4F200024FF0FF30106040F22801C4F2B7
:1002A00000010D801A8842F0010018804BF6504082
:1002B000C0F603004FF0070140F29932C0F6020287
:1002C00007F070FE40F20023C2F2000318604FF006
:1002D000010140F28812C2F200021170217028461A
:1002E00038BD4FF0140038BD4FF0000038BD00BFDE
:1002F00070B508F023FB054643F2D30440F2100624
:10030000C4F2000608F01AFB401BA04209D940F2D3
:100310008813C2F200034FF0050119704FF000007E
:1003200070BD07F04BFE336803F010018AB2002A5B
:10033000E8D040F24000C4F20000006870BD00BF89
:1003400030B583B005460C464FF0F60001A94FF0DA
:10035000020203F01FFDBDF80430C3F340222A70EF
:100360004FEAC3514FEAD153236003B030BD00BF01
:1003700000B583B04FF0000360F3492361F3080335
:1003800002A820F8043D4FF002014FF0F60203F0FE
:100390009DFD03B000BD00BFF8B54FF00000014661
:1003A00001F0FEFD40F24003C4F200031B68FFF7BA
:1003B0009FFF0646002800F0F980FFF799FF0746E7
:1003C000002800F0F380861B304617F03BFE044601
:1003D0000D4687A3D3E9002318F096FA002862D1CE
:1003E0002046294684A3D3E9002318F0A9FA00285F
:1003F00059D140F2FC10C2F200000660FFF778FF0E
:100400000546002800F0D280C71BBE4294BFC6EB51
:100410000703C7EB0603012B66D940F2FC11C2F2B9
:1004200000010F60FFF764FF0446002800F0BE8063
:10043000461BB74294BFC7EB0603C6EB0703012B6D
:100440004FD940F2FC12C2F200021660FFF750FFD3
:100450000546002800F0AA80041BA64294BFC6EB04
:100460000403C4EB0603012B3ED940F2FC17C2F291
:1004700000073C60FFF73CFF0746002800F096802D
:10048000461BB44294BFC4EB0603C6EB0403012B26
:1004900029D940F2FC13C2F200031E60FFF728FFC7
:1004A000014640B982E040F28813C2F200034FF0E7
:1004B000020119707AE0C01BB04234BFC0EB0601E4
:1004C000C6EB000101290FD940F2FC12C2F2000272
:1004D000106040F28813C2F200034FF0020119705D
:1004E00064E03E4600E02646304617F0ABFD02468B
:1004F0000B4643A1D1E9000117F0CAFE17F08CFEAC
:1005000017F06EFE4FF000024FF00003C4F2E0035C
:1005100018F004F83AA3D3E9002318F0B5F84FF027
:1005200000024FF00003C4F2400317F0F7FF17F08A
:1005300073FE044618F020FA0546204617F050FED8
:1005400018F03EFF4FF000024FF00003C3F6E073D7
:1005500017F0A0FE17F00AFE0446B0F5007F07D39F
:1005600040F28810C2F200004FF0040202701DE059
:10057000003518BF01250DB1C0F50074284621468D
:1005800001F00EFD28462146FFF7F2FE38B940F291
:100590008813C2F200034FF00301197006E040F225
:1005A0008810C2F200004FF00002027042F62400F0
:1005B000C4F200004FF0CA0202604FF05303036020
:1005C00042F60802C4F2000211686FF3D3411160D1
:1005D00013686FF3D75313604FF0FF02026040F2CD
:1005E0000020C2F200004FF000010160F8BD00BF22
:1005F0000000000053126341000000004D136341EE
:1006000000000000D012634108B54FF440504BF693
:100610009C41C0F6030140F21822C2F200020BF026
:10062000E7F808BD70B582B00C461646684611461C
:100630004FF0080219F0BCFC009809F0E9FC40F208
:100640001023C2F200031860019809F0E1FC014692
:1006500040F21420C2F2000001600B2C00F2DD8099
:10066000DFE804F00613202D3A4754616EA2AFBCB8
:1006700040F21020C2F20000006818F05FFD40F266
:100680002423C2F200031860B4E040F21024C2F246
:100690000004206818F000FA40F22422C2F200029E
:1006A0001060A7E040F21023C2F20003186818F0AF
:1006B000EBFD40F22421C2F2000108609AE040F212
:1006C0001020C2F20000006818F016FC40F224224C
:1006D000C2F2000210608DE040F21021C2F200016F
:1006E000086818F0DBFB40F22424C2F2000420600A
:1006F00080E040F21022C2F20002106818F020FCE4
:1007000040F22423C2F20003186073E040F210208C
:10071000C2F20000006818F0EBFE40F22424C2F29E
:100720000004206066E040F21023C2F20003186863
:1007300018F04EFE40F22421C2F20001086059E098
:1007400040F21025C2F20005286817F049FD044662
:100750000D464FF000024FF0000318F0B9F860B1F9
:10076000204629464FF000024FF00003C3F6E07325
:1007700017F090FD17F0D2FC0BE0204629464FF011
:1007800000024FF00003C3F6E07317F081FD17F08D
:10079000C5FC07EE100AF8EEC77A40F22422C2F236
:1007A0000002C2ED007A25E040F21020C2F2000003
:1007B000006818F03DFE40F22421C2F200010860FA
:1007C00018E040F21024C2F20004206818F0AEFADB
:1007D00040F22423C2F2000318600BE040F2102123
:1007E000C2F20001086818F0E7F940F22422C2F2D0
:1007F0000002106040F22421C2F20001086809F0F2
:10080000DDFB00904FF000040194304669464FF044
:10081000080219F0CDFB204601E04FF0140002B0B1
:1008200070BD00BF4BF6D043C0F603031A684EF606
:100830000C50CEF200000260FEE700BF08B5FFF7E3
:10084000F1FF00BF51E8002FBFF35F8F41E80003C5
:10085000012B3FF4F7AF1046704700BF13461A460E
:100860002DE9F00F0B460C460D460E460F46884606
:1008700089468A468B46092AC0F00780A0E8F80F0F
:10088000A2F10902092ABFF4F9AF4FF0080303FBF4
:1008900002F2144B1A44974600F020B800BF00BF84
:1008A000046000F01BB800BF80E8300000F016B80C
:1008B00080E8700000F012B880E8F00000F00EB898
:1008C00080E8F00100F00AB880E8F00300F006B814
:1008D00080E8F00700F002B880E8F00FBDE8F00F04
:1008E0007047134698080208EFF311804FF080011B
:1008F00081F3118870474FF0000000BF80F311882A
:10090000704700BF30B440F20003C0F6000340F26D
:100910008812C0F60002D01A4FEAA001B1F5C47FD8
:1009200004D81346264A9A4201D324E0FEE7254D17
:10093000254C601B20F003054FF0000340F200023D
:10094000C2F2000240F20001C0F6000105F104000D
:10095000C5F380045D589D5003F10403834226D102
:1009600009E05C589C5003F104035C58D45003F137
:1009700004038342F5D14EF60853CEF2000340F251
:100980000002C2F200021A604FF0B501CBF26B1107
:1009900043F25850C2F2000001604EF61453CEF2FA
:1009A00000031A6842F01001196030BC7047002C37
:1009B000D7D05C589C5003F104038342D1D1DAE7CD
:1009C00000000008040000088B01000810B4034672
:1009D00000283ED002F1100440F20000C2F20000F4
:1009E00040F82430002A0ADA12F10C0F35DB02F14C
:1009F0000C024EF61850CEF2000011542DE04EF2CB
:100A00000014CEF200040F299CBF0901C9B24EF2B6
:100A10000043CEF20003D1541146002AB8BF02F1C0
:100A20001F014FEA611004EB80014FF01F03C8F271
:100A300000031340002B05DA03F1FF3262F01F03BD
:100A400003F1010358B24FF0010202FA00F30B6008
:100A500003E0002AC8DB024CD5E710BC704700BF9A
:100A600080E100E01EF0040F0CBFEFF30880EFF30D
:100A7000098020E9F00F00F001B800BF10B502684E
:100A800043F20C53C2F200031A6041685960826855
:100A90009A60C168D96002691A61416959618269C5
:100AA0009A61C169D961026A1A62416A5962826AAD
:100AB0009A62C16AD962026B1A63416B5963826B95
:100AC0009A63C16BD96300F1400018644EF6285058
:100AD000CEF2000002685A641BF04AF8002800F0C9
:100AE000FB814BF6D440C0F603001BF047F84EF6EE
:100AF0002C54CEF200042368002B05DA4BF6E440B8
:100B0000C0F603001BF03AF84EF62C51CEF200016D
:100B1000086810F0020F05D04BF6F440C0F6030051
:100B20001BF02CF84EF62852CEF200025478002C1E
:100B300072D04BF60C50C0F603001BF01FF84EF6B7
:100B40002853CEF20003597811F0010F05D04BF66F
:100B50001C50C0F603001BF011F84EF62850CEF2E0
:100B60000000427802F00204E3B22BB14BF63C5095
:100B7000C0F603001BF002F84EF62851CEF2000139
:100B8000487800F00402D4B22CB14BF66050C0F6A5
:100B900003001AF0F3FF4EF62853CEF20003597803
:100BA00001F00800C2B22AB14BF68450C0F603002F
:100BB0001AF0E4FF4EF62854CEF20004637803F0F6
:100BC0001001C8B228B14BF6A450C0F603001AF0C9
:100BD000D5FF4EF62852CEF20002547804F02003DE
:100BE000D9B229B14BF6C450C0F603001AF0C6FFC3
:100BF0004EF62850CEF20000427802F08004E3B2B4
:100C000053B14EF63851CEF2000109684BF6E4506C
:100C1000C0F603001AF0B2FF4EF62850CEF20000E4
:100C2000428894B2002C5ED04BF60460C0F60300FC
:100C30001AF0A4FF4EF62853CEF20003598811F0A3
:100C4000010F05D04BF61460C0F603001AF096FFB2
:100C50004EF62850CEF20000428802F00204A3B201
:100C60002BB14BF64060C0F603001AF087FF4EF63A
:100C70002851CEF20001488800F0040294B22CB151
:100C80004BF66460C0F603001AF078FF4EF6285366
:100C9000CEF20003598801F0080082B22AB14BF667
:100CA000A460C0F603001AF069FF4EF62854CEF295
:100CB0000004638803F4807188B228B14BF6D460D5
:100CC000C0F603001AF05AFF4EF62852CEF2000288
:100CD000548804F4007399B229B14BF6F060C0F661
:100CE00003001AF04BFF4EF62850CEF200000278B7
:100CF000002A63D04BF60870C0F603001AF03EFFDE
:100D00004EF62854CEF20004237813F0010F05D0DC
:100D10004BF61870C0F603001AF030FF4EF628515B
:100D2000CEF20001087800F00202D4B22CB14BF6EA
:100D30003870C0F603001AF021FF4EF62853CEF2A9
:100D40000003197801F00800C2B22AB14BF65070C6
:100D5000C0F603001AF012FF4EF62854CEF200043B
:100D6000237803F01001C8B228B14BF67470C0F6B6
:100D700003001AF003FF4EF62852CEF20002147858
:100D800004F02003D9B229B14BF69870C0F60300E5
:100D90001AF0F4FE4EF62850CEF20000027802F06F
:100DA0008004E3B253B14EF63451CEF2000109682B
:100DB0004BF6B870C0F603001AF0E0FE43F20C5494
:100DC000C2F20004216A4BF6E470C0F603001AF088
:100DD000D5FE616A4BF6F870C0F603001AF0CEFE3D
:100DE000A16A4CF20C00C0F603001AF0C7FEE16ADB
:100DF0004CF22000C0F603001AF0C0FE21684CF24D
:100E00003400C0F603001AF0B9FE61684CF24800E5
:100E1000C0F603001AF0B2FEA1684CF25C00C0F606
:100E200003001AF0ABFEE1684CF27000C0F603005C
:100E30001AF0A4FE21694CF28400C0F603001AF0F7
:100E40009DFE61694CF29800C0F603001AF096FE10
:100E5000A1694CF2AC00C0F603001AF08FFEE16904
:100E60004CF2C000C0F603001AF088FE216B4CF271
:100E7000D400C0F603001AF081FE216C4CF2E800A9
:100E8000C0F603001AF07AFE616B4CF2FC00C0F66B
:100E900003001AF073FEA16B4CF22010C0F60300A1
:100EA0001AF06CFE43F25450C2F2000002684CF299
:100EB0004410C0F60300114612681AF05FFE40F6B7
:100EC0003C13C2F200031A684CF25C10C0F6030037
:100ED000114612681AF052FEFFF7B0FC10BD00BFB9
:100EE00000B507F011FA002808BF5DF804FBEFF326
:100EF0000981EFF3118221E9F40F5DF804EB1EF094
:100F0000100F08BF21ED108A41F804ED0B4C226848
:100F1000002A18BF516007F069FA2268516851F839
:100F200004EB1EF0100F08BFB1EC108AB1E8F40F0B
:100F300082F3118881F3098870470000543500203E
:100F400008B540F6E160C0F602004FF0FF016FF017
:100F50000102FFF73BFD08BDF8B507460C461E46EB
:100F60000799089D14F0030F00D0FEE722B1A4EB0F
:100F70008500A0F1480401E004F14800012D01D8EA
:100F8000A16205E02A4602F043F9A7EB8507A762B4
:100F90004FF0000363604FF01130E0624FF02231F8
:100FA00021634FF0333262634FF04433A3604FF05C
:100FB0005530E0604FF0663121614FF07732626169
:100FC0004FF08833A3614FF09930E0614FF0AA31C0
:100FD00021624FF0BB3262624FF0CC33A363E66311
:100FE000069820644FF0807161646FF00202226005
:100FF00005F11200F8BD00BF62B64EF60453CEF202
:1010000000031A6842F08050186000BF4FEA0010D9
:101010004CF27413C0F603031A584CF6A041C0F604
:10102000030151F82200704738B504460D46FFF71A
:10103000EDFF4CF27413C0F6030303EB0414616874
:10104000012902D0022903D101E0856038BD456144
:1010500038BD00BF10B540F20401C4F202010C68B3
:101060004CF25032C0F60302136824EA03044CF237
:101070004423C0F60303186804430C6040F20441A3
:10108000C4F202010C68506824EA00045868044362
:101090000C6040F60401C4F202010C68906824EA76
:1010A0000004986804430C6040F60441C4F2020155
:1010B0000C68D06824EA0004D86804430C6041F24C
:1010C0000401C4F202010868126920EA02001B69E7
:1010D00040EA03040C6041F20441C4F202010868D2
:1010E000086041F60403C4F202031A681A6041F66C
:1010F0000444C4F202042168216042F20400C4F2F4
:1011000002000368036040F20C01C4F202010C68A3
:101110004CF2A032C0F60302106824EA00044CF23C
:10112000F413C0F60303186804430C6040F20C414A
:10113000C4F202010C68506824EA000458680443B1
:101140000C6040F60C01C4F202010C68906824EABD
:101150000004986804430C6040F60C41C4F202019C
:101160000C68D06824EA0004D86804430C6041F29B
:101170000C01C4F202010868126920EA02001B692E
:1011800040EA03040C6041F20C41C4F20201086819
:10119000086041F60C03C4F202031A681A6041F6B3
:1011A0000C44C4F202042168216042F20C00C4F233
:1011B0000200036803604CF2A824C0F6030422680E
:1011C00040F21401C4F202010A60606840F2144364
:1011D000C4F202031860A26840F61401C4F20201CE
:1011E0000A60E06840F61443C4F202031860246900
:1011F00041F21402C4F2020214604FF0000141F205
:101200001440C4F20200016041F61403C4F2020368
:10121000196041F61444C4F20204216042F214023F
:10122000C4F20202116040F20001C4F202010C6833
:101230004CF27432C0F60302106824EA00044CF247
:10124000FC23C0F60303186804430C6040F200411D
:10125000C4F202010C68506824EA00045868044390
:101260000C6040F60001C4F202010C68906824EAA8
:101270000004986804430C6040F60041C4F2020187
:101280000C68D06824EA0004D8682043086041F262
:101290000001C4F202010868126920EA02001B6919
:1012A0001843086041F20041C4F202010A680A6072
:1012B00041F60003C4F202031868186041F60041C9
:1012C000C4F202010A680A6042F20003C4F2020397
:1012D000186818604FF0010004F0CEFB10BD00BF8D
:1012E00008B543F63002C4F2020213686FEA5320D5
:1012F0006FEA4021116043F62003C4F201031A682B
:1013000042F001001860FFF7A5FE08BD2DE9F001CD
:101310009DF814709DF81860079D4CF22024C0F6CB
:10132000030454F820004FEA4104FF2F12D0D0F8F4
:101330000C804CF2182CC0F6030C1CF8077007FA4E
:1013400004FC4FF0030707FA04F728EA07074CEA02
:101350000707C760FF2B10D0D0F804C04CF2A427B9
:10136000C0F60307FF5C07FA01F74FF0010303FA29
:1013700001F32CEA03033B434360FF2E0FD0876841
:101380004CF29C33C0F603039E5D06FA04F64FF060
:10139000030303FA04F327EA030333438360B5F13D
:1013A000FF3F16D04FEAD10303F1080350F8236042
:1013B00001F007014FEA810105F00F0505FA01F57B
:1013C0004FF00F0707FA01F126EA0101294340F81F
:1013D0002310FF2A10D001684CF29833C0F60303A3
:1013E0009B5C03FA04F34FF0030202FA04F421EACF
:1013F000040143EA01040460BDE8F001704700BF46
:101400002DE9F007079F089E099D4CF22024C0F6A5
:10141000030454F820004FEA41044FEAD10801F0D8
:10142000070C4FEA8C0C6FB1D0F80C9029FA04FA33
:101430000AF003094CF26C2AC0F6030A1AF8099064
:1014400087F8009053B1476827FA01F101F00101D4
:101450004CF27027C0F60307795C197056B18368A7
:1014600023FA04F303F003034CF26821C0F60301EE
:10147000CB5C337045B108F1080850F8281021FA08
:101480000CFC0CF00F032B6052B1006820FA04F43E
:1014900004F003044CF21C21C0F603010B5D137031
:1014A000BDE8F007704700BF4CF27423C0F6030399
:1014B00053F820100A684CF2CC23C0F6030353F80B
:1014C00020100A404CF22033C0F6030353F82000EA
:1014D000824214BF00200120704700BF4CF220233D
:1014E000C0F6030353F82000006970474CF2CC2388
:1014F000C0F6030353F820307BB139B14CF2C4116C
:10150000C0F6030151F82020136070474CF294128A
:10151000C0F6030252F82000036070473A2800F238
:10152000938000EB80004CF2C433C0F6030353F801
:10153000202002F1FF300D2800F28680DFE800F065
:10154000071019222B343D464F58616A737C43F6CD
:101550004400C4F20200036861F3000303607047B3
:1015600043F64003C4F202031A6861F300021A60F2
:10157000704743F64003C4F20203186861F3410068
:101580001860704743F64000C4F20200026861F33D
:1015900082020260704743F64000C4F20200036812
:1015A00061F3C3030360704743F64003C4F20203D0
:1015B0001A6861F304121A60704743F64003C4F2DC
:1015C0000203186861F345101860704743F6440041
:1015D000C4F20200026861F341020260704743F600
:1015E0004400C4F20200036861F3104303607047D3
:1015F00043F64403C4F202031A6861F351421A60CD
:10160000704743F64403C4F20203186861F3924042
:101610001860704743F64000C4F20200026861F3AC
:1016200086120260704743F64000C4F2020003686D
:1016300061F3C7130360704743F64003C4F202032B
:101640001A6861F308221A60704700BF00EB80003F
:101650004CF2C433C0F6030353F820204CF6E441A7
:10166000C0F6030151F82200704700BF2DE9F84F82
:1016700004468A46914698469DF928709DF92C604B
:101680009DF930503A2800F2B680FFF7DFFF04EBF7
:1016900084024CF2C433C0F6030303EB82035A689E
:1016A000022A94BF8369C369016A02F1FF3CBCF15D
:1016B000030F2ED8DFE80CF0021802186FF30103B5
:1016C000BAF1000FC8BF6AF38203B9F1000FC8BFB7
:1016D00069F3C303B8F1000FC8BF68F30613002F06
:1016E00017DD67F3C71314E06FF30923BAF1000F96
:1016F000C8BF6AF38A23B9F1000FC8BF69F3CB23CF
:10170000B8F1000FC8BF68F30E33002FC8BF67F3EE
:10171000CF3302F1FF37032F44D8DFE807F002147C
:101720002638332C04D1002E06DD66F3820103E057
:10173000002EC8BF66F30001002DC8BF65F341014C
:101740006FF3C30130E0362C04D1002E06DD66F3C2
:10175000861103E0002EC8BF66F30411002DC8BF38
:1017600065F345116FF3C7111EE0382C04D1002E2C
:1017700006DD66F38A2103E0002EC8BF66F3082168
:10178000002DC8BF65F349216FF3CB210EE0002E79
:10179000C8BF66F30C31002DC8BF65F34D316FF340
:1017A000CF3103E0022A01D8836100E0C361016206
:1017B00004EB84044CF2C430C0F6030050F824302B
:1017C000012B02D0082B16D10BE04CF66003C0F6BB
:1017D00003031A6840F24401C4F201010A60BDE843
:1017E000F88F4CF66002C0F60302116840F24440E4
:1017F000C4F201000160BDE8F88F00BF38B50446AF
:101800000D46FFF723FF04EB84014CF2C433C0F60E
:10181000030303EB8104626802F1FF3103290AD854
:10182000DFE801F002040608456338BD856338BD72
:10183000C56338BD056438BD40F22823C2F20003F9
:1018400018684FF000020261016801F01003002BDC
:101850000CBF01204FF0FF3040F22C23C2F20003F6
:101860001A8810FA82F188B2188070472DE9F04F7B
:1018700089B0154640F22823C2F200034FF000025F
:101880001A604FEA01104CF66804C0F603042458AD
:10189000142900F2F480092C00F2F4804CF6D013E5
:1018A000C0F6030353F82430002B00F0EE804FEA1B
:1018B00005124CF66800C0F603008258944240F0CE
:1018C000E78004F1FF36072E4DD8DFE806F0340438
:1018D000101C284C4C4043F64007C4F202073868FD
:1018E00040F001023A604FF0000605963EE043F6F4
:1018F0004007C4F20207386840F002023A604FF035
:101900000106059632E043F64007C4F20207386844
:1019100040F004023A604FF00106059626E043F6D7
:101920004007C4F20207386840F008023A604FF0FE
:10193000000605961AE043F64407C4F20207386829
:1019400040F001023A604FF0010605960EE043F6C2
:101950004407C4F20207386840F002023A604FF0D0
:101960000106059602E04FF00107059740F2282096
:101970008246C2F2000ACAF800304CF66809C0F686
:10198000030909EB011898F804B0D8F8081004917D
:101990000DF11F0300934FF0000601960296584682
:1019A00032460DF11E03FFF72BFD9DF81E309DF80A
:1019B0001F2000924FF003070197D8F80C00029007
:1019C000584604993A46FFF7A1FC09EB051595F82E
:1019D0000490D5F808800DF11F0100910196029640
:1019E0004846414632460DF11E03FFF709FD9DF8BA
:1019F0001F3000930197EA680292484641463A46F2
:101A00003346FFF783FCDAF800104CF6F810C0F606
:101A1000030003680B604CF66402C0F60302106812
:101A200088604CF6CC13C0F603031A688A610E6214
:101A30006FF07F40C862059B93B14CF6C812C0F6A8
:101A400003021068C86041F63900C0F602004FF08A
:101A50000F014CF6B813C0F603031A57FEF7B6FF92
:101A600040F22821C2F2000108684FF000028262B1
:101A7000036843F0010101604FF001000AE04FF0FC
:101A8000000007E04FF0000004E04FF0000001E02C
:101A90004FF0000009B0BDE8F08F00BF40F22823EE
:101AA000C2F200031B689BB1A8B91A686FF3000269
:101AB0001A604FF00000586240F22C21C2F200017F
:101AC00008801A6842F0010018604FF0010070476A
:101AD0004FF0000070474FF00000704710B483B023
:101AE00040F22823C2F200031B6803B310BB40F28C
:101AF0002C22C2F20002586A148840EA0440019085
:101B000000BF00BF00BF00BF00BF586A148840EA92
:101B100004400090019C00988442ECD1DDED017AF4
:101B2000B8EEE70A81ED000A4FF0010004E04FF043
:101B3000000001E04FF0000003B010BC704700BF90
:101B400040F22823C2F200031B689BB1A8B91A68AF
:101B50006FF300021A6059624FEA114140F22C20E3
:101B6000C2F2000001801A6842F0010119604FF0D2
:101B7000010070474FF0000070474FF000007047C1
:101B800043F67403C4F20203186847F20402C4F275
:101B90000002136840F22E22C2F200024FF0000150
:101BA000117013F0010F04D010464FF004020270C0
:101BB0003EE04FEA106212F0600F07D040F22E2193
:101BC000C2F200014FF020030B7031E002F004017B
:101BD000C9B239B140F22E20C2F200004FF04002EB
:101BE000027025E0C3F3400343EAD06010F0010F18
:101BF00007D040F22E21C2F200014FF080030B709B
:101C000016E002F01001CBB23BB140F22E20C2F23E
:101C100000004FF0010202700AE002F00202D0B2AE
:101C200030B140F22E21C2F200014FF002030B70DE
:101C300043F67401C4F202010B6843F0807008603F
:101C400047F20001C4F200010A6842F008030B6089
:101C500043F25450C2F20000016840F23022C2F256
:101C600000021160704700BF40F22E23C2F2000351
:101C70001878704708B547F61021C1F6FF714FF08C
:101C80000C0218F095F94FF00C0008BD00B583B0B8
:101C900043F64003C4F202031A6842F08050186011
:101CA00047F20001C4F200010B6843F480720A603D
:101CB0000DF107006946FEF743FB43F67001C4F2DD
:101CC00002010A684CF62023C0F6030319684A4053
:101CD0004CF61823C0F6030319680A421FD1F0B16D
:101CE00042F63C00C4F2000002684FEAC2534FEAD9
:101CF000D3510098814212D142F63C02C4F2000254
:101D00001368C3F3C0319DF80700814207D140F248
:101D10003423C2F200034FF001021A700BE04CF6BC
:101D20000420C0F603004FF0070142F20D02C0F696
:101D3000020206F037F903B000BD00BF70B50646D9
:101D400040F23424C2F2000442F60C05C4F200054D
:101D500003E000F0C9FA06F031F92378002BF8D03F
:101D6000286810F0200FF4D042F60001C4F2000100
:101D70000A6842F60403C4F200031B68C2F30210AF
:101D800000EB800102F00F0000EB41013160C2F373
:101D9000023000EB8001C2F3032000EB41017160CF
:101DA000C2F3015000EB8001C2F3034202EB410099
:101DB000B060C3F3072101F0E002E02A14BFC3F3CF
:101DC00042320022B261C3F3011000EB800203F043
:101DD0000F0101EB4200F060C3F300324FEA8201D1
:101DE0008818C3F3032202EB400101F1FF30306198
:101DF000C3F3035202EB8201C3F3034303EB41003D
:101E000000F16400706170BD70B58AB0014601A830
:101E10004FF0240218F0CCF801A817F0EFFE059C53
:101E200004F10104E4B2019A46F26763C6F2666304
:101E300083FB02104FEAE271C1EBA0054FF00006F0
:101E400065F3061605EB8500A2EB400262F303067C
:101E5000029D83FB05104FEAE571C1EBA00262F31E
:101E60000E3602EB8200A5EB400565F30B26039AC4
:101E700083FB02034FEAE271C1EBA30060F3155646
:101E800000EB8005A2EB450262F31346079B13B1FA
:101E900003F0070101E04FF007014FF0000561F387
:101EA0004F35049946F26762C6F2666282FB0130E2
:101EB0004FEAE173C3EBA00060F3051500EB80036C
:101EC000A1EB430161F303054CF6CD40CCF6CC40C9
:101ED000A0FB04034FEAD30161F30C3501EB810051
:101EE000A4EB400464F30B25069982FB01304FEA12
:101EF000E173C3EBA00382FB03024FEAE370C0EB84
:101F0000A20202EB8200A3EB400262F3175503EB3F
:101F10008303A1EB430161F3134540F23420C2F285
:101F20000000027852B940F23424C2F2000400F0FA
:101F3000DBF906F043F82378002BF8D042F62401B1
:101F4000C4F200014FF0CA0008604FF053020A606B
:101F500042F60C03C4F20003196841F080001860D7
:101F60001A46136813F0400FFBD042F60001C4F28A
:101F700000010E6042F60400C4F20000056042F663
:101F80000C03C4F200031A686FF3C7121A6042F61A
:101F90002401C4F200014FF0FF0008600AB070BDD8
:101FA00070B506460D46B1F5007F2ED242F60C0301
:101FB000C4F20003186810F4803F09D042F60C0404
:101FC000C4F2000405F0FAFF216811F4803FF9D152
:101FD00042F62403C4F200034FF0CA021A604FF025
:101FE000530018604FF0000242F61801C4F20001DD
:101FF0000A6065F3080266F3CF3242F63C00C4F291
:10200000000002604FF0FF021A6070BD30B583B06F
:102010000DF107006946FEF793F905464CF61C23BF
:10202000C0F603031A6843F67000C4F202000260AF
:102030004CF62021C0F603010B680360026812F021
:10204000020F09D143F67004C4F2020405F0B6FF92
:10205000206810F0020FF9D042F62401C4F200010A
:102060004FF0CA030B604FF053020A6042F60C00B7
:10207000C4F20000016841F080030360026812F0BE
:10208000400F09D142F60C04C4F2000405F096FF9B
:10209000206810F0400FF9D04CF6FC11C0F6030197
:1020A0000A6842F61003C4F200031A601A604CF684
:1020B0000020C0F60300016842F60802C4F20002E4
:1020C000116042F60C03C4F2000318686FF3C710E6
:1020D000186042F62401C4F200014FF0FF020A60CA
:1020E0002DB19DF807000099FFF75AFF04E04FF06B
:1020F00000000146FFF754FF40F23423C2F2000310
:102100004FF00100187003B030BD00BF00000000A8
:1021100010B542F20803CEF204031A6842F0100030
:10212000186042F2C910C0F602004FF00F014FF0E4
:102130003602FEF74BFC43F64001C4F202010C6884
:1021400044F010030B6041F20004C4F200044CF6AA
:102150002422C0F60302106820604CF6A841C0F6A5
:102160000301886915F06EFF15A3D3E9002316F06B
:10217000D5F94FF000024FF00003C3F6F07316F0EC
:1021800087F815F0F3FF41F22C03C4F20003188026
:1021900041F22800C4F200004FF0000202804CF629
:1021A0002821C0F60301086841F20C03C4F20003C1
:1021B0001860228842F00101218010BDAFF3008039
:1021C0002D431CEBE2362A3F684620F007018D467E
:1021D00001B541F21003C4F200034FF000021A608F
:1021E00006F0B6FBBDE801408546704770B5044671
:1021F000B0F5CC7F2FD940F23233984216D940F255
:102200006560844215D940F6CB418C4214D941F621
:102210009712944213D943F22F36B44212D946F2A0
:102220005F639C4298BF06250ED90FE04FF0010571
:102230000AE04FF0020507E04FF0030504E04FF01D
:10224000040501E04FF00505072D06D1FEF7F6FA6B
:102250004FF0070501E04FF00005FEF745FB06468D
:1022600004EB84044FEAC4004CF62C21C0F60301B1
:1022700051F83520B0FBF2F39CB2012C05D9B4F52E
:10228000805F04D3FEF7DAFA01E04FF0020443F274
:102290000000C4F2000045F2555101604CF62C22BA
:1022A000C0F6030202EBC5052B7943F20401C4F228
:1022B00000010B6043F20802C4F2000214604AF607
:1022C000AA2303603046FEF719FB70BD08B543F240
:1022D0000003C4F200034CF6CC421A604FF0C80071
:1022E000FFF784FF08BD00BF43F20003C4F2000300
:1022F0004AF6AA221A60704710B5044643F210034A
:10230000C4F20003186810F0010F74D04FF03200CF
:1023100007F0D6FD43F21001C4F200010A6812F082
:10232000010F68D04FF0320007F0CAFD43F21003EE
:10233000C4F20003186810F0010F5CD04FF03200B7
:1023400007F0BEFD43F21001C4F200010A6812F06A
:10235000010F50D04FF0320007F0B2FD43F21003EE
:10236000C4F20003186810F0010F44D04FF032009F
:1023700007F0A6FD43F21001C4F200010A6812F052
:10238000010F38D04FF0320007F09AFD43F21003EE
:10239000C4F20003186810F0010F2CD04FF0320087
:1023A00007F08EFD43F21001C4F200010A6812F03A
:1023B000010F20D04FF0320007F082FD43F21003EE
:1023C000C4F20003186810F0010F14D04FF032006F
:1023D00007F076FD43F21001C4F200010A6812F022
:1023E000010F08D04FF0320007F06AFD43F21003EE
:1023F000C4F200031B682046FFF7F8FE10BD00BFC3
:1024000002469CF8043043B1DCF8000040B140F2D1
:10241000C021C2F2000141F82200DCF8000050B9EE
:1024200040F2C023C2F2000353F8220049F64042B2
:10243000002808BF104670474FF0010303FA00F070
:1024400010F4E26F0CBF00200120704770B50D46FC
:102450004CF69C23C0F6030353F82040002C45D0D3
:1024600000EB800040F23826C2F2000606EBC00600
:1024700030464FF0000105F08DF9122D07D142F2E0
:102480000431C4F201010A6842F480030B60606BFE
:1024900065F304006063E36C4FF0050007F010FD86
:1024A000A16841F08042A260236813F0020FFBD0C4
:1024B000E46C122D16D142F20430C4F2010001681E
:1024C0006FF39651016042F20002CEF204021368EB
:1024D0004FEA03504FEA105140F2194291420CBFAB
:1024E000A4006400304605F063FA01E04FF0FF34C9
:1024F000204670BDF8B504460F464CF68823C0F65A
:10250000030303EB80056E88002E53D013F82000E0
:10251000012803D16878FFF799F801E04FF0000037
:102520005FB940F2B020C2F2000000EB84044FF02B
:10253000000121604FF000012BE0BE420BD840F2B9
:10254000B022C2F2000202EB84044FF07E532360FB
:102550004FF6FF711DE02A78012A0CBFC16A40F6D0
:10256000FF7140F2B023C2F2000303EB840406EED5
:10257000907AB8EE667A00EE101AF8EE407AC7EE5E
:10258000270AC4ED000A06F1FF3007FB0101B1FB89
:10259000F6F12A78012A03D16878FFF72FF9F8BD00
:1025A000022A07D1687840F6FF73994228BF19467E
:1025B000FEF73AFDF8BD00BF38B52DED028B04469D
:1025C00008EE101A4CF68825C0F6030505EB8005C9
:1025D000F7EE007AB4EEE78AF1EE10FA09DC08466D
:1025E00016F0CAF900289FED260A18BFB0EE408AFF
:1025F00001E0B7EE008A2B78012B1CD16878FFF739
:1026000025F8D0ED0B1A6D78B8EE612A62EE082A33
:1026100012EE900A15F0E4FD4FF000024FF00003B7
:10262000C3F6E07315F036FE15F0A0FD014628460E
:10263000FFF7E4F818E0022B16D16D78DFED110AF0
:1026400028EE201A11EE100A15F0CAFD4FF0000214
:102650004FF00003C3F6E07315F01CFE15F086FD85
:1026600001462846FEF7E0FC40F2B020C2F200002E
:1026700000EB840484ED008ABDEC028B38BD00BF02
:102680000000000000F07F4510B54FF000044FF04F
:1026900000002146FFF790FF4FF001002146FFF7B1
:1026A0008BFF4FF002002146FFF786FF4FF003003B
:1026B0002146FFF781FF40F20C03C4F202031A68BF
:1026C0001A6040F20C40C4F202000168016040F65A
:1026D0000C03C4F202031A684CF6D820C0F60300BB
:1026E000816822EA01024CF66420C0F6030081688A
:1026F0000A431A6040F60C43C4F202031A681A60D7
:1027000041F20C00C4F202000168016041F20C4386
:10271000C4F202031A681A6041F60C00C4F2020007
:102720000168016041F60C43C4F202031A681A60A2
:1027300042F20C00C4F202000168016040F20003A2
:10274000C4F202031A681A6040F20040C4F20200A8
:102750000168016040F60003C4F202031A684CF6F7
:102760000830C0F60300816822EA01024CF6A82076
:10277000C0F6030081680A431A6040F60043C4F2C1
:1027800002031A681A6041F20000C4F202000168F4
:10279000016041F20043C4F202031A681A6041F674
:1027A0000000C4F202000168016041F60043C4F277
:1027B00002031A681A6042F20000C4F202000168C3
:1027C000016010BD08B502280ED84CF60433C0F6DF
:1027D0000303195CFF290AD04CF63032C0F603021D
:1027E000105CFFF733FE08BD4FF0FF3008BD4FF01F
:1027F000FF3008BD10B50446FFF7E4FF07EE900A6E
:10280000B8EE677A4CF60433C0F60303185D11285E
:102810000BD147F62A21C1F6FF710A8801EE102A72
:10282000F8EEC11AC1EE870A03E09FED030AC7EE76
:10283000000A10EE900A10BD00F07F4540F2B02370
:10284000C2F2000303EB80000068704738B50D4604
:10285000044600B30E2801D9FDF7F0FF4CF6A8435B
:10286000C0F6030353F8240055B1B0FBF5F14FEA6D
:10287000114202F10103B0FBF3F0B0FBF5F502E009
:102880004FF000052A464CF6E441C0F6030151F82A
:1028900024309A62DD6238BD10B582B000918DF8A7
:1028A0000420042840F0E2804FF00000FFF7C4FD50
:1028B00048B1EC464FF00000FFF7A2FD01464FF093
:1028C0000000FFF7C3FF4FF00100FFF7B5FD48B16F
:1028D000EC464FF00100FFF793FD01464FF0010079
:1028E000FFF7B4FF4FF00200FFF7A6FD48B1EC463A
:1028F0004FF00200FFF784FD01464FF00200FFF7A2
:10290000A5FF4FF00300FFF797FD48B1EC464FF0ED
:102910000300FFF775FD01464FF00300FFF796FF38
:102920004FF00400FFF788FD48B1EC464FF004007B
:10293000FFF766FD01464FF00400FFF787FF4FF0F9
:102940000500FFF779FD48B1EC464FF00500FFF7B1
:1029500057FD01464FF00500FFF778FF4FF00600E6
:10296000FFF76AFD48B1EC464FF00600FFF748FD5F
:1029700001464FF00600FFF769FF4FF00700FFF731
:102980005BFD48B1EC464FF00700FFF739FD01460B
:102990004FF00700FFF75AFF4FF00800FFF74CFD1C
:1029A00048B1EC464FF00800FFF72AFD01464FF012
:1029B0000800FFF74BFF4FF00900FFF73DFD48B15E
:1029C000EC464FF00900FFF71BFD01464FF00900F0
:1029D000FFF73CFF4FF00A00FFF72EFD48B1EC4631
:1029E0004FF00A00FFF70CFD01464FF00A00FFF719
:1029F0002DFF4FF00B00FFF71FFD48B1EC464FF0E5
:102A00000B00FFF7FDFC01464FF00B00FFF71EFF28
:102A10004FF00C00FFF710FD48B1EC464FF00C00F2
:102A2000FFF7EEFC01464FF00C00FFF70FFF4FF0F1
:102A30000D00FFF701FD48B1EC464FF00D00FFF728
:102A4000DFFC01464FF00D00FFF700FF4FF00E00D6
:102A5000FFF7F2FC48B3EC464FF00E00FFF7D0FC56
:102A600001464FF00E00FFF7F1FE1EE04CF6882302
:102A7000C0F6030313F82010012916D14CF6882262
:102A8000C0F6030202EB8000447804EB84034CF2AE
:102A9000C431C0F6030151F82340EC462046FFF74D
:102AA000AFFC01462046FFF7D1FE02B010BD00BFCB
:102AB00070B584B040F23825C2F200054CF6D4243B
:102AC000C0F603042846214604F04CFE05F1280018
:102AD000214604F047FE05F15000214604F042FE75
:102AE00043F64403C4F202031A6842F4807018608B
:102AF000196841F400761E604CF60035C0F60305F7
:102B00002C6842F20433C4F201031C604CF6CC2260
:102B1000C0F60302106842F20401C4F20101086029
:102B200042F20416C4F2010630604CF69825C0F655
:102B300003052C6842F20C03C4F201031C6042F24C
:102B40000C12C4F2010214604CF62C30C0F60300E3
:102B5000016842F21006C4F20106316042F210151B
:102B6000C4F2010529604CF63434C0F6030423682E
:102B700042F22C02C4F20102136042F22C10C4F2A1
:102B8000010003604CF6D021C0F603010E6842F24A
:102B90000805C4F201052E6042F20814C4F20104D3
:102BA00026604FF016004FF00101FEF7B7FC4FF022
:102BB00008004FF00101FEF7B1FC4FF00C004FF0A0
:102BC0000101FEF7ABFC4FF005004FF00101FEF7ED
:102BD000A5FC4FF0000400944FF00106019602940A
:102BE0004FF01600214632464FF00603FEF73EFD39
:102BF0004CF2C435C0F6030595F8C401D5F8C811E8
:102C000000940194D5F8C03102934FF0030223469B
:102C1000FEF77CFB0094019602944FF008002146D9
:102C200032464FF00603FEF721FD95F8AC00D5F8CB
:102C3000B01000940194D5F8A82002924FF003023E
:102C40002346FEF763FB0094019602944FF00C00BC
:102C5000214632464FF00603FEF708FD95F8FC00CA
:102C6000D5F8001100940194D5F8F83002934FF094
:102C700003022346FEF74AFB0094019602944FF0AC
:102C80000500214632464FF00603FEF7EFFC95F8AB
:102C90007000696F00940194ED6E02954FF003028D
:102CA0002346FEF733FB4FF0040021462246FFF790
:102CB000F3FD4FF0000520462946FFF77DFC304626
:102CC0002946FFF779FC4FF002002946FFF774FC14
:102CD0004FF003002946FFF76FFC3046FFF7ACFBCF
:102CE00050B14CF6E440C0F6030041684CF6FC22BB
:102CF000C0F6030213680B604FF00200FFF79CFB65
:102D000050B14CF6E440C0F6030081684CF6FC225A
:102D1000C0F6030213680B604FF00300FFF78CFB53
:102D200050B14CF6E440C0F60300C1684CF6FC22FA
:102D3000C0F6030213680B604FF00400FFF77CFB42
:102D400050B14CF6E440C0F6030001694CF6FC2299
:102D5000C0F6030213680B604FF00500FFF76CFB31
:102D600050B14CF6E440C0F6030041694CF6FC2239
:102D7000C0F6030213680B604FF00600FFF75CFB20
:102D800050B14CF6E440C0F6030081694CF6FC22D9
:102D9000C0F6030213680B604FF00700FFF74CFB0F
:102DA00050B14CF6E440C0F60300C1694CF6FC2279
:102DB000C0F6030213680B604FF00800FFF73CFBFE
:102DC00050B14CF6E440C0F60300016A4CF6FC2218
:102DD000C0F6030213680B604FF00900FFF72CFBED
:102DE00050B14CF6E440C0F60300416A4CF6FC22B8
:102DF000C0F6030213680B604FF00A00FFF71CFBDC
:102E000050B14CF6E440C0F60300816A4CF6FC2257
:102E1000C0F6030213680B604FF00B00FFF70CFBCA
:102E200050B14CF6E440C0F60300C16A4CF6FC22F7
:102E3000C0F6030213680B604FF00C00FFF7FCFABA
:102E400050B14CF6E440C0F60300016B4CF6FC2296
:102E5000C0F6030213680B604FF00D00FFF7ECFAA9
:102E600050B14CF6E440C0F60300416B4CF6FC2236
:102E7000C0F6030213680B604FF00E00FFF7DCFA98
:102E800050B14CF6E440C0F60300816B4CF6FC22D6
:102E9000C0F6030213680B60FFF7F6FB04B070BDC9
:102EA00010B504464FF000004FF01101FFF7CEFAC5
:102EB00047F62A23C1F6FF73198807EE901AB8EE79
:102EC000670A06EE900AB8EE667AC0EE070AC4ED0D
:102ED000000A4FF0010010BD10B504464FF000008D
:102EE0004FF01201FFF7B2FA07EE900AB8EE677AD8
:102EF0009FED0B0AC7EE000A10EE900A15F070F96C
:102F000005A3D3E9002315F009FB15F085F920602E
:102F10004FF0010010BD00BF6666666666660A4037
:102F200000F07F45AFF3008010B504464FF000007D
:102F30004FF01001FFF78AFA07EE900AB8EE677AB1
:102F40009FED1B0AC7EE000A10EE900A15F048F933
:102F500011A3D3E9002315F0E1FA15F05DF915F09E
:102F60003FF90FA3D3E9002315F092F90EA3D3E99B
:102F7000002315F089FB4FF000024FF00003C4F26C
:102F8000390315F087F915F047F920604FF001007B
:102F900010BD00BFAFF300806666666666660A40D5
:102FA00052B81E85EB51E83F7B14AE47E17A643F8F
:102FB00000F07F45AFF3008030B472B64CF6443376
:102FC000C0F603031A684EF63470CEF200000260B9
:102FD0004CF65031C0F603010A684EF68853CEF223
:102FE00000031A604CF64C30C0F60300016842F250
:102FF0000802CEF2040211604CF65433C0F603030B
:10300000186842F20C01CEF20401086043F6000396
:10301000C4F202031A6842F48030186019460B6843
:1030200013F4003FFBD043F64000C4F202000268F4
:1030300042F08051016047F20003C4F200031868B7
:1030400040F480421A604CF63C31C0F60301086837
:1030500043F60803C4F2020318604CF64832C0F687
:103060000302116843F60040C4F2020001604CF60E
:103070003833C0F603031A6843F60401C4F20201B0
:103080000A6043F60000C4F20200036843F0807255
:1030900002600146086810F0007FFBD043F6080389
:1030A000C4F202031A684FF0020161F301021A60D0
:1030B0001846036803F00C02082AFAD143F64401CB
:1030C000C4F20201086840F480430B6043F630000C
:1030D000C4F20200026842F48011016047F200036A
:1030E000C4F200031A6842F48071196047F20403C5
:1030F000C4F200031A6842F400711960036843F4D3
:103100008022026043F61440C4F2020001684BF6CC
:103110004043C0F603031B684CF64032C0F603027E
:1031200010686FEA000259400A4206D04BF6404050
:10313000C0F603004178CC2904D12A4B2A49994290
:1031400021D344E043F60841C4F2020142F63B2099
:10315000C0F61900086046F67F60C4F65D4008605E
:10316000134043F61442C4F202021360136843F0A2
:103170000201116043F60C40C4F20200026812F42E
:10318000803FFBD1D9E7194C194D281B20F00305CE
:103190004FF0000340F20002C1F200024EF6A461BB
:1031A000C0F6030105F10404C5F380005D589D508D
:1031B00003F10403A3420CD109E05858985003F1DD
:1031C00004035858985003F10403A342F5D130BCCE
:1031D00070470028F1D05858985003F10403A342D7
:1031E000EBD1F4E7302B0408A4EE0308A8EE0308A3
:1031F000332B040843F63003C4F202031A6842F486
:1032000000101860196841F480021A60704700BF0E
:103210002DE9F0011546002A66D040F64C13C2F2A3
:10322000000353E8002F02F1010243E80024012CBF
:10323000F7D04CF66032C0F60302146846F2084636
:10324000C4F2020634604CF65C37C0F603073A68F5
:1032500046F22843C4F202031A604FF6FF7846F2A2
:10326000304CC4F2020C46F23447C4F2020746F274
:103270002C46C4F202061C46454534BF2B46434645
:10328000CCF8001038603360226842F001022260FE
:10329000ED1A4FEA8303C918C018226812F0010F13
:1032A000FBD1002DE8D140F64C13C2F2000353E8E5
:1032B000002FA2F1010243E80024012CF7D053E8CB
:1032C000002FB2F1004F0DD14FF0000243E800246F
:1032D000012CF4D04EF60450CEF20000016841F00B
:1032E00080510160BFF32F8FBDE8F001704700BF30
:1032F00070B41646002A37D046F21045C4F20205D3
:103300002C6814F0010FFBD14CF65832C0F60302C2
:10331000146846F20842C4F20202146046F21842EF
:10332000C4F20202116046F21C41C4F202010860BC
:1033300046F21440C4F2020006604CF66432C0F655
:103340000302116846F21040C4F2020001600268F4
:1033500042F0010101603BB146F21040C4F20200AC
:10336000036813F0010FFBD170BC704743F61043A4
:10337000C4F20203186800280DDA43F60441C4F2CF
:10338000020140F22312C4F267520A6048F6AB13FE
:10339000CCF6EF530B6043F61040C4F20200016814
:1033A00001F00042002A14BF02200020704700BF35
:1033B00043F61043C4F202031868002807DB43F603
:1033C0001041C4F202010A6842F000430B607047EA
:1033D00000F17840B0F5801F2CBF0020012070471D
:1033E0002DE9F04F83B006460D46FFF7F1FF0028A8
:1033F00056D02846FFF7ECFF002854D0AE4255D8EF
:10340000FDF772FA0190FFF7B1FF0446002841D1A1
:1034100006F178434FEA93304CF66832C0F6030267
:1034200012F8008041F28830FEF766FF4FF0020983
:1034300043F6104BC4F2020B43F60C47C4F20207EA
:103440004CF6AC3AC0F6030AFEF74EFF494668F365
:10345000C60169F3092141F48033CBF800303868A4
:1034600010F4803FFBD15AF82820B61808F1010863
:103470005FFA88F8B542E7D24FF06400FEF73CFFF0
:103480004CF6E031C0F60301086843F61043C4F27D
:1034900002031860FFF78CFF0198FDF72FFA07E091
:1034A0004FF0020404E04FF0020401E04FF0020488
:1034B000204603B0BDE8F08F2DE9F04106460C46EA
:1034C00015460846FFF784FF002861D005F1FF305C
:1034D0002018FFF77DFF00285DD040F64C13C2F2A4
:1034E000000353E8002F02F1010243E80021012903
:1034F000F7D0FFF73BFF074630BB4CF6A831C0F6CC
:1035000003010A6843F61040C4F2020002608DB164
:1035100006F1FF3843F60C46C4F20206336813F492
:10352000803FFBD118F8011F04F8011BFEF7DCFEF9
:10353000013DF3D14CF6DC34C0F60304226843F6B7
:103540001040C4F202000260FFF732FF40F64C1355
:10355000C2F2000353E8002FA2F1010243E8002465
:10356000012CF7D053E8002FB2F1004F0DD14FF0EE
:10357000000243E80024012CF4D04EF60450CEF2B1
:103580000000016841F080510160BFF32F8F04E01B
:103590004FF0020701E04FF002073846BDE8F08126
:1035A00040F20433C2F2000318684CF6F432C0F65D
:1035B0000302116801604FF0000303604CF6F8321B
:1035C000C0F60302116841604CF6E433C0F6030311
:1035D0001A68C2614FF00D0101624CF6FC33C0F66F
:1035E00003031A680260704740F2FC23C2F2000332
:1035F0001868704770B48568C668446806FB054063
:103600004118196040F2FC20C2F2000000688142BB
:103610000CD2521890420CD340F20030C2F200009B
:103620000268891819604FF0010004E04FF00000B3
:1036300001E04FF0000070BC704700BF2DE9F04181
:103640000546FEF751FE4FF01E044FF0000840F211
:103650000436C2F200064FF00107052D26D8DFE838
:1036600005F0030A0F14191E3268936983F00200F3
:10367000C0F340011BE03068416901F0010116E030
:1036800032685369C3F3400111E030684169C1F306
:10369000C0110CE032685369C3F3801107E033684E
:1036A000986980F0010101F0010100E0414689B90B
:1036B00033685A6912F4807F10D1586910F4806F12
:1036C00010D1384606F0FCFB013CC6D14FF000009B
:1036D000BDE8F0814FF00100BDE8F0814FF000003F
:1036E000BDE8F0814FF00000BDE8F0812DE9F04128
:1036F00084B014461D46072900F2AD80072A00F267
:10370000AD8001EB81024CF60043C0F6030303EBEE
:103710008202137C002B40F0A48004EB84024CF660
:103720000043C0F6030303EB8202137C012B40F03D
:103730009B804CF60043C0F6030301EB810653F86F
:10374000262004EB840653F826309A4240F08F80FE
:1037500040F20837C2F200073870022A15D0032A57
:1037600025D0012A34D143F64000C4F20200066895
:1037700046F40012026040F20433C2F2000345F244
:103780000047C4F200071F6022E043F64000C4F285
:103790000200066846F48002026040F20433C2F27E
:1037A000000345F60007C4F200071F6010E043F66F
:1037B0004000C4F20200066846F40002026040F2D3
:1037C0000433C2F2000345F60047C4F200071F604D
:1037D0004CF60048C0F6030801EB810108EB8102BA
:1037E000107991684FF0000700974FF0010601969D
:1037F000D36802934FF003023B46FDF787FD04EBCD
:10380000840408EB84042079A16800970196E2689B
:1038100002924FF003023346FDF778FDFFF7C0FE3A
:1038200045B340F20030C2F200000A99016040F254
:10383000FC22C2F200020B9B136040F20C30C2F279
:1038400000004CF6E831C0F603012A463B4608F07A
:1038500095F8304610E04FF000000DE04FF000000A
:103860000AE04FF0000007E04FF0000004E04FF0E6
:10387000000001E04FF0010004B0BDE8F08100BF9E
:1038800038B5044640F20433C2F200031D68A8694B
:1038900010F0020F63D0FFF783FEA96911F0020F49
:1038A0005DD03BE040F20435C2F200052B684FF0DA
:1038B000A0021A614FF00200FFF7C0FE286881697C
:1038C00011F0010F08D0456915F4806F00F03882BF
:1038D000036843F4007202604FF0050004F0A0FB9F
:1038E0004FF0000516E040F20430C2F2000001681B
:1038F0004FEA14230B614FF00300FFF79FFE38B12E
:1039000040F20432C2F200021068E4B2046101E045
:103910004FF00005281C18BF012038BD4FF00000F3
:1039200038BD4FF0000038BD4FF0000038BD4FF0FB
:10393000000038BD4FF0000038BD4FF0000038BD2A
:103940004FF0000038BD4FF0000038BD4FF00000D0
:1039500038BD4FF0000038BD4FF0000038BD40F2D8
:103960000432C2F2000213684FF000005861196877
:1039700060F3492119601A6842F4807018604FF0B2
:103980000100FFF75BFE0028CBD040F20435C2F205
:1039900000052B684FF0A00119614FF00200FFF7FE
:1039A0004DFE2868826912F0010F08D0436913F4B4
:1039B000806F00F0C881016841F4007202604FF02E
:1039C000050004F02DFB40F20430C2F20000036851
:1039D0004FF0000159611A6861F349221A601868B2
:1039E00040F4807119604FF00100FFF727FE0028B6
:1039F0009AD040F20435C2F200052B684FF0A002C5
:103A00001A614FF00200FFF719FE2868816911F072
:103A1000010F08D0436913F4806F00F097810268AA
:103A200042F4007101604FF0050004F0F9FA40F231
:103A30000430C2F2000003684FF0000159611A68B7
:103A400061F349221A60186840F4807119604FF0E0
:103A50000100FFF7F3FD00283FF469AF40F20435A1
:103A6000C2F200052B684FF0A0021A614FF002006D
:103A7000FFF7E4FD2868816911F0010F08D0436960
:103A800013F4806F00F06581026842F400710160F8
:103A90004FF0050004F0C4FA40F20430C2F2000016
:103AA00003684FF0000159611A6861F349221A60F6
:103AB000186840F4807119604FF00100FFF7BEFDF7
:103AC00000283FF437AF40F20435C2F200052B68FE
:103AD0004FF0A0021A614FF00200FFF7AFFD286817
:103AE000816911F0010F08D0436913F4806F00F071
:103AF0003381026842F4007101604FF0050004F068
:103B00008FFA40F20430C2F2000003684FF0000167
:103B100059611A6861F349221A60186840F480718B
:103B200019604FF00100FFF789FD00283FF405AF51
:103B300040F20435C2F200052B684FF0A0021A6172
:103B40004FF00200FFF77AFD2868816911F0010F3C
:103B500008D0436913F4806F00F00181026842F4D9
:103B6000007101604FF0050004F05AFA40F2043091
:103B7000C2F2000003684FF0000159611A6861F356
:103B800049221A60186840F4807119604FF00100F2
:103B9000FFF754FD00283FF4D3AE40F20435C2F2E3
:103BA00000052B684FF0A0021A614FF00200FFF7EA
:103BB00045FD2868816911F0010F08D0436913F4AD
:103BC000806F00F0CF80026842F4007101604FF016
:103BD000050004F025FA40F20430C2F20000036848
:103BE0004FF0000159611A6861F349221A601868A0
:103BF00040F4807119604FF00100FFF71FFD0028AD
:103C00003FF4A1AE40F20435C2F200052B684FF03C
:103C1000A0021A614FF00200FFF710FD28688169C9
:103C200011F0010F08D0436913F4806F00F09D80FC
:103C3000026842F4007101604FF0050004F0F0F9F1
:103C400040F20430C2F2000003684FF000015961F5
:103C50001A6861F349221A60186840F4807119608B
:103C60004FF00100FFF7EAFC00283FF46FAE40F28E
:103C70000435C2F200052B684FF0A0021A614FF024
:103C80000200FFF7DBFC2868816911F0010F07D003
:103C9000436913F4806F6BD0026842F400710160D5
:103CA0004FF0050004F0BCF940F20430C2F200000D
:103CB00003684FF0000159611A6861F349221A60E4
:103CC000186840F4807119604FF00100FFF7B6FCEE
:103CD00000283FF43EAE40F20435C2F200052B68E6
:103CE0004FF0A0021A614FF00200FFF7A7FC28680E
:103CF000816911F0010F07D0436913F4806F3AD046
:103D0000026842F4007101604FF0050004F088F988
:103D100040F20430C2F2000003684FF00001596124
:103D20001A6861F349221A60186840F480711960BA
:103D30004FF00100FFF782FC00287FF4B3AD0BE6E3
:103D40004FF0010519E04FF00A0516E04FF00905A4
:103D500013E04FF0080510E04FF007050DE04FF0BD
:103D600006050AE04FF0050507E04FF0040504E002
:103D70004FF0030501E04FF0020540F20830C2F2B7
:103D80000000017801F1FF33DAB2012A3FF6B8AD45
:103D9000A9E500BFF8B50D461446002A6FD080B2E1
:103DA000FFF76EFD002865D04FF00300FFF746FCDB
:103DB00000285FD040F20433C2F2000318680268A2
:103DC00042F4807101604FF00100FFF737FC0028DA
:103DD00050D040F20433C2F20003186814F1FF31EE
:103DE00018BF0121026861F38A2202604FF0A1032B
:103DF00003614FF00200FFF721FC00283AD040F2A7
:103E00000430C2F2000001688A6912F0010F31D05B
:103E10004B6913F4806F2DD14FF0040640F2043744
:103E2000C2F200073046FFF709FC18B304F1FF3473
:103E3000012C27D1FCF758FD39680A696FEA0203A3
:103E400005F8013B0A686FF38A220A60FCF756FD09
:103E5000E8E72B681B6902E04FF004060E4D304680
:103E6000FFF7ECFB0028F4D10B4B1868016841F414
:103E700000720260D4F1010038BF0020F8BD4FF09D
:103E80000100F8BD386801696FEA010205F8012BED
:103E9000002CC7D1E0E700BF0403002030B583B099
:103EA00015461C461A4601ABFFF7A4FB48B1019822
:103EB00029462246FFF76EFF00280CBF182000207D
:103EC00001E04FF01F0003B030BD00BF2DE9F84FF7
:103ED00093460D4600295DD004464FF0030840F29A
:103EE0000439C2F2000901E0002E40D01FFA8BF025
:103EF000FFF7C6FC00283DD00BF0070715F0010FB7
:103F00004CD14046FFF79AFB002836D0072F1AD82D
:103F1000DDB13CB1D9F8000014F8011B6FEA0103D0
:103F2000036104E0D9F800604FF0FF02326107F14D
:103F30000107BA4605F1FF3635464046FFF77EFBDE
:103F4000002845D119E02E4600E02E46D9F80000A1
:103F5000026842F4007101600BF1080B2BF0070BB3
:103F60004FF00500FFF76AFB0028BDD107E04FF0D6
:103F7000010004E04FF0000001E04FF0000040F2CB
:103F80000433C2F2000319680A6842F400730B603C
:103F9000BDE8F88F4FF00100BDE8F88F4046FFF70D
:103FA0004DFB0028E9D0072FCDD82CB9D9F8003027
:103FB0004FF0FF021A6106E0D9F8000014F8011B67
:103FC0006FEA0103036107F1010705F1FF3598E787
:103FD000072FB8D82CB9D9F800504FF0FF022A614A
:103FE00006E0D9F8000014F8011B6FEA0103036131
:103FF00007F1010706F1FF3583E700BF30B583B055
:1040000015461C461A4601ABFFF7F4FA48B128469C
:104010002146019AFFF75AFF00280CBF1820002004
:1040200001E04FF01F0003B030BD00BF08B543F200
:104030005850C2F2000043F65802C2F20002131AAE
:104040004FF0FF314FEAA302FCF708FC43F658009B
:10405000C2F2000044F25801C2F200010A1A4FEA0B
:10406000A2024FF0FF31A2F12002FCF7F7FB02F0B1
:1040700087FB40F21C30C2F2000044F20001C4F29F
:1040800002014FF480524FF0030313F0B5FFFCF729
:10409000B3FF4FF0000008BDBFF36F8F704700BF44
:1040A0004CF62053C0F60303185C00EB40014CF6BD
:1040B0004C62C0F6030252F821305B68704700BFC3
:1040C00038B54CF62053C0F603031B5C03EBC30466
:1040D00040F23432C2F2000202EB840282F8211074
:1040E00014693CB140F23435C2F200051346D2697E
:1040F0009B69A04738BD00BFF8B506460F464CF691
:104100002053C0F603031D5C05EBC50040F23434B8
:10411000C2F2000404EB8004D4F810C0BCF1000F1C
:1041200007D0E2698A4204D030464FF00001A3690B
:10413000E047E76163695BB105EBC50040F23432EB
:10414000C2F2000202EB800230463946926998477B
:1041500094F8201079B127696FB105EBC50540F2DD
:104160003433C2F2000303EB8505304694F8211086
:10417000E269AB69B847F8BD4CF62053C0F60303BB
:10418000185C00EB40014CF64C62C0F6030252F89A
:104190002130D86840F08001D9607047F8B50446F6
:1041A00000EB40024CF64C63C0F6030353F8226068
:1041B00035686FEA0500306005F0010215F0020F66
:1041C0001CBF42F00202D2B215F0040F18BF42F039
:1041D000080215F0080F18BF42F0040215F4807FA2
:1041E00005D0316911F4804F18BF42F0100215F06C
:1041F000200F00D1E2B104EBC40740F23433C2F225
:10420000000303EB870087688FB1716804EBC4007B
:1042100040F23433C2F2000303EB80034CF6186023
:10422000C0F60300005DC9B29B69B84700E073683F
:10423000F26812F0800F1CD015F0800F19D0F168D1
:104240006FF3C711F16004EBC40040F23433C2F2E3
:10425000000353F8203063B140F23432C2F200025E
:1042600002EB80024CF61860C0F60300005D916915
:10427000984715F0400F17D004EBC40140F23433D7
:10428000C2F2000303EB810253686BB1084640F2AF
:104290003431C2F2000101EB80024CF61860C0F626
:1042A0000300005D91699847F8BD00BF684620F0A3
:1042B00007018D4601B54FF00600FFF76FFFBDE81F
:1042C00001408546704700BF684620F007018D46D3
:1042D00001B54FF00500FFF761FFBDE801408546DD
:1042E000704700BF684620F007018D4601B54FF0CA
:1042F0000400FFF753FFBDE801408546704700BF4B
:10430000684620F007018D4601B54FF00300FFF726
:1043100045FFBDE801408546704700BF684620F074
:1043200007018D4601B54FF00200FFF737FFBDE8EA
:1043300001408546704700BF684620F007018D4662
:1043400001B54FF00100FFF729FFBDE801408546A8
:10435000704700BF10B582B08DF807104CF620539F
:10436000C0F60303185C00EB40024CF64C61C0F64B
:10437000030151F82240236813F0800FFBD002A9FB
:1043800011F8012D626000EBC00040F23434C2F23B
:10439000000404EB8004608C4FF0010205F0A8FDDE
:1043A000608404F1200402B010BD00BF70B582B07B
:1043B0008DF807104CF62053C0F60303185C00EB91
:1043C00040014CF64C62C0F6030252F821402568C9
:1043D00015F0800F1DBF9DF807506560012600266F
:1043E00000EBC00340F23430C2F2000000EB830562
:1043F000688C0DF107014FF0010205F079FD68842A
:1044000005F12005E16841F08002E260304602B02B
:1044100070BD00BF2DE9F84F81468B4690461E4681
:104420009DF828A04CF62053C0F603031D5C05EB55
:1044300045024CF64C60C0F6030050F822409DF84F
:104440002C70012F14BF00270127082E06D0072E3D
:1044500002D1B8F1000F01D1FCF7F0F90AF1FF31F8
:10446000CBB2012B01D9FCF7E9F94CF6FC52C0F6AE
:10447000030252F82500B0FBFBF1A1604FF00002EF
:1044800067F38612BAF1010F04D0002F0CBF02238C
:10449000002301E04FF0000363F30D3267F38E3227
:1044A00022614FF06C00B8F1020F14BF002301230A
:1044B00063F3492018F1000818BF4FF0010868F3B2
:1044C0008A20082E18BF4FF0000868F30C3040F423
:1044D0000051E1604846FFF7E3FDBDE8F88F00BFFB
:1044E000F0B585B00D461E464CF62053C0F60303CA
:1044F000195C01EB41044CF64C67C0F6030757F812
:1045000024704CF62C63C0F60303185C00EB4001EA
:104510004CF62454C0F6030404EBC1040AB1FCF7C2
:104520008DF975B9207B21699DF82C2000924FF000
:1045300001030193626902924FF003023346FCF7D4
:10454000E5FE207861689DF8283000934FF0010265
:104550000192A36802934FF003023346FCF7D6FEA4
:104560004CF62060C0F603000168012D14BF002541
:10457000012565F3C301796105B0F0BD2DE9F8436C
:1045800005464CF62053C0F60303185C00EBC0024E
:1045900040F23434C2F2000404EB82044CF64C6165
:1045A000C0F6030100EB40064FEA860301EB030867
:1045B00051F80390FCF798F9064694F82000B8B13A
:1045C0004FF00007C9F80C703846394698F90420B6
:1045D000FCF7FCF928463946FFF772FDE3681BB18A
:1045E0002846E169A26998474FF0000284F820202C
:1045F0003046FCF783F9BDE8F88300BF2DE9F04FA2
:1046000085B005468B46924699464CF62053C0F637
:1046100003031E5C40F23438C2F2000806EBC60702
:104620004FEA870708EB070406EB46004CF64C619F
:10463000C0F6030101EB8006FCF756F9039043F640
:104640004003C4F2020318684CF62461C0F603016B
:104650000A6820EA020E4CF63062C0F603021068C7
:104660004EEA0000186043F64403C4F202031868DF
:10467000496820EA01005268104318604CF638611E
:10468000C0F6030105EB8503C818C95C427883783E
:1046900090F803C0CDF800C0007901902846FFF7DC
:1046A0001FFF9DF8382000929DF83C10019128468C
:1046B000594652464B46FFF7ADFE109B48F807306F
:1046C0001298A060119A62601399E160149BA36133
:1046D000B0684FF00F0196F90420FCF777F94FF01E
:1046E000010084F820000398FCF708F905B0BDE844
:1046F000F08F00BF4CF62053C0F60303185C00EBAC
:10470000C00340F23430C2F2000000EB83031961B1
:104710005A6170474CF62C63C0F60303185C00EB3B
:1047200040014CF66C52C0F6030202EB01107047D8
:10473000FA2884BF0530C0B2032812D84CF62053A3
:10474000C0F60303185C00EBC00140F23432C2F241
:10475000000202EB81034FF6FF7058844FF0010016
:1047600070474FF000007047FA2884BF0530C0B290
:1047700003280ED84CF62053C0F60303185C00EB58
:10478000C00140F23432C2F2000202EB8103588CC5
:1047900070474FF000007047082806D9102807D945
:1047A00020288CBF4020202070474FF00800704721
:1047B0004FF01000704700BF022809D0032804D032
:1047C000012814BF0020012070474FF003007047FC
:1047D0004FF00200704700BF40F60013C5F200031F
:1047E000186840F60802C5F200021168C1F34103DF
:1047F000022B12BF6FF30200032363F3020040F4A5
:1048000000406FF3995040F60012C5F200021060AC
:1048100040F60401C5F200010B6843F480700860A3
:10482000704700BF4CF63C73C0F603031A6840F6AD
:104830001030C5F200000260704700BF10B440F6AF
:104840005073C2F200031A5CE0B14FF0000340F66F
:104850000841C2F200014FF04C0404FB0212D1687F
:1048600021F0030202F1040262F312034FF001018E
:1048700061F3DC434CF6BC62C0F6030202EB40106D
:1048800081690B6010BC704770B440F22003C5F220
:1048900000031868C0F34342022A01D0062A29D136
:1048A00000F00F014CF64075C0F6030555F8216085
:1048B000C0F30A1505F1030398081BD041F200016B
:1048C000C5F2000100F1FF3404F001040A68334628
:1048D00072604FF0010282420ED10AE00C6803F1CF
:1048E000040343F8044F0C685C6002F10202824248
:1048F000F4D1356070BC7047002CEFD00C6803F128
:1049000004035C6002F101028242E7D1F1E700BFDB
:1049100070B44CF6A063C0F6030353F8206032680D
:10492000002A3CD04CF6BC61C0F6030101EB4011FB
:1049300002F103024FEA9202CB691B689A420CD93A
:1049400040F63402C5F2000211684FF0010303FA89
:1049500000F008431060184623E006F10403C2B1DA
:1049600002F1FF3000F00105086953F8044B0460C0
:10497000501E18D10DE00C691A4652F8045B2560F0
:1049800000F1FF300C695B68236002F10403013819
:10499000F1D14FF0000131604FF0010001E04FF024
:1049A000000070BC7047002DE5D00A6953F8044B35
:1049B00014600138DFD1ECE708B54FF0010303FACA
:1049C00000F040F23242C2F200021388184210D0C6
:1049D00023EA000340F23240C2F200000380CA6BB7
:1049E00052B1086A4FF0000104F0C0FC4FF0000023
:1049F00008BD4FF0000008BD4FF0010008BD00BF2A
:104A000070B540F21403C5F200031C684CF6B460A4
:104A1000C0F6030001680C4200F0BB8140F64C7206
:104A2000C2F200021378012B40F2B38140F2180069
:104A3000C5F2000001684CF65872C0F60302136814
:104A4000194200F0A68140F61800C5F20000016886
:104A500011F0010F56D040F60815C5F200052A687E
:104A600040F60830C5F2000003682A60036040F693
:104A70005071C2F20001087840F60841C2F200010C
:104A80004FF04C0505FB001503F00100E96A0143F6
:104A9000E962C3F3C000296B0143296303F00803F3
:104AA000D8B258BBD2B212F0010F0ED01DE0EA6AA4
:104AB00022B105F1100000F087FF2BE02B6B002BDB
:104AC000F7D1686B0028F4D124E012F0900FEED0FB
:104AD00040F63403C5F20003186820F001011960A4
:104AE0004FF00000FFF714FFE1E76E6B4FF000009E
:104AF0002946FFF761FF30436863D8E74FF00001B4
:104B0000E963CFE740F61802C5F20002136813F418
:104B1000803FA0D140F61801C5F200010A6802F0FA
:104B2000020398B2002856D040F62815C5F20005B9
:104B30002A6840F62830C5F2000003682A60036046
:104B400040F65071C2F20001487840F60841C2F2C6
:104B500000014FF04C0505FB001503F00100E96A68
:104B60000143E962C3F3C000296B0143296303F0E9
:104B70000803D8B258BBD2B212F0010F0ED01DE01C
:104B8000EA6A22B105F1100000F01EFF2FE02B6B46
:104B9000002BF7D1686B0028F4D128E012F0900FB9
:104BA000EED040F63403C5F20003186820F002018D
:104BB00019604FF00100FFF7ABFEE1E76E6B4FF0BD
:104BC00001002946FFF7F8FE30436863D8E74FF04D
:104BD0000001E963CFE740F61801C5F200010A6859
:104BE0004FEA124303F0020081B200299CD140F643
:104BF0001801C5F200010A6802F0040398B2002807
:104C000056D040F64815C5F200052A6840F64830EF
:104C1000C5F2000003682A60036040F65071C2F2DA
:104C20000001887840F60841C2F200014FF04C05BF
:104C300005FB001503F00100E96A0143E962C3F3D3
:104C4000C000296B0143296303F00803D8B258BBA5
:104C5000D2B212F0010F0ED01DE0EA6A22B105F1C6
:104C6000100000F0B1FE2FE02B6B002BF7D1686B2A
:104C70000028F4D128E012F0900FEED040F6340373
:104C8000C5F20003186820F0040119604FF002001B
:104C9000FFF73EFEE1E76E6B4FF002002946FFF79B
:104CA0008BFE30436863D8E74FF00001E963CFE73C
:104CB00040F61801C5F200010A684FEA124303F0FA
:104CC000040081B200299CD140F61801C5F2000110
:104CD0000A6802F0080398B258B940F61801C5F204
:104CE00000010A684FEA124303F0080081B200296C
:104CF0004FD040F66815C5F200052A6840F66830C6
:104D0000C5F2000003682A60036040F65071C2F2E9
:104D10000001C87840F60841C2F200014FF04C058E
:104D200005FB001503F00100E96A0143E962C3F3E2
:104D3000C000296B0143296303F00803D8B210B106
:104D40004FF00001E963D2B212F0010F08D06E6B90
:104D50004FF003002946FFF72FFE304368630EE053
:104D600012F0900F0BD040F63403C5F20003186820
:104D700020F0080119604FF00300FFF7C9FDEA6A4F
:104D80001AB92B6B0BB9686B18B105F1100000F064
:104D90001BFE14F0100F01D0FFF776FD14F4805FB6
:104DA0000DD040F61D71C2F200014FF001020A70F1
:104DB00040F61473C2F20003186802F09BFF14F46B
:104DC000005F01D0FFF708FD14F4006F14D040F627
:104DD0006860C2F200004FF00101017040F64073BC
:104DE000C2F200034FF000021A7040F61470C2F2D3
:104DF0000000006802F07EFF002C14DA40F66861C3
:104E0000C2F200014FF000030B7040F64070C2F296
:104E100000004FF00102027040F61471C2F200016E
:104E2000086802F067FF40F21403C5F200031C603B
:104E300070BD00BF684620F007018D4689B500AF00
:104E4000FFF7DEFDBD46BDE889408546704700BFDF
:104E50002DE9F04140F60846C2F200064FF04C033F
:104E600003FB0066304650F8205F4CF6BC68C0F685
:104E700003084FEA451708EB07044FF000014FF015
:104E80001C0215F0B9F835624FF00100B06258F815
:104E900007204FF00003136061690B60A0684FF0BA
:104EA000FF02026061680B60A0690360E1680A604C
:104EB0004CF64072C0F6030252F8250003604CF62F
:104EC000A061C0F6030151F825201360BDE8F08110
:104ED00000B583B04FF00003019340F21001C5F21A
:104EE00000010A68B0F1FF3F08BF102060F389128B
:104EF00042F0200040F21003C5F20003186019468A
:104F000040F63F52C0F20302019800F10100019007
:104F10000B6813F0200F02D001989042F4D94FF0A3
:104F2000030004F0CDFF03B000BD00BF2DE9F8433E
:104F30004FF04C0303FB00F040F60841C2F20001C1
:104F40004418256A4FF0010606FA05F64CF6BC62D5
:104F5000C0F6030202EB45174058002867D0A3684B
:104F6000FBB1D7F80080D8F8001011F4004F18D129
:104F7000D8F80020914663F30A09007AFFF71CFC79
:104F800060F3934949F4004965F3995949F0805019
:104F9000C0F3404363F39A60C8F800002846FFF767
:104FA00097FFE168F1B17A68106810F4004F19D1E9
:104FB0002846FFF743FCD7F80480D8F80070E36870
:104FC00063F30A072168087AFFF7F6FB60F393475B
:104FD00047F4004242F01047C7F3404060F39A673D
:104FE000C8F800704CF64073C0F6030353F8251060
:104FF0004FF000020A60A06858B140F61C03C5F2E9
:105000000003196846EA010290B2196860F30F01C3
:105010001960E3685BB140F61C00C5F2000002684D
:1050200046EA1246B6B2016866F31F410160BDE868
:10503000F88300BF70B582B04FF00002019240F2D9
:105040001003C5F20003196841F0010018600192D5
:105050001A6812F0010F19D0019940F63F53C0F2BF
:105060000303994212D840F21000C5F2000040F646
:105070003F52C0F20302019901F10101019103685D
:1050800013F0010F02D001999142F4D94FF00300BF
:1050900004F016FF4FF00000019040F21002C5F23C
:1050A00000021368002B1DDB019940F63F50C0F24F
:1050B0000300814216D84FF0030640F21005C5F2F6
:1050C000000540F63F54C0F20304304604F0F8FEF9
:1050D000019A02F1010201922B68002B02DB019977
:1050E000A142F2D902B070BD00B583B04FF0000309
:1050F000019340F21000C5F20000026842F0100176
:10510000016040F63F52C0F20302019B03F101032C
:105110000193016811F0100F02D0019B9342F4D962
:105120004FF0030004F0CCFE03B000BD50B14CF6CC
:105130005071C0F603010A6840F21803C5F200037B
:105140001A6070474CF65473C0F603031A6840F2B5
:105150001800C5F200000260704700BF38B54FF07C
:10516000000440F60063C5F200031C6040F6000234
:10517000C5F20002106840F0030164F3820164F399
:105180000A11116040F22405C5F200052B684FF0AA
:10519000400262F30F032B60204662F31F4021465A
:1051A00062F31F4162F30F0140F22805C5F20005CA
:1051B00029604FF0800363F30F0040F20412C5F240
:1051C000000210604FF0C00161F30F0040F20815BB
:1051D000C5F2000528604FF4807363F30F0040F2BE
:1051E0000C12C5F2000210604FF0FF30FFF770FEA6
:1051F000FFF77AFF40F61000C5F20000046040F6A9
:105200001401C5F200010C604FF0FF3540F61803A1
:10521000C5F200031D6040F61C02C5F200021460D6
:105220002046FFF715FE4FF00100FFF711FE4FF08B
:105230000200FFF70DFE4FF00300FFF709FE4FF0ED
:105240000400FFF705FE4FF00500FFF701FE4FF0E9
:105250000600FFF7FDFD4FF00700FFF7F9FD40F2F4
:105260001800C5F20000046040F21401C5F200010C
:105270000D604FF00100FFF759FF38BD40F2324397
:10528000C2F2000319884FF0010202FA00F0084050
:1052900000280CBF02200320704700BF40F6001317
:1052A000C5F200031B68C3F3076202F08000C1B2BD
:1052B00009B143F0804343F4001040F60012C5F2F8
:1052C00000021060704700BF2DE9F84305461646FE
:1052D0004CF6BC68C0F6030808EB40184CF6A06317
:1052E000C0F6030353F820704FF0010909FA00F9E2
:1052F0000C46A9B9386840B940F23243C2F2000303
:10530000188819EA000F5AD10AE040F23241C2F27D
:1053100000010A8819EA020F02D02846FFF7D8FDDB
:1053200006F1030107F1040388081CD000F1FF32E5
:1053300002F0010CA4F1040151F8042F43F8042BEE
:1053400001383ED10FE001F1040249681C4644F8DF
:10535000041B00F1FF3002F1040152685A6004F1AD
:1053600004030138EFD13E6040F23243C2F2000341
:10537000198849EA0109A3F8009065B940F61010B0
:10538000C5F2000002684FF0010161F3D44266F3F8
:105390000602026009E0D8F8140002684FF0010329
:1053A00063F3DC4266F312020260D8F8003018683A
:1053B00040F004421A6016B12846FFF7A9FABDE88A
:1053C000F883BCF1000FBED051F8042F43F8042B32
:1053D0000138B8D1C7E700BF70B504464CF640733A
:1053E000C0F6030353F82060334653F8045BAA4227
:1053F00038BF1546084619462A4614F0D9FD4FF025
:10540000000030602046FFF719FA4CF6BC61C0F688
:10541000030101EB441463681A6842F00440186009
:10542000284670BDF8B5054640F60843C2F20003B1
:105430001868002871D040F60841C2F20001CA6C19
:10544000002A71D040F60844C2F20004D4F89860F3
:10545000002E6DD040F60847C2F20007D7F8E430BE
:10546000002B69D040F60840C2F20000D0F830119D
:10547000002965D040F60842C2F20002D2F87C4111
:10548000002C61D040F60846C2F20006D6F8C8717A
:10549000002F5DD040F60843C2F20003D3F8140297
:1054A000002859D040F60841C2F20001D1F860222C
:1054B000002A55D0464E4FF00807FBF7BFF92C7A6B
:1054C000002C53D040F23042C2F200021088014654
:1054D00010F0020F55D04FF0010404F1010441FA1D
:1054E00004F212F0010FF8D14FF0010101FA04F1BA
:1054F000084340F23043C2F20003188044B968897F
:10550000FFF74AF9B060A889FFF746F9F06042E07A
:105510006A89B260A989F1603DE040F60846C2F2AE
:1055200000064FF000071EE02A4E4FF001071AE078
:10553000294E4FF0020716E0284E4FF0030712E005
:10554000274E4FF004070EE0264E4FF005070AE005
:10555000254E4FF0060706E0244E4FF0070702E005
:105560001B4E4FF00807072FA9D9A6E740F230439A
:10557000C2F20003188840F0010119804FF00004C6
:10558000BDE740F0020440F23043C2F200031C8049
:105590004FF00104BCE740F65070C2F2000007551E
:1055A000374647F8205B38464FF000014FF01C02A9
:1055B00014F022FD34626B68B36306F110004FF003
:1055C00006012A683B4600F0DFF92046F8BD00BF1F
:1055D000680E0020540C0020A00C0020EC0C0020D1
:1055E000380D0020840D0020D00D00201C0E00205E
:1055F000022907D140F60003C5F200031A6860F3E0
:105600000A121A60704700BF10B54FF0000440F650
:105610003403C5F200031C6040F60400C5F200002C
:10562000026842F0010101602046FFF711FC4FF0D3
:105630000100FFF70DFC4FF00200FFF709FC4FF0EF
:105640000300FFF705FC4FF00400FFF701FC4FF0EB
:105650000500FFF7FDFB4FF00600FFF7F9FB4FF0E9
:105660000700FFF7F5FB4FF0FF30FFF731FC40F28A
:105670003243C2F200031C8040F61800C5F200005D
:105680004FF0FF3202604CF65C71C0F6030108680F
:1056900040F61C03C5F2000318604CF6B862C0F671
:1056A0000302116840F61400C5F2000001604CF6D8
:1056B000B063C0F603031A6840F61001C5F200019A
:1056C0000A6020464FF00201FFF792FFFFF7AAF8A9
:1056D0002046FFF72BFC4FF00100FFF727FC4FF0AF
:1056E0000200FFF723FC4FF00300FFF71FFC4FF011
:1056F0000400FFF71BFC4FF00500FFF717FC4FF00D
:105700000600FFF713FC4FF00700FFF70FFC10BD7A
:1057100008B5FFF779FF08BD704700BFF0B585B049
:10572000054641F28830FCF7E7FD002D62D043F6D4
:105730003401C4F202010C6844F080060E604FF0A0
:10574000000400944FF0030601964FF00A070297F9
:1057500020464FF00B0132462346FBF7D7FD00945D
:105760000196029720464FF00C0132462346FBF784
:10577000CDFD40F20C06C5F20006336843F040024E
:105780003260FFF757FC40F23800C5F200004FF4DA
:105790000411016044F6206004F092FBFCF7A4FDC4
:1057A000336843F0400064F3082064F349204FF06D
:1057B000050262F38D2064F35D7040F0804131603A
:1057C00044F6206004F07CFBFCF78EFDFFF7C6FC7E
:1057D00040F20803C5F2000340F28110186044F65D
:1057E0003560C0F602004FF00F014FF04302FBF7A7
:1057F000EDF813E04FF000004FF00F014FF04302BF
:10580000FBF7E4F84FF0000340F23802C5F2000263
:10581000136040F21800C5F2000003602846FFF74D
:105820007BFF4FF06400FCF767FD05B0F0BD00BFE3
:105830002DE9F04182B04CF66077C0F6030745F6DB
:105840001116C0F6020640F28C15C2F200054FF0A8
:105850000408CDF8008038464FF0800132462B46D0
:1058600002F094FB40F26444C2F200042060CDF8E0
:10587000008038464FF08101324605EB080302F004
:1058800085FB6060CDF8008038464FF082013246DB
:1058900005F1080302F07AFBA060CDF800803846DD
:1058A0004FF08301324605F10C0302F06FFBE0601C
:1058B000CDF8008038464FF08401324605F11003E0
:1058C00002F064FB2061CDF8008038464FF085017E
:1058D000324605F1140302F059FB6061CDF80080F7
:1058E00038464FF08601324605F1180302F04EFBB0
:1058F000A061CDF8008038464FF08701324605F1AF
:105900001C0302F043FBE06102B0BDE8F08100BF80
:1059100080B505464FF0000640F23C49C2F200094E
:1059200040F28448C2F2000840F23847C2F2000751
:105930001FE0FAF7D9FF2C68616829604FF0000278
:105940006260237B062B0ED1216849F82610092EB0
:105950009CBF0136F6B2012E03D93A8802F101024A
:105960003A8088F80060FAF7C9FF23680BB1A06895
:1059700098472B6803F1FF3010F1030FD9D902F0DB
:1059800087F94FF00006F4E70260B3F1FF3F18BF5C
:105990008360FF290ED143F25453C2F200031A6808
:1059A00022B192F829304FEA530101E04FF007018C
:1059B0000173704701F07F010173704710B14FF020
:1059C00000020260704700BF38B50446FAF78CFF4A
:1059D000054640F28643C2F200031A8802F1010232
:1059E0001A80002C35D06368EBB940F28840C2F2CF
:1059F0000000028802F101020280207B40F28C1339
:105A0000C2F2000353F82010616043F82040247B69
:105A100040F26442C2F2000252F8240002F06AF935
:105A20004FF0010422E040F23440C2F2000002884C
:105A300002F101020280247B062C15D140F23A418A
:105A4000C2F200010B8803F101030B804FF0000448
:105A50000CE040F23640C2F20000018801F1010181
:105A600001804FF0000401E04FF000042846FAF7EF
:105A700045FF204638BD00BF10B5044640F2946093
:105A8000C2F200004FF000014FF0240214F0B4FA0B
:105A9000D4B140F2D440C2F200004FF000014FF008
:105AA000480214F0A9FA40F26450C2F200004FF02C
:105AB00000014FF0240214F09FFA40F25C53C2F24E
:105AC00000034FF002021A7010BD00BF38B54CF64B
:105AD000C873C0F6030353F8205040F22051C2F2BD
:105AE000000151F820404DF20C02C0F60302105C98
:105AF000FBF7F4FC2840A04214BF0020012038BD71
:105B00004DF20C03C0F603031A5C40F26451C2F27A
:105B1000000151F822204CF6C873C0F6030353F875
:105B2000200002420CBF00200120704770B440F6F4
:105B30004C13C2F2000353E8002F02F1010243E8C4
:105B400000210129F7D04DF20C02C0F60302155CCA
:105B500040F29461C2F2000151F825404CF6C8763B
:105B6000C0F6030656F8202024EA020041F825007A
:105B700053E8005FA5F1010543E80056012EF7D078
:105B800053E8005FB5F1004F0DD14FF0000543E839
:105B90000056012EF4D04EF60450CEF200000168FB
:105BA00041F080510160BFF32F8F14420CBF0020E1
:105BB000012070BC704700BF4DF21C03C0F6030308
:105BC000185C704708B54FF0000040F25851C2F21F
:105BD0000001FAF737FE003018BF012008BD00BFF2
:105BE00010B50446FBF77AFC40F2AC13C2F2000396
:105BF00053F82410484010BD10B504464FF0010082
:105C0000FFF73AFF4CF69073C0F6030353F83420C5
:105C100040F26051C2F200010A6003EBC404606804
:105C200040F28C53C2F20003186010BD00B585B07D
:105C30004FF00000FFF7E0FF4FF00003009340F249
:105C40009052C2F2000201924FF0400002904DF2D9
:105C50000000C0F603004FF0020145F60152C0F605
:105C6000020202F07FF840F29063C2F20003186073
:105C700005B000BD2DE9F001804600283CD04FF072
:105C800000034FEA8302086850F823404D6855F836
:105C9000236086EA0407886850F8235084EA050CDC
:105CA0004CEA07076FEA070CC86850F8235026EA49
:105CB000050707EA0C0705EA0C0C66EA0C063540F6
:105CC00040F82350CD6855F82300384345F82300A9
:105CD0000D6955F82300384345F823004D690DB18F
:105CE00045F823704868855888688550486884500E
:105CF00003F101034345C4D1BDE8F001704700BF83
:105D00002DE9F84340F26058C2F2000840F288568C
:105D1000C2F2000640F28C44C2F200044FF00005CB
:105D200040F28C57C2F20007D8F8000000EB800068
:105D300002F076F93368002B40F00B8220462946AA
:105D40004FF0240214F058F903E24FF009004CF62A
:105D5000B071C0F60301FFF78DFF40F25C53C2F251
:105D60000003197859B101F1FF3040F25C52C2F2E0
:105D70000002107040F29463C2F200031D6040F212
:105D80005851C2F200010868E8B940F25852C2F214
:105D90000002156040F21C53C2F20003197849B9A1
:105DA00040F25851C2F20001086860B1284606F07E
:105DB0005FFD08E040F25850C2F20000026842F075
:105DC00000630360ECE740F25C52C2F20002137819
:105DD0005BB103F1FF3140F25C50C2F20000017090
:105DE00040F29462C2F20002556040F25853C2F28F
:105DF0000003196841BB4CF66C70C0F603004268A2
:105E000040F2B043C2F2000359680A4040F25850D1
:105E1000C2F20000026040F21C52C2F2000213788B
:105E20004BB940F25853C2F20003196861B12846D9
:105E300006F01EFD08E040F25851C2F20001086869
:105E400040F000620A60ECE740F25C50C2F20000F1
:105E500002785AB102F1FF3340F25C51C2F2000104
:105E60000B7040F29460C2F20000856040F258521C
:105E7000C2F200021368EBB940F25851C2F20001BD
:105E80000D6040F21C50C2F2000002784AB940F2A4
:105E90005852C2F20002136863B1284606F0E8FCCB
:105EA00008E040F25853C2F20003196841F0006064
:105EB0001860ECE740F25C51C2F20001087858B17A
:105EC00000F1FF3340F25C52C2F20002137040F264
:105ED0009461C2F20001CD6040F25850C2F200005D
:105EE0000368EBB940F25852C2F20002156040F26A
:105EF0001C51C2F20001087848B940F25850C2F271
:105F00000000036863B1284606F0B2FC08E040F2E6
:105F10005853C2F200031A6842F000611960ECE7BE
:105F200040F25C52C2F20002117859B101F1FF3027
:105F300040F25C53C2F20003187040F29462C2F265
:105F40000002156140F25851C2F20001086840BBDE
:105F50004CF66C73C0F603031A6940F2B041C2F20A
:105F600000010869024040F25853C2F200031A606F
:105F700040F21C52C2F20002117849B940F2585165
:105F8000C2F20001086860B1284606F071FC08E022
:105F900040F25850C2F20000036843F00062026011
:105FA000ECE740F25C53C2F200031A785AB102F1F6
:105FB000FF3140F25C50C2F20000017040F2946385
:105FC000C2F200035D6140F25852C2F20002116851
:105FD000E9B940F25850C2F20000056040F21C538B
:105FE000C2F200031A784AB940F25852C2F20002D3
:105FF000116861B1284606F03BFC08E040F25851B8
:10600000C2F20001086840F000630B60ECE740F268
:106010005C50C2F2000003785BB103F1FF3140F243
:106020005C52C2F20002117040F29460C2F20000B1
:10603000856140F25853C2F200031968E9B940F291
:106040005852C2F20002156040F21C50C2F2000029
:1060500003784BB940F25853C2F20003196861B19A
:10606000284606F005FC08E040F25851C2F2000153
:106070000A6842F000600860ECE740F25C52C2F24D
:106080000002107858B100F1FF3340F25C51C2F2C7
:1060900000010B7040F29462C2F20002D56140F23E
:1060A0005850C2F200000368EBB940F25851C2F2F6
:1060B00000010D6040F21C52C2F20002107848B993
:1060C00040F25850C2F20000036863B1284606F05F
:1060D000CFFB08E040F25853C2F20003196841F0C8
:1060E00000621A60ECE740F25C51C2F200010A78EB
:1060F0005AB102F1FF3040F25C53C2F20003187053
:1061000040F29461C2F200010D6240F25852C2F2B4
:1061100000021068D8B940F25853C2F200031D6063
:1061200040F21C51C2F200010A783AB140F25850D4
:10613000C2F20000036843F00061016040F258526F
:10614000C2F20002106810B1284606F091FB3560DB
:10615000EAE5D4F800902846FFF742FD40EA09013D
:106160002160D4F804904FF00100FFF739FD40EAB8
:1061700009026260D4F808904FF00200FFF730FD8A
:1061800040EA0900A060D4F80C904FF00300FFF73C
:1061900027FD40EA0903E360D4F810904FF00400B3
:1061A000FFF71EFD40EA09012161D4F814904FF079
:1061B0000500FFF715FD40EA09026261D4F8189066
:1061C0004FF00600FFF70CFD40EA0900A061D4F88B
:1061D0001C904FF00700FFF703FD40EA0903E3615D
:1061E000D4F820904FF00800FFF7FAFC40EA0901CC
:1061F0002162306800F1010030603A689042FFF49B
:1062000093ADA2E500B585B04FF00003009340F2D6
:10621000FC62C2F2000201924FF0400002904DF287
:106220002C10C0F603004FF0060146F24522C0F6DE
:10623000020201F097FD40F2B863C2F20003186059
:1062400005B000BD2DE9F04F85B040F66C031E4649
:10625000C2F2000640F624000746C2F2000740F2F0
:10626000D861C2F20001019101F012FD3268002AEA
:10627000FAD061E1E359002B53D02846FFF7B0FC78
:1062800001996258605090434BD0E35910EA0302E1
:1062900047D0039991F800E04DF23419C0F6030994
:1062A0004FEA451840F2BC61C2F200014FF6FF7C94
:1062B0004DF22C0AC0F6030A40F6000BC2F2000BA6
:1062C00000957046C2F10003134022EA030218B998
:1062D00054F80B502B4221D15FEA136E04D01AF808
:1062E0000E3003F118030EE01D0C04D01AF805302F
:1062F00003F1100307E05FEA132E1ABF1AF80E30FD
:1063000008331AF80330434419F8035031F815E004
:10631000E6451CBF0EF1010E21F815E0002AD1D18F
:10632000009D05F1010504F10404092DA2D1029C90
:10633000621E029240F0F7800399087800F1010094
:10634000C3B20B700B2B03D14FF000040C7002E0B2
:10635000002B40F0E58040F64802C2F200021168CE
:1063600091B16FEA01003B6803403B6040F60005D5
:10637000C2F200052C682040286040F64801C2F2B5
:1063800000014FF000020A6040F64800C2F200002F
:10639000436893B16FEA03057C682C407C6040F64B
:1063A0000002C2F2000251680D40556040F64800FC
:1063B000C2F200004FF00003436040F64805C2F20D
:1063C0000005AC6894B16FEA0400BA680240BA6094
:1063D00040F60003C2F2000399680840986040F656
:1063E0004805C2F200054FF00004AC6040F64800DA
:1063F000C2F20000C26892B16FEA0203F968194064
:10640000F96040F60005C2F20005EC682340EB603D
:1064100040F64800C2F200004FF00002C26040F6B1
:106420004803C2F20003196991B16FEA01053C69A2
:106430002C403C6140F60000C2F2000002691540A9
:10644000056140F64803C2F200034FF000011961F4
:1064500040F64805C2F200056C6994B16FEA040089
:106460007A6902407A6140F60003C2F2000359697A
:106470000840586140F64805C2F200054FF000049C
:106480006C6140F64800C2F20000826992B16FEA86
:106490000203B9691940B96140F60005C2F200056E
:1064A000AC692340AB6140F64800C2F200004FF0F7
:1064B0000002826140F64803C2F20003D96991B13B
:1064C0006FEA0105FC692C40FC6140F60000C2F255
:1064D0000000C2691540C56140F64803C2F20003DE
:1064E0004FF00001D96140F64805C2F200052C6A60
:1064F00094B16FEA04003A6A02403A6240F600033F
:10650000C2F20003196A0840186240F64805C2F258
:1065100000054FF000042C624FF4FA70029002E084
:106520004FF4FA7502954FF0010001F079FD3268E1
:10653000002A3FF499AE07E04FF4FA75029540F255
:10654000FC74C2F2000403944FF00004254691E667
:1065500010B54FF0000440F66C03C2F200031C605B
:1065600040F60000C2F2000021464FF00902FAF79F
:1065700075F940F62400C2F2000021464FF00902EE
:10658000FAF76CF940F64800C2F2000021464FF0DD
:106590000902FAF763F940F2D860C2F2000021461E
:1065A0004FF00902FAF75AF940F2BC60C2F200005B
:1065B00021464FF01A0213F01FFD40F2FC70C2F2A8
:1065C0000000047010BD00BF70B54DF20C03C0F6A2
:1065D00003031B5C4CF6C872C0F6030252F820207D
:1065E00040F66C00C2F20000046840F62405C2F2D6
:1065F000000555F82300104206D104F1010640F6CB
:106600006C05C2F200052E6049B140F60001C2F2ED
:10661000000151F82350154341F8235009E040F69A
:106620000001C2F2000151F8235025EA020541F8A9
:106630002350104340F62401C2F2000141F8230028
:1066400040F64801C2F2000151F8230020EA02029C
:1066500041F8232034B940F2B863C2F2000318684D
:1066600001F048FB70BD00BF30B44DF20C03C0F622
:1066700003031B5C4CF6C872C0F6030252F82020DC
:1066800040F62400C2F2000050F82300104229D046
:1066900040F66C04C2F20004256805F1010525608E
:1066A00071B140F64801C2F2000151F82340144391
:1066B00041F8234040F2FC71C2F20001097889B927
:1066C0006FEA020240F60001C2F2000151F82340D5
:1066D000144041F82340024040F62400C2F200007A
:1066E00040F8232030BC704730B4034640F64C12CB
:1066F000C2F2000252E8000F00F1010042E800047B
:10670000012CF7D040F2BC60C2F2000030F8132038
:1067100039B140F2BC61C2F200014FF0000421F82F
:10672000134040F64C13C2F2000353E8004FA4F1AB
:10673000010443E80045012DF7D053E8004FB4F1C0
:10674000004F0DD14FF0000443E80045012DF4D077
:106750004EF60450CEF20000016841F08051016015
:10676000BFF32F8F104630BC704700BF40F2FC7360
:10677000C2F200031878D0F1010038BF0020704742
:106780002DE9F84FDFF834814B4FC8EB07004FEA93
:10679000D00707F101074FF0000540F2982AC0F634
:1067A000000A40F28039C0F6000931E044464FF05B
:1067B00000066FEA060B0BEB070101F0010B58F81E
:1067C000043CAB4229D135E054F8043CAB4205D13E
:1067D00054F8080C8047FBF787FD0BE0FF2B09D925
:1067E000FF2D07D154F8040C4FF0070154F8082C82
:1067F00001F0D8FB06F1010604F1080454F8041C6A
:10680000A94240D14CE005F10105B5F5807F02D0E9
:10681000CA45CBD3F7E7BDE8F88FFF2B0FD9FF2D83
:106820000DD158F8040C4FF0070158F8082C01F06E
:10683000B9FB04E058F8082C9047FBF755FD06F12A
:10684000010604F10804BE42DDD0BBF1000FBBD04D
:1068500054F8040CA8420AD0FF280DD9FF2D0BD103
:106860004FF0070154F8082C01F09CFB04E054F8A9
:10687000081C8847FBF738FD06F1010604F10804FF
:10688000BE42A1D1BFE7FF290FD9FF2D0DD154F88A
:10689000040C4FF0070154F8082C01F083FB04E0CE
:1068A00054F8082C9047FBF71FFD06F1010604F190
:1068B0000804BE4288D1A6E787030008A0020008AA
:1068C000027840F6E103C2F200031B789A4206D335
:1068D0004FF000020270087800F1010008700A7899
:1068E00040F6E203C2F200031878824224BF00207F
:1068F0000870704738B140F61840C4F202004FF0FB
:1069000002010180704740F61A43C4F202034FF0BF
:1069100002021A80704700BF08B540F61843C4F25F
:1069200002034FF008021A8000EA0201CBB23BB129
:1069300040F61843C4F202034FF08001198006E0CC
:1069400040F61A41C4F202014FF080020A8000F0C2
:106950000402D3B23BB140F61841C4F202014FF039
:1069600040030B8006E040F61A41C4F202014FF0EA
:1069700040020A8010F0010F19BF40F61841C4F21E
:10698000020140F61A41C4F202014FF010020A80DF
:1069900000F00200C1B239B140F61840C4F2020062
:1069A0004FF02001018006E040F61A43C4F20203D2
:1069B0004FF020021A804FF0010003F081FA40F6F8
:1069C0001A43C4F202034FF008021A8008BD00BF48
:1069D00010B50C46FFF78EFF40F61843C4F20203D1
:1069E0004FF008021A8014F0800F19BF40F61843C8
:1069F000C4F2020340F61A43C4F202034FF08000CF
:106A0000188004F04001CBB23BB140F61841C4F20B
:106A100002014FF040030B8006E040F61A40C4F23A
:106A200002004FF04002028004F01000C2B23AB1FE
:106A300040F61840C4F202004FF01002028006E057
:106A400040F61A41C4F202014FF010030B8004F02B
:106A50002001CBB23BB140F61841C4F202014FF025
:106A600020030B8006E040F61A40C4F202004FF00B
:106A7000200202804FF0010003F022FA40F61A4093
:106A8000C4F202004FF0080202802046FFF744FFE4
:106A90004FF0320003F014FA10BD00BF08B503290F
:106AA00014D8DFE801F0020B05084FF0800107E081
:106AB0004FF0940104E04FF0D40101E04FF0C00129
:106AC0000A184FF00000D1B2FFF782FF08BD00BFE7
:106AD00008B540F6F603C2F20003187830B940F664
:106AE000EC01C2F20001086801F004F940F6F60377
:106AF000C2F200034FF002021A7008BD10B5A0F1F7
:106B00000803052B3DD8DFE803F01F3C2C3C038530
:106B100040F67C00C2F200004FF020014FF054021A
:106B200013F06AFA40F6D400C2F200004FF0FF31D1
:106B30004FF00C0213F060FA40F6F000C2F20000D1
:106B4000026802F1010202604FF0000140F6760394
:106B5000C2F20003197040F67700C2F20000017023
:106B600056E040F67601C2F200014FF000030B70D0
:106B700040F67700C2F20000027802F101020270D2
:106B80003CE040F67602C2F20002127840F677014D
:106B9000C2F200010B7840F6E101C2F2000109786F
:106BA00001FB032340F67C01C2F20001C95C814273
:106BB0001DD040F67C04C2F20004E0544FEA5310AA
:106BC00040F6D401C2F2000103F01F034FF00104AC
:106BD00004FA03F351F820401C4341F8204040F6EA
:106BE000F000C2F20000016801F10101016002F150
:106BF000010240F67603C2F200031A7040F67600F6
:106C0000C2F2000040F67701C2F20001FFF758FE21
:106C1000FFF75EFF4FF0000010BD00BF70B4039D92
:106C2000049C064628B140F6E300C2F2000000785A
:106C3000307029B140F6F400C2F20000007808700C
:106C40002AB140F6E001C2F20001087810702BB1C1
:106C500040F6F502C2F20002117819702DB140F62B
:106C60007603C2F20003187828702CB140F6770240
:106C7000C2F200021178217070BC704706281DD83E
:106C8000002808BF022040F6E303C2F20003187098
:106C90004DF25823C0F6030313F8101040F6E1023A
:106CA000C2F20002117003EB4000417840F6E203AB
:106CB000C2F2000319704FF0010070474FF000005E
:106CC000704700BF10B540F6F403C2F200034FF066
:106CD00001021A704FF00200FFF7D0FF4FF00004DE
:106CE00040F67800C2F20000046040F6E801C2F20B
:106CF00000010C604DF25420C0F603004FF08701F4
:106D000047F26922C0F6020201F04CF940F6EC03AA
:106D1000C2F2000318604FF00C002146FFF7EEFEB0
:106D200010BD00BF034628B140F6E100C2F20000EA
:106D30000078187029B140F6E203C2F20003187817
:106D400008702AB140F6F001C2F200010B6813602E
:106D500040F67C00C2F20000704700BF2DE9F04110
:106D600040F67C07C2F200073F1853284DD8002A8E
:106D70004BD03B4607F1010702F1FF3257FA82F789
:106D80004FF0000640F6D404C2F200044FF00105B3
:106D90006FEA030C0CEB070202EA050C13F8018BF7
:106DA00001F1FF3111F8012F904530D13EE013F889
:106DB00001CB01F1010049788C450ED003F8011C8C
:106DC0004FEA521102F01F0605FA06FC54F8216042
:106DD0004CEA060644F821602E4602F10102D2B2C6
:106DE000542A07D013F801CB00F101014078844503
:106DF00043D151E04EB140F6F003C2F200031968EE
:106E000001F101011960FFF763FEBDE8F08103F8AD
:106E1000012C4FEA501600F01F0805FA08F854F844
:106E2000262048EA020244F826202E4600F10100FE
:106E3000C2B2542ADED0BB42DCD0BCF1000FB6D0C7
:106E400013F801CB11F8010F84450ED003F8010CA3
:106E50004FEA521002F01F0605FA06FC54F82060B3
:106E60004CEA060644F820602E4602F10102D2B236
:106E7000542ABFD0BB429AD1BCE703F8010C4FEAB9
:106E8000521002F01F0605FA06FC54F820604CEA86
:106E9000060644F820602E4602F10102D2B2542ABE
:106EA000A8D0BB4283D1A5E740F6D003C2F20003CD
:106EB0004FF000021A7070474FF05400704700BF47
:106EC00038B540F6D003C2F20003187868B14FF02D
:106ED000050540F6D004C2F20004FBF705FA284687
:106EE00001F09EF821780029F7D140F6D003C2F2D4
:106EF00000034FF001021A7038BD00BF38B54FF0E3
:106F0000000240F6E803C2F200031868B0F1FF3F48
:106F100000F0CE8010B140F001010847FFF7D0FF2C
:106F200040F6F600C2F200004FF0010202704FF08E
:106F3000000340F67001C2F200010B6040F67500DC
:106F4000C2F20000037089E040F67403C2F200034D
:106F50004FF000021A704FF001026BE040F670052E
:106F6000C2F200052B684FF0010103F01F0401FA83
:106F700004F44FEA531340F6D405C2F2000555F865
:106F800023301C4245D0AAB140F67501C2F200017F
:106F90000978FFF783FD40F6E800C2F20000494B94
:106FA00003604FF0010038BD40F6E804C2F200046F
:106FB000444A226040F67004C2F2000421684FF097
:106FC000010040F67C02C2F20002515CFFF700FDB6
:106FD00020684FEA501240F6D403C2F2000300F0DA
:106FE0001F044FF0010000FA04F153F8224024EA94
:106FF000010443F8224040F6E803C2F20003324A9B
:107000001A6038BD40F6E803C2F200032E4818604B
:1070100000E00A4640F67403C2F20003197801F159
:107020000101197040F67000C2F20000036803F11C
:107030000103036040F67401C2F20001087840F6D3
:10704000E103C2F200031978814287D840F6750047
:10705000C2F20000027802F10102027040F67503EC
:10706000C2F20003197840F6E200C2F20000027892
:107070009142FFF469AF40F6F603C2F200031978BB
:1070800001297FF44DAF40F6F600C2F200004FF048
:107090000002027040F67603C2F20003187840F650
:1070A0007701C2F200010978FFF7F8FCFFF7FCFE58
:1070B00040F6E801C2F200014FF000020A604FF012
:1070C000030038BDA86F02080470020808B500303C
:1070D00018BF012040F6F403C2F20003187000311B
:1070E00018BF012140F6E000C2F20000017000323A
:1070F00018BF012240F6F503C2F200031A70FFF731
:10710000DFFE40F6E401C2F20001087800B340F669
:10711000F402C2F200021378002B14BF04200020F6
:1071200040F6E001C2F200010A78002A14BF0223EF
:10713000002340F6F501C2F200010A78002A14BFCC
:107140000921082101434FF000001943FFF740FCDB
:10715000FFF7AAFE08BD00BF10B540F60043C4F219
:1071600002031A684FF0010464F387121A6018686A
:1071700064F383001860196864F3092119601A68C0
:1071800064F38B221A60186864F30D301860196874
:1071900064F38F3119604FF00000FFF7ABFB4FF045
:1071A0000300FFF7B9FB41F2040002F089FE4FF043
:1071B0000300FFF7B1FB4FF0640002F081FE4FF0D7
:1071C0000300FFF7A9FB4FF0320002F079FE4FF009
:1071D0000200FFF7A1FB4FF0320002F071FEFFF753
:1071E0006FFE4FF000004FF02801FFF7F1FB4FF06A
:1071F00000004FF00601FFF7EBFBFFF755FE40F6EE
:10720000E403C2F200031C7040F6F402C2F2000272
:10721000107840F6E001C2F20001097840F6F5036B
:10722000C2F200031A78FFF751FFFFF749FE4FF053
:1072300000002146FFF7CCFB40F2A46002F040FEC4
:10724000FFF732FEFFF73CFE40F67600C2F2000088
:10725000007840F67702C2F200021178FFF71EFCB8
:10726000FFF722FE10BD00BF10B540F6F603C2F2D4
:1072700000034FF001021A704FF47A7000F0D0FE54
:10728000FFF76AFF4FF0020402E0204600F0C8FE5C
:10729000FFF734FE0128F8D000F0FAFCF8E700BF51
:1072A0002DE9F04180460C46174640F6E403C2F251
:1072B0000003187868B94FF0320640F6E405C2F2D0
:1072C0000005FBF711F8304600F0AAFE29780029E6
:1072D000F7D04FF4FA6002F0F3FDFFF7F1FD4FF045
:1072E000000048F04001FFF773FB4FF0320002F05E
:1072F000E7FD4FEAC702D3B203F1FF37FFB2FBB19C
:1073000007F10107E7194FF001066FEA0405781944
:1073100000EA0605304614F8011BFFF759FBBC4292
:1073200022D10DE0254615F8011B3046FFF750FB32
:10733000617805F101043046FFF74AFBBC42F1D108
:1073400040F67401C2F20001087840F67502C2F2FC
:1073500000021178FFF7A2FB4FF0320002F0B0FDFF
:10736000FFF7A2FDBDE8F081002DDBD0304614F818
:10737000011BFFF72DFBBC42D4D1E1E708B540F675
:107380007602C2F20002107040F67703C2F20003E8
:10739000197010461946FFF793FA40F6E000C2F262
:1073A0000000017879B1FFF78BFD40F67602C2F25A
:1073B0000002107840F67703C2F200031978FFF755
:1073C0006DFBFFF771FD08BD10B5044640F6F800EF
:1073D000C2F2000001F0C2F92CB140F62710C2F24F
:1073E0000000017804E040F62613C2F20003197889
:1073F00040F62412C2F20002117040F62513C2F2C8
:1074000000031C704FF00300FBF774F810BD00BFC1
:1074100010B582B040F62014C2F20004206800309B
:1074200018BF0120FFF7D0FF216879B14FF00003AA
:107430000093019340F6F800C2F200004FF0FF0203
:1074400047F2C933C0F6020301F02EFA02B010BDB4
:1074500010B5082824DC082925DC002804DB40F6C8
:107460002614C2F200042070002904DB40F6271025
:10747000C2F200000170002A08DBC2EB02124FEAE0
:10748000820040F62011C2F20001086040F61C1292
:10749000C2F200021370FFF7BBFF4FF0010010BDF6
:1074A0004FF0000010BD4FF0000010BD40F6241357
:1074B000C2F2000318787047034628B10868834277
:1074C00014BF0020012070474FF00000704700BF3C
:1074D00010B440F64C13C2F2000353E8002F02F13F
:1074E000010243E800210129F7D00468C4B16268B1
:1074F000824202D19268626002E0436881689960CA
:107500002368834202D15B68236002E0826841689D
:107510005160A26802F1FF31A1604FF000040460E5
:1075200040F64C13C2F2000353E8002FA2F101020F
:1075300043E80024012CF7D053E8002FB2F1004FAC
:107540000DD14FF0000243E80024012CF4D04EF698
:107550000450CEF20000016841F080510160BFF399
:107560002F8F10BC704700BF38B504460D464FF052
:1075700000014FF0100212F03FFDE56038BD00BF82
:10758000F8B504460F46C6688D192946FFF794FFE3
:1075900000283CD140F64C13C2F2000353E8002F00
:1075A00002F1010243E800210129F7D04FF0000069
:1075B00068606168A96001B14D60226802B9256008
:1075C0006560BC51A36803F10103A36040F64C134E
:1075D000C2F2000353E8002FA2F1010243E80024A5
:1075E000012CF7D053E8002FB2F1004F0DD14FF02E
:1075F000000243E80024012CF4D04EF60450CEF2F1
:107600000000016841F080510160BFF32F8FF8BD89
:107610002DE9F04104468846C6688D199719C2B90C
:1076200040F64C13C2F2000353E8002F02F10102AE
:1076300043E800210129F7D002686A6005604FF035
:107640000000A860616809B9656020E06B689D6012
:107650001DE03946FFF730FF00283FD02846FFF7EE
:1076600037FF40F64C13C2F2000353E8002F02F13B
:10767000010243E800210129F7D0B868A8606F60D3
:10768000BD602168B9420EBF2560A9684D6048F809
:107690000640A26802F10102A26040F64C13C2F259
:1076A000000353E8002FA2F1010243E80024012C5B
:1076B000F7D053E8002FB2F1004F0DD14FF0000288
:1076C00043E80024012CF4D04EF60450CEF2000022
:1076D000016841F080510160BFF32F8FBDE8F08158
:1076E000C368C918486808B1C01A70474FF0000055
:1076F000704700BF036813B1C068181A70474FF095
:107700000000704708B5C368C918FFF7D5FE08BD6B
:1077100008B5C0680818FFF7DBFE08BD08B540F6DD
:107720002810C2F200004FF01C01FFF71DFF08BD3A
:1077300070B5054600F108063046FFF7DBFF04464A
:10774000686050B130462146FFF7E2FF4FF001007C
:10775000A861204600F0CEFA70BD4FF00003AB6187
:1077600070BD00BF38B504460D464FF000014FF024
:10777000280212F041FC204640F8085B4FF01C0143
:10778000FFF7F2FE40F62810C2F200002146FFF794
:10779000F7FE38BD2DE9F0410746884643F25453C1
:1077A000C2F200031868002800F0FE8040F64C1476
:1077B000C2F2000454E8002F02F1010244E8002163
:1077C0000129F7D0796831B143F25452C2F2000274
:1077D000136899422ED143F25450C2F2000004685B
:1077E0007C60B96901F10101B96140F64C13C2F244
:1077F000000353E8002FA2F1010243E80024012C0A
:10780000F7D053E8002FB2F1004F0DD14FF0000236
:1078100043E80024012CF4D04EF60450CEF20000D0
:10782000016841F080510160BFF32F8F4FF00100DC
:10783000BDE8F081B8F1FF3F24D140F64C13C2F20D
:10784000000353E8002FA2F1010243E80024012CB9
:10785000F7D053E8002FB2F1004F0DD14FF00002E6
:1078600043E80024012CF4D04EF60450CEF2000080
:10787000016841F080510160BFF32F8F4FF000008D
:10788000BDE8F08107F108052846FFF733FF0246FF
:10789000F0B143F25456C2F20006306892F8294023
:1078A00090F829108C4208D912E0336892F8290028
:1078B00093F82940A04204D90AE043F25456C2F298
:1078C000000628461146FFF70BFF02460028ECD1C0
:1078D000284643F25451C2F200010968FFF798FEAE
:1078E00040F64C16C2F2000656E8002FA2F1010243
:1078F00046E80024012CF7D056E8002FB2F1004FE3
:107900000DD14FF0000246E80024012CF4D04EF6D1
:107910000450CEF20000016841F080510160BFF3D5
:107920002F8FB8F1000F04D008EB880000F078FB2F
:1079300001E000F0ADF940F64C14C2F2000454E846
:10794000003F03F1010344E80032012AF7D043F27B
:107950005456C2F2000628463168FFF7D9FE54E8B3
:10796000003FA3F1010344E80032012AF7D054E8B4
:10797000003FB3F1004F0DD14FF0000344E8003257
:10798000012AF4D04EF60450CEF20000016841F016
:1079900080510160BFF32F8F78683268904214BF26
:1079A00000200120BDE8F0814FF00100BDE8F0812A
:1079B00010B5044643F25453C2F20003186800287D
:1079C00060D06268904201D0F8F738FF40F64C135F
:1079D000C2F2000353E8002F02F1010243E8002144
:1079E0000129F7D0A16901F1FF30A06118B340F679
:1079F0004C13C2F2000353E8002FA2F1010243E846
:107A00000024012CF7D053E8002FB2F1004F0DD124
:107A10004FF0000243E80024012CF4D04EF604504D
:107A2000CEF20000016841F080510160BFF32F8F5A
:107A30004FF0000010BD2046FFF77AFE40F64C13D1
:107A4000C2F2000353E8002FA2F1010243E8002430
:107A5000012CF7D053E8002FB2F1004F0DD14FF0B9
:107A6000000243E80024012CF4D04EF60450CEF27C
:107A70000000016841F080510160BFF32F8F4FF08B
:107A8000010010BD4FF0010010BD00BFF8B5054664
:107A900040F64C13C2F2000353E8002F02F101023A
:107AA00043E800210129F7D040F62810C2F2000077
:107AB000FFF720FE0446E0B140F62817C2F20007A7
:107AC0006068A84203D12046FFF732FE0AE004F1C5
:107AD000080630462946FFF715FE18B130462946FC
:107AE000FFF716FE38462146FFF7FAFD0446002848
:107AF000E6D140F64C13C2F2000353E8002FA2F186
:107B0000010243E80024012CF7D053E8002FB2F122
:107B1000004F0DD14FF0000243E80024012CF4D0B7
:107B20004EF60450CEF20000016841F08051016031
:107B3000BFF32F8FF8BD00BF02282BD111F0030F28
:107B40001FD148F21F52C5F2EB12A2FB01204FEAEF
:107B500050134FF0640202FB131083B2A3B948F232
:107B60001F52C5F2EB12A2FB01204FEAD0134FF4D3
:107B7000C87202FB131188B2D0F1010338BF002391
:107B800004E04FF0000301E04FF0010303F11C0398
:107B9000D8B2704700F1FF3042F29343C9F2492353
:107BA00083FB00210B184FEAE072C2EBA301C1EB8B
:107BB000C103C21A4FF00101C8F2000111400029AF
:107BC00005DA01F1FF3060F0010101F10101C1F1BD
:107BD0001F03D8B2704700BF08B54DF26423C0F64A
:107BE0000303195C012906D011B102290BD105E06C
:107BF000FCF790FD08BD02F023F908BDF8F71EFE62
:107C00004FF0000008BD4FF0000008BD4EF60453D1
:107C1000CEF200031A6842F080501860704700BF2F
:107C20004FF0010280F8282040F64813C2F200030A
:107C300090F8291002FA01F2188802431A8070475E
:107C400010B440F64413C2F200031A68C2B1904265
:107C500013D104E088420FD102F1140203E040F690
:107C60004412C2F2000243691BB19C698169611828
:107C700099614369136003E00A4651690029E9D11B
:107C80004FF0000282614FF0FF31416110BC70473C
:107C900010B5F8F729FE044643F25453C2F200032C
:107CA000186890F82820032A1BD0F8F71DFE43F22D
:107CB0005453C2F2000319684FF0000281F82820E3
:107CC00091F82920096940F63823C2F2000343F8ED
:107CD0002210F8F713FE2046F8F710FEFFF796FF84
:107CE00010BD4FF0020180F828102046F8F706FE7C
:107CF00010BD00BF38B5044690B3036883B3F8F7EE
:107D0000F3FD054694F8280010BB2046FFF788FFD6
:107D100043F25451C2F200010B6843B194F8292098
:107D200093F8290020F00101531A002B15DA40F6D0
:107D30004C12C2F20002106838B140F0004140F627
:107D40004C13C2F20003196007E0FFF75FFF04E085
:107D5000022804BF032084F828002846F8F7CEFD47
:107D600038BD00BF2DE9F04F85B006460F4693465B
:107D700098460F9DDDF84090F8F7B6FD824640F634
:107D80009013C2F200031968504881420FD240F2AA
:107D90000002C2F2020252F82C4C54B14C4B1C4669
:107DA0008B4207D953F82C090028F8D102E0474C40
:107DB00000E0464CA14206D1A1F12C0140F6901200
:107DC000C2F20002116020464FF000014FF02C0279
:107DD00012F012F94FF0FF3161611EB94DF26826C1
:107DE000C0F603062660B8F1000F08D00E9B042BE6
:107DF00008D9184600F103004FEA900604E04FF05E
:107E0000000601E04FF000060DBB44F25809C2F233
:107E1000000940F63815C2F20005296848F28120B1
:107E2000C0F602000090CDF80480029648464FF05C
:107E300000025B46F9F790F82A68A260E0604FEA1A
:107E4000800153182B60C1EB0900606020E02846D8
:107E50004FF0FF314A46F8F701FD4AF2ED52CDF6F8
:107E6000CE622A60E56005EB8905656048F28121F4
:107E7000C0F602010091CDF80480029628462946FA
:107E80004FF001025B46F9F767F8A5EB80036360EA
:107E90006FEA0702C2F3C01101EB470707F0FF07C3
:107EA00084F8297040F65013C2F2000353F82700FB
:107EB000206143F827405046F8F720FD2046FFF7A1
:107EC00019FF204605B0BDE8F08F00BFD4FF0120A8
:107ED000A8FF012030B585B04FF0000143F25453A4
:107EE000C2F200031960284C40F20005C2F20205FC
:107EF0002A1B20464FEAA202F8F7B0FC40F63810E1
:107F0000C2F200000460A5F12C0540F69011C2F207
:107F100000010D6043F65803C2F200034FF0B504B0
:107F2000CBF26B141C6003F14C004FF0FF3243F8AE
:107F3000042F43F8042F43F8042F8342F9D14FF064
:107F40000004009440F69411C2F2000101914FF038
:107F5000280302934DF27420C0F603004FF007018E
:107F600048F20102C0F602022346FFF7FBFE40F68C
:107F70003422C2F20002106040F65010C2F200003B
:107F8000C46305B030BD00BF5C40002010B584B0B4
:107F9000069C00944FF0000401940294FFF7E2FE67
:107FA00004B010BD00B585B04FF0000300930193FD
:107FB0000293FFF7D7FE05B000BD00BF38B543F20E
:107FC0005453C2F200031868C0B1F8F78DFC05469F
:107FD00043F25454C2F200042068FFF721FE2168E6
:107FE00091F82920086940F63823C2F2000343F8CB
:107FF00022002846F8F782FCFFF708FE38BD00BFD4
:1080000038B543F25455C2F2000540F65014C2F29E
:1080100000042B6822681A61FFF7D0FFF9E700BF60
:1080200038B543F25453C2F200031968002900F036
:10803000918020B9FFF7C2FF4FF001029AE0B0F142
:10804000FF3F04D1FFF724FE4FF0000292E040F61C
:108050004C14C2F2000454E8002F02F1010244E87B
:1080600000210129F7D040F64412C2F2000215683F
:10807000002D7AD0AB6998426FD3C01A05F1140174
:108080006D691DB1AB698342F7D96AE043F254557B
:10809000C2F200052B689861086858611846F8F725
:1080A000D1FB40F64C14C2F2000454E8003FA3F1A7
:1080B000010344E80032012AF7D054E8003FB3F14D
:1080C000004F0DD14FF0000344E80032012AF4D0F4
:1080D0004EF60450CEF20000016841F0805101607C
:1080E000BFF32F8FFFF7D4FD54E8003F03F10103E6
:1080F00044E80032012AF7D028684169B1F1FF3F16
:1081000004D0FFF79DFD4FF0000201E04FF00102A7
:1081100040F64C13C2F2000353E8004FA4F10104EF
:1081200043E80045012DF7D053E8004FB4F1004F6C
:108130000DD14FF0000443E80045012DF4D04EF678
:108140000450CEF20000016841F080510160BFF39D
:108150002F8F0FE04FF001020CE040F64411C2F205
:108160000001AC69221AAA6190E740F64411C2F2FC
:1081700000018BE7104638BDF8B5044600287AD0D8
:10818000F8F7B2FB064640F69013C2F200031968F6
:108190003948814211D240F20002C2F2020252F882
:1081A0001C5CA54263D0354B1D468B4205D9A3F11B
:1081B0002C03D86BA042F7D15AE094F8293040F64E
:1081C0005012C2F2000252F82300A04206D1016907
:1081D00040F65012C2F2000242F823102046FFF788
:1081E0002FFD2046FFF752FC94F82900236940F642
:1081F0003821C2F2000141F8203043F25452C2F259
:1082000000021068A04229D0A06838B3E76800EBEC
:10821000870540F63817C2F200073B685A1B29460B
:108220004FEAA2024FF00003FBF762F8E1683868FA
:10823000A0EB81033B6040F69012C2F2000211688D
:108240000D4B99420AD29A68954203D8E068A2EB96
:1082500080029A60A3F12C038B42F4D84FF0000106
:10826000216084F828103046F8F748FBF8BD024D2D
:1082700021692961A1E7F8BDD4FF0120A8FF0120F1
:1082800000BFF04772B643F25454C2F200042068B3
:10829000FFF772FF4FF000032360F8F7ADFE00BF59
:1082A00040F64413C2F20003196849B1886950B11D
:1082B00000F1FF328A61D2F1010038BF002070471F
:1082C0004FF0000070474FF00000704770B540F667
:1082D0004413C2F200031C68A4B1A06990B940F62F
:1082E0004415C2F200054FF0FF3660692946F8F7E1
:1082F000A9FA66612046FFF7FDFC2C6814B1A1695C
:108300000029F2D070BD00BFF0B472B640F6481339
:10831000C2F200031C882CB940F63423C2F20003D9
:1083200018685FE04DF27C2CC0F6030C40F638254F
:10833000C2F2000540F65016C2F20006C4F1000376
:1083400023401A0A1ABF1CF8021008311CF8031047
:1083500011F0010F0AD141F0010055F8200038B1A9
:1083600090F82820012A38D81F4602E01F4600E076
:108370001F4655F82120B2B192F828307BB140F663
:108380004810C2F20000048010462BE090F828301C
:1083900033B140F64812C2F20002148022E01046C7
:1083A00000690028F2D156F82100824207D1BC436F
:1083B000C4D140F64811C2F200010C80ACE745F888
:1083C000210011F0010FD4D114EA4703D1D04FEAB4
:1083D0004707BFB241F00101CBE740F64811C2F2B6
:1083E00000010C8062B6F0BC704700BF70B543F26C
:1083F0005453C2F200031B6883420FD193F8282024
:10840000012A9CBF022283F8282093F8291040F605
:108410003820C2F2000040F8213070BD40F63C1216
:10842000C2F20002136043F25451C2F2000108602C
:1084300090F8292040F63823C2F2000343F82200C6
:1084400090F8281001299CBF022180F8281082682A
:10845000AAB9C1684AF2ED53CDF6CE6308689842D6
:1084600001D0F8F7EBF943F25452C2F2000211685E
:108470004868CB6898427ED2F8F7E0F970BD40F6C4
:108480004013C2F200031B68984274D093B358683B
:1084900044F25804C2F20004251A4FEAA501D9603B
:1084A00043F65802C2F2000290420AD34FF0B503DD
:1084B000CBF26B1343F65800C2F2000004689C42F2
:1084C00001D0F8F7BBF940F64015C2F200052A6862
:1084D00040F63814C2F2000420685168D2684FF0A8
:1084E0000003FAF705FF296823688B60C86803EB6F
:1084F0008002226043F25451C2F200010B6840F640
:108500004010C2F200000360DA68002A33D05868D5
:1085100099684FF00103FAF7EBFE43F25456C2F2AA
:1085200000063568A868EC6800EB840440F638164D
:10853000C2F200063268131B21464FEAA3024FF035
:108540000003FAF7D5FEE9683068A0EB81023260DB
:1085500040F69013C2F200031968074B99420AD201
:108560009A68944203D8E868A2EB80029A60A3F16B
:108570002C038B42F4D870BDD4FF012000B585B028
:1085800040F6D430C2F200004FF00001FEF7ECFFDD
:1085900040F67C20C2F200004FF00001FEF7E4FF3D
:1085A0004FF00003009340F69422C2F200020192C1
:1085B0004FF0500002904DF27C30C0F60300194697
:1085C00048F6F902C0F60202FFF7CCFB40F678232A
:1085D000C2F20003186005B000BD00BF08B5FFF788
:1085E00089F8034648B1C06850B100F1FF31D96045
:1085F000D1F1010038BF002008BD4FF0000008BDD8
:108600004FF0000008BD00BF70B505460E46144689
:1086100040F64C13C2F2000353E8002F02F10102AE
:1086200043E800210129F7D0FFF764F8024600284B
:1086300039D0C06884422DD3241A28461146FFF74A
:108640004FF8024600282ED0C068A042F4D921E09D
:1086500040F64C13C2F2000353E8002FA2F10102CE
:1086600043E80024012CF7D053E8002FB2F1004F6B
:108670000DD14FF0000243E80024012CF4D04EF657
:108680000450CEF20000016841F080510160BFF358
:108690002F8F70BDF460D1680B1BD3602846314624
:1086A000FEF7B6FFD4E7F46028463146FEF768FFD0
:1086B000CEE700BFF8B50646FFF71CF80446F8B150
:1086C000C368EBB930462146FFF70AF80546F8F7CC
:1086D0000BF9074630462146FFF71AF83846F8F7F7
:1086E0000DF922691AB130462146FFF78DFF04F1DA
:1086F0001400FDF769F91DB12C46E8680028E1D0A7
:10870000F8BD00BF08B540F69023C2F200031A6816
:1087100002F101021A6040F67C20C2F20000FFF76D
:108720005DFF28B140F67C20C2F20000FFF7C2FFD7
:1087300008BD00BF08B5014640F6D430C2F20000C3
:10874000FEF7E0FF20B140F6D430C2F2000008BDD1
:1087500040F67C20C2F2000008BD00BF70B50446A0
:1087600040F64C13C2F2000353E8002F02F101025D
:1087700043E800210129F7D0FFF7DCFF0546214639
:10878000FEF7C0FF002845D040F64C10C2F20000B2
:1087900050E8002F02F1010240E800210129F7D042
:1087A00028462146FEF79CFF18B1C168E2688B1885
:1087B000C360F8F799F8064628462146FEF7A8FF59
:1087C0003046F8F79BF84FF0FF35E56040F64C1364
:1087D000C2F2000353E8002FA2F1010243E8002592
:1087E000012DF7D053E8002FB2F1004F0DD14FF01B
:1087F000000243E80025012DF4D04EF60450CEF2DD
:108800000000016841F080510160BFF32F8F4FF0ED
:10881000010501E04FF0000504F11400FDF7CEF86A
:1088200040F64C13C2F2000353E8002FA2F10102FC
:1088300043E80024012CF7D053E8002FB2F1004F99
:108840000DD14FF0000243E80024012CF4D04EF685
:108850000450CEF20000016841F080510160BFF386
:108860002F8F284670BD00BF2DE9F04105460F4609
:1088700014469846FFF772FF064694B19DF82030E3
:10888000002B14BF20460020286105F1140041464A
:10889000069A079BFDF778F8384629462246FFF7E7
:1088A000B3FE3046BDE8F08170B584B00E46154683
:1088B0000093089C01949DF82430029340F67C219B
:1088C000C2F2000132462B46FFF7CEFF04B070BD66
:1088D00070B584B00E4615460093089C01949DF82F
:1088E0002430029340F6D431C2F2000132462B46C6
:1088F000FFF7BAFF04B070BD00B583B04FF00003BE
:1089000000934FF00100019040F6E430C2F2000005
:1089100041F288314FF0FF0248F20573C0F60203BE
:10892000FFF7D6FF40F6D434C2F20004FFF7CEFCC6
:108930002046FFF7BFFEFFF7ABF9F7E740F68C23C1
:10894000C2F2000318681A689042FBD1704700BF5A
:1089500010B540F68C23C2F200031A6802F101023E
:108960001A60FFF79DFC044640F6D430C2F20000C6
:10897000FFF734FE204310F0FF0F06D040F67820BA
:10898000C2F200000068FFF7B5F910BD08B54DF25E
:108990001840C0F603004FF0060148F6C952C0F671
:1089A0000202FFF7FFFA40F61473C2F200031860E8
:1089B00008BD00BF38B504460D4640F60843C2F274
:1089C0000003586AA0420AD040F60841C2F20001F2
:1089D0004C620A681AB115B14948FCF7F5FF40F638
:1089E0000843C2F20003186F84420AD040F60841DF
:1089F000C2F200010C67CA6C1AB115B14148FCF70C
:108A0000E3FF40F60843C2F20003D3F8BC008442FF
:108A10000CD040F60841C2F20001C1F8BC40D1F8C8
:108A200098201AB115B13848FCF7CEFF40F608433C
:108A3000C2F20003D3F8080184420CD040F608418A
:108A4000C2F20001C1F80841D1F8E4201AB115B111
:108A50002E48FCF7B9FF40F60843C2F20003D3F8F2
:108A6000540184420CD040F60841C2F20001C1F822
:108A70005441D1F830211AB115B12548FCF7A4FFB3
:108A800040F60843C2F20003D3F8A00184420CD0A0
:108A900040F60841C2F20001C1F8A041D1F87C21A2
:108AA0001AB115B11B48FCF78FFF40F60843C2F21C
:108AB0000003D3F8EC0184420CD040F60841C2F226
:108AC0000001C1F8EC41D1F8C8211AB115B1124822
:108AD000FCF77AFF40F60843C2F20003D3F83802ED
:108AE000A0420CD040F60841C2F20001C1F8384261
:108AF000D1F814221AB115B10848FCF765FF38BD4A
:108B0000180C0020640C0020B00C0020FC0C00208D
:108B1000480D0020940D0020E00D00202C0E0020B8
:108B20002DE9F04707460D4691460898DDF8288064
:108B30000C683E68D8F800108A19944202D80219CD
:108B4000964203D304192C60BDE8F087341B061B42
:108B5000B14234BF8A46B246099931B1D9F8000012
:108B600008181919524611F023FAD8F80030CAEB48
:108B70000302C8F800203E6806EB0A013960D9F804
:108B8000000000EB0A03C9F800302E68A419544411
:108B90002C60BDE8F08700BF70B584B09CF8196008
:108BA000157A947B4FF007038CF810304FF00502D4
:108BB0008CF8112006F00F0260F3C7128CF8122017
:108BC0004FF0000065F301008CF813004FF0000235
:108BD00061F30A02ACF814208CF81640DCF80C1093
:108BE0000093DCF804300193CDF808C001F10400D3
:108BF0000CF108020CF11003FFF792FF04B070BDF6
:108C00002DE9F04F8FB00746059114464FF0000351
:108C10000793136012896068131A8B4238BF05935B
:108C20000599002900F0AA8040F61875C2F20005E7
:108C30002D6815B34FEAC5054FF000024FF0FF0154
:108C4000134640F62070C2F20000A5F10806C6F3F4
:108C5000C00E1658F6798E4240F0958096E0165870
:108C6000F6798E421CBF0133314602F10802865864
:108C7000F6798E4240F09F80A0E04FF0000303EBB6
:108C800043024FEAC20000F1100008904FF48071D7
:108C9000ADF824104FF00402ADF826208DF82830EE
:108CA0000DF129004FF000014FF0070211F0A4F977
:108CB00004F1040B04944FF010030093019705A8EE
:108CC00002905846214607AA08ABFFF729FF0599ED
:108CD000002951D04FF001028DF821200DF1320012
:108CE0004FF000014FF0060211F086F940F61873BC
:108CF000C2F20003186800283ED04FF0FF014FF089
:108D0000000440F62079C2F200094DF28838C0F61E
:108D1000030840F6187AC2F2000A59F83450ED7987
:108D20008D4223D08DF820404FEA05160DF1220028
:108D300008EB06014FF0080211F03AF906F10801BC
:108D40000DF12A0041444FF0080211F031F94FF0C3
:108D500018020092019705AB02935846049907AA9E
:108D600008ABFFF7DDFE059830B1294604F1010498
:108D7000DAF80020A242D0D8079801E04FF0FF3087
:108D80000FB0BDE8F08F03F10103314602F1080294
:108D9000AA423FF474AFBEF1000F3FF460AF165823
:108DA000F6798E421CBF0133314602F10802AA4215
:108DB0007FF455AF63E703F10103314602F1080286
:108DC000AA427FF44CAF5AE72DE9F0414FF0010081
:108DD000FCF7A4FC4DF20840C0F60300FCF722FBB0
:108DE00040F64C73C2F200034FF001021A7040F6D5
:108DF000D060C2F20000016841B940F6D064C2F20E
:108E00000004FEF745FF2568002DFAD040F61D77D7
:108E1000C2F2000740F64C74C2F2000440F66866E5
:108E2000C2F2000640F64075C2F2000540F6CC687A
:108E3000C2F200083B783BB14FF000023A704FF0AD
:108E400002002070FCF764FC317859B14FF0000348
:108E50003370227862F07F0020704FF001000146ED
:108E6000FFF7A8FD297851B14FF000002870237852
:108E700003F07F0222704FF00101FFF79BFD98F88D
:108E8000000010B9FEF704FFD4E740F64C71C2F2BF
:108E900000014FF002030B704FF00000FCF73EFCA6
:108EA000BDE8F08108B540F6D063C2F20003186057
:108EB00040F61470C2F200000068FEF71BFF08BD08
:108EC00070B505460E4640F66473C2F2000318689A
:108ED000032801D9F7F7B2FC40F66472C2F200022F
:108EE000116840F6AC64C2F2000444F8316004EB4F
:108EF000C104656001F10101116070BD70B50546E6
:108F00000C461646032801D9F7F798FC40F6207363
:108F1000C2F2000353F8350008B1F7F78FFC40F6B2
:108F20002071C2F2000141F8354001EBC5056E60C9
:108F300040F61873C2F200031A6802F101021A60C7
:108F4000206930B1FCF76EFA04F1040420690028AE
:108F5000F8D170BD08B540F60843C2F200031968A5
:108F600081425AD040F60842C2F20002D36C8342DA
:108F700034D040F60841C2F20001D1F89820824274
:108F80002FD040F60843C2F20003D3F8E410814228
:108F90002AD040F60842C2F20002D2F830318342B1
:108FA00025D040F60841C2F20001D1F87C2182426E
:108FB00020D040F60843C2F20003D3F8C811814222
:108FC0001BD040F60842C2F20002D2F814328342AB
:108FD00016D0F7F733FC4FF0080013E04FF0010014
:108FE00010E04FF002000DE04FF003000AE04FF0F8
:108FF000040007E04FF0050004E04FF0060001E038
:109000004FF0070040F60841C2F200014FF04C0259
:1090100002FB001090F8200008BD4FF00000F1E7BF
:109020002DE9F04F8FB0089007910A924FF000039E
:1090300009931360546813891B1B8B4238BF079335
:109040000799002900F04A81082C69D840F6187465
:10905000C2F20004D4F800E040F66475C2F20005E4
:109060002E680EEBCE0707EBC60404F109044FF09F
:10907000000140F62077C2F20007CB598BB1DD68C2
:10908000641903F110051B695BB15E890EB104F12F
:1090900007049B890BB104F1070455F8043F002B2A
:1090A000F3D101F108012029E7D140F6D061C2F2E5
:1090B00000010D682F7E6E7EEB8A03F10103C3F37E
:1090C00047054FF000010C914FF009038DF82C304B
:1090D0004FF002018DF82D10ADF82E408DF830E0E4
:1090E0004FF001018DF831104FF0000167F3451189
:1090F00066F3861161F07F018DF833108DF83450DE
:109100000093019007A8029002F10400114609AAF9
:109110000BABFFF705FD079A002A00F0DD80E0E0C9
:109120004FF009001060DCE05BF83640002C00F0E6
:10913000CE80059D286800284BD07A68B2420CD0BA
:109140004FF0000310F0010F3ED1DFE007EBC30248
:109150005268B24240F0E38001E04FF0000357F85C
:109160003300D2B290F8048090F805C090F806E081
:10917000C579016819B143F01000C3B201E04FF0A6
:1091800000034FF008008DF82C004FF00B018DF814
:109190002D108DF82E208DF82F808DF830C08DF891
:1091A00031E08DF832508DF833300A990090089AEA
:1091B000019207AB029301F1040009AA0BABFFF780
:1091C000AFFC079828B987E003F101052B468542DB
:1091D000BCD104F1100523697BB129464FF0000290
:1091E000588908B102F101029B890BB102F1010219
:1091F00051F8043F002BF3D101E04FF000025FFA79
:1092000086FCD2B294F804E06079A17923681BB19E
:1092100046F02003DBB201E04FF000038DF82CA0F4
:109220004FF004088DF82D808DF82EC04FF0000C03
:109230008DF82FC08DF830208DF831E08DF8320098
:109240008DF833108DF834300A99CDF800A0089AC3
:10925000019207A8029001EB080009AA0BABFFF7E7
:109260005FFC0799002937D0A3686BB10A99E268BF
:1092700000920898019007AA029201EB080009AA3F
:10928000FFF74EFC079B3BB3246904B34FF0010882
:109290004FF000092046FFF75DFE8DF8350061892B
:1092A00039B10DF11C0C40462246FFF775FC0799B9
:1092B00091B1A18939B10DF11C0C48462246FFF746
:1092C0006BFC079840B155F8044F002CE2D106F131
:1092D0000106042E7FF428AF099814E04FF0FF3008
:1092E00011E04FF0000640F6207BC2F2000B40F682
:1092F0006474C2F2000405944FF0090A40F6AC67AA
:10930000C2F2000710E70FB0BDE8F08F03F10103D0
:1093100007EBC3014A68B2427FF456AF1FE705F17D
:10932000010307EBC3014A68B2427FF44DAF16E771
:1093300008B540F65073C2F200031A5C40F60841CB
:10934000C2F200014FF04C0000FB0210436AD3F15F
:10935000010238BF002242634FF00001C163016483
:10936000416400F11000FCF72FFB08BD2DE9F84F18
:1093700081468A4640F65073C2F200031A5C40F6FA
:109380000840C2F200004FF04C0404FB020404F158
:1093900048064FF001084FF0000740F6D46BC2F2C8
:1093A000000B354640463146F7F74CFA30B14FF0E6
:1093B00002003146F7F746FABDE8F88FBAF1000F20
:1093C00005D148464146FBF759FF032827D0256CB5
:1093D00075B15846A168E26BA8470546B0F1FF3F5A
:1093E00014D06064484659462A46FBF76DFF0EE0EC
:1093F000616CA5688D4228BF0D464846E16B2A4640
:10940000FBF762FFE36B5A19E26300E03D46606CD4
:10941000A16888423CBFE7632764451B6564384602
:109420003146F7F70FFA0228BBD0BDE8F88F00BF2E
:10943000F8B505460E46174640F65073C2F20003D3
:109440001A5C40F60840C2F200004FF04C0404FBE6
:1094500002044FF00000FBF769FEE76326644FF05B
:109460000001616428464FF00101FFF77FFF4FF0D4
:109470000100FBF75BFEF8BDF8B505460F46164642
:1094800040F65073C2F200031A5C40F60840C2F284
:1094900000004FF04C0404FB0204A168B1420DD25D
:1094A00043F65803C2F200039F4207D344F2580226
:1094B000C2F20002974201D2F7F7C0F94FF0000064
:1094C000FBF734FEE7634FF0000020646664284633
:1094D0004FF00101FFF74AFF4FF00100FBF726FEB6
:1094E000F8BD00BF08B5FBF777FF08BD70B586B0C3
:1094F00005460C46164602A8F8F7BCFB01462EB1FD
:1095000002A82A46234600F0A5FD07E04FF001031C
:10951000009302A82A46234600F04EFE06B070BD16
:1095200070B58AB00378212B00F0938004D86BB11A
:10953000012B40F0D88186E0A12B00F0A781C02B41
:1095400000F0B481802B40F0CE8195E04178052970
:1095500003D0092940F0CA8146E0408840F64C72A9
:10956000C2F200021378022B02D0032B33D118E091
:1095700000F1FF318AB27E2A30D8C0B240F6607363
:10958000C2F2000318704FF00201FCF731F840F608
:109590004C70C2F200004FF0030101704FF0010067
:1095A000C3E170B940F66072C2F20002107040F67A
:1095B0004C70C2F200004FF0020303704FF0010044
:1095C000B3E17F280DD840F66071C2F20001087047
:1095D0004FF00100A9E14FF00200A6E14FF00200B8
:1095E000A3E14FF00200A0E1827840F64C73C2F292
:1095F00000031978022923D972B940F64C73C2F2DC
:1096000000034FF0030119704FF001000146FFF70E
:10961000D1F94FF0010088E1012A18BF022040F083
:10962000848140F64C70C2F200004FF004020270D8
:109630004FF000000146FFF7BDF94FF0010074E163
:109640004FF0020071E140780B280CBF012002208E
:109650006BE18388032B00F24C8140F62074C2F248
:10966000000404EBC3035B68002B00F045819847BE
:10967000002808BF022058E142781AB1062A40F0BB
:109680003E8121E0C18802291BD14FF00000ADF8D6
:10969000040040F6D062C2F2000212680346517E16
:1096A00061F30003ADF80430127E62F341030AA9AE
:1096B00021F8243D4FF00202FFF7DEFE4FF00300D9
:1096C00033E14FF0020030E18278C1888CB2C37878
:1096D000022B2ED0032B3DD0012B40F0D48040F63E
:1096E0006C65C2F2000528464DF22C41C0F603011C
:1096F0004FF0120210F05CFC40F6D060C2F20000A5
:1097000001688A892A81CB896B81088AA8818A7C31
:109710002A71CB7C6B71097DA9714FF0000029463D
:10972000122C34BF22461222FFF7A6FE4FF0030090
:10973000FBE040F66872C2F2000211814FF00000B7
:10974000506049F22101C0F60201FFF771FE4FF0AF
:109750000300EAE0D2B940F66C64C2F2000404F1FE
:1097600002004DF22841C0F603014FF0020210F052
:109770001FFC4FF0040222704FF0030565704FF09C
:1097800000002146FFF778FE2846CEE0012A06D1E8
:1097900040F6D063C2F20003196809682FE0022A7C
:1097A00006D140F6D062C2F200021068416826E09D
:1097B000032A06D140F6D063C2F200031968896813
:1097C0001DE002F00F0022F00F03102B08D15A4BBE
:1097D000196888420EDA594A52F8300001680EE0E2
:1097E000202B07D1032805D8554951F8300008B17E
:1097F000016804E0EE2A04D04FF0020095E009B9B8
:109800003EE05049B1F1FF3F40F0888001A84FF0A1
:1098100020014FF00102FFF769FE0AAD2A184FF050
:10982000000002F8240C01A978E000F10206428051
:1098300003F10102134611F8015F5DB100F104006C
:10984000758002F1010311F8012F002A6FD101E0A8
:109850004FF0000340F66C61C2F200014FF00305C7
:109860004D7003F101034FEA4303DAB20A704FF07F
:109870000000A24228BF2246FFF7FEFD284654E022
:109880004FF0020051E04FF002004EE08388032BBE
:1098900038D840F62074C2F2000404EBC3035B68BE
:1098A0009BB39847002808BF02203EE04378212B55
:1098B0002ED1C18840F66873C2F2000319814FF0BF
:1098C00000025A608088042825D1104648F60141DC
:1098D000C0F6020140F66872C2F20002FFF7A8FD6E
:1098E0004FF0030021E04FF002001EE04FF00200B5
:1098F0001BE04FF0020018E04FF0020015E04FF0BF
:10990000020012E04FF002000FE04FF002000CE006
:109910004FF0020009E04FF0020006E00A78002A4A
:1099200096D009484FF000037FE70AB070BD1E2BA8
:109930007FF47BAF8EE700BF640F0020AC0E0020E9
:10994000200F00201CD403086C0E002010B5044624
:10995000436993B14FF00000606140F64C71C2F270
:1099600000010A78032A08D140F66073C2F20003AE
:1099700018784FF00301FBF73BFE206958B34FF016
:1099800000002061E06040F61C71C2F20001087026
:1099900040F64471C2F200014FF00802FFF7A2FD49
:1099A000082853D140F64472C2F20002137813F033
:1099B000800F06D140F64470C2F20000C188002931
:1099C00044D140F64470C2F200004FF000010A4654
:1099D000FFF7A6FD2DE0E168002937D04FF0000029
:1099E000E06040F61C72C2F20002137840F66C612F
:1099F000C2F20001C3F14002FFF774FD034628B331
:109A000040F61C70C2F2000001785A18D2B20270FF
:109A100040F64473C2F20003D888904216D140F653
:109A20004470C2F2000040F66C61C2F20001FFF720
:109A300077FD012804D0022808D1FBF72FFC10BDC8
:109A40004FF0000001460246FFF716FD10BD00BFB3
:109A500008B540F67473C2F200031B693BB14FF0C6
:109A6000000140F67472C2F200025269984740F653
:109A70007470C2F200004FF000010170416081601B
:109A8000C1600161416108BD40F67470C2F200001E
:109A900081614DF26041C0F603018A5C42778377B1
:109AA000037F6FF3070303774FF0000141627047B4
:109AB00030B583B040F67474C2F200042070089D83
:109AC0006560099DA5600A9DE5600B9D25610C9D63
:109AD00065619DF8184000949DF81C400194FFF7C3
:109AE000D3FF03B030BD00BF40F67473C2F2000371
:109AF0005B6AB3F1FF3F09D140F67471C2F2000115
:109B00004FF000034B624FF0010070473F2B0BD822
:109B100040F67472C2F20002106AC15403F10103EC
:109B200053624FF0010070474FF00000704700BFD4
:109B3000704700BF70B540F67474C2F2000404F1BF
:109B400018004DF2B441C0F603014FF0070210F0C7
:109B50002FFA4FF000004DF2BC41C0F60301FFF7B1
:109B6000AFF949F6A956C0F602064FF000004DF2D3
:109B70006441C0F603013246FFF7C0F94DF2C44517
:109B8000C0F603054FF0010029463246FFF7B6F94B
:109B90002869FFF7DFF984F8280040F6A070C2F2C8
:109BA00000004FF0070149F6B932C0F602024FF04B
:109BB0000003FBF7E9FE70BD38B541F25403C2F271
:109BC00000034FF001021A7040F67474C2F20004F0
:109BD00094F828004FF000010A46FFF74DFC60683A
:109BE00068B140F67474C2F200044FF0FF3565624C
:109BF0006368207861699847616A0029F7D040F668
:109C00007470C2F200004FF000024262836833B108
:109C100040F67471C2F2000108784969984738BD6E
:109C20002DE9F04F83B0804643680BB9806828B1B6
:109C30004FF00001C8F80810FFF7BEFFD8F80C205D
:109C4000002A45D04FF00003C8F80C30D8F80000C7
:109C500041F21401C2F200014FF04002FFF742FC52
:109C6000814640F67470C2F20000C16800292FD00E
:109C7000B9F1000F2CD040F67474C2F2000441F226
:109C80001406C2F200064FF0000509F1FF3B0BF08D
:109C9000010B2078715D2A466369E768B84705F1D2
:109CA000010AD14570D113E0207816F80A102A462F
:109CB0006369E768B8470AF1010A207816F80A10C4
:109CC0002A466369E768B8470AF1010AD145EBD132
:109CD000D8F81420002A54D04FF0000441F2540365
:109CE000C2F200031C70C8F8144040F6F070C2F2D3
:109CF0000000FEF733FD40F67470C2F200004462CB
:109D00004168002936D040F67475C2F2000540F66D
:109D1000B074C2F200042C622C46656A6268207836
:109D200061699047636A9D42F7D11DB3D8F800007E
:109D300040F6B071C2F200012A46FFF79DFB4FF0DA
:109D400000000090019040F6F070C2F200004FF069
:109D50004B014FF0FF0249F6B933C0F60203FEF79C
:109D6000B7FD0EE040F67472C2F20002107851693D
:109D7000984706E040F67471C2F200018B68002B30
:109D8000F0D103B0BDE8F08FBBF1000F8CD020788C
:109D900016F80A102A466369E768B8470AF1010A0B
:109DA000D14581D194E700BF10B544780378212BC9
:109DB00002D0A12B1BD10EE0202C04D0222C14BFEA
:109DC0000020012010BD072A14D10D4810F0F0F832
:109DD0004FF0010010BD212C0FD14FF000000849B9
:109DE0004FF00702FFF748FB4FF0030010BD4FF0A4
:109DF000000010BD4FF0020010BD4FF0000010BD7C
:109E00008C0F002008B541F25403C2F20003187809
:109E100070B940F67471C2F200014A6A72B940F634
:109E20007473C2F2000393F82800FFF781FA08BDAB
:109E300040F6A070C2F20000FBF7C6FD08BD00BFEF
:109E40004DF2F040C0F60300704700BF70B40378D5
:109E500001298CBF4478002402298CBF8578002515
:109E6000DCF8000048B34FEA93064DF22050C0F6EC
:109E70000300365C16704FEA031343EA141303F031
:109E80003F031B5C5370012907D94FEA840444EA5D
:109E9000951303F03F04205C01E04FF03D0090700B
:109EA000022907D905F03F054DF22053C0F6030300
:109EB000E95C01E04FF03D01D17070BC704700BF1C
:109EC00082B04FF015010CE00191019B03F1FF32CC
:109ED000019233B100BF019B03F1FF320192002BCD
:109EE000F8D100F1FF30B0F1FF3FEDD102B0704783
:109EF00070B4C4B24FEA10204DF2B456C0F6030657
:109F00004DF2B465C0F6030511F8013B1AB94BB91F
:109F100044EA00200BE06340F45C4440E85C013A12
:109F2000F2D1F5E76340F45C4440E85CECE770BCD8
:109F3000704700BF10B444F6FB43C0F2861311F81B
:109F4000014B02B9ACB380EA04404FEA400010F084
:109F5000807F18BF58404FEA400010F0807F18BF44
:109F600058404FEA400010F0807F18BF58404FEA39
:109F7000400010F0807F18BF58404FEA400010F0BA
:109F8000807F18BF58404FEA400010F0807F18BF14
:109F900058404FEA400010F0807F18BF58404FEA09
:109FA000400010F0807F18BF5840002AC7D0013A07
:109FB000C5D120F07F4010BC704700BF82B0019037
:109FC0009DF806304FF0000063F307009DF8052070
:109FD00062F30F209DF8042062F317409DF80720DC
:109FE00012F0800F14BF63F07F0103F07F0161F373
:109FF00007004FEA4201CAB262F31F6013F0800FFC
:10A0000018BF42F0010262F31F6002B0704700BF48
:10A0100084B0C0F307438DF80C30C0F307228DF8ED
:10A020000D20C3B24FEA10604FEA500210F0010F4A
:10A0300014BF63F07F0103F07F018DF80E1013F061
:10A04000800F18BF62F07F028DF80F20039804B0D4
:10A05000704700BF2DE9F04F83B005460F46144608
:10A060001E46019201F1FF3313F1050F44D8032E70
:10A0700043D9A6F10400C0F380080DF1040C284672
:10A08000FFF7E4FE05F10305A7F1030104F1040461
:10A09000A6F10406A7F1040717F1050F67D92CE014
:10A0A0000DF1040C284639462246FFF7CFFE05F194
:10A0B000030B5D46A7F1030104F1040A5446A6F11F
:10A0C00004094E46A7F1040717F1050F15D80F46EE
:10A0D0000DF1040C58465246FFF7B8FE0BF103058C
:10A0E000A7F103010AF10404A9F10406A7F1040889
:10A0F00018F1050F59D900E0FFE799B396B30DF1B8
:10A10000040C28466A46FFF7A1FE022E11D0032E4A
:10A1100002D0012E26D11AE0019929B19DF8002024
:10A1200022704FF0010301E04FF0000304F101043D
:10A1300001E04FF00003019830B102A9CA1812F8EB
:10A14000080C207003F1010304F1010401E04FF059
:10A150000003019921B102AAD31813F8080C20704A
:10A1600004F101040199601A03B0BDE8F08F0F46B5
:10A17000032EC2D9B8F1000F92D00DF1040C28467D
:10A180002246FFF763FE05F10305A7F1030104F181
:10A190000404A6F10406A7F1040717F1050FACD8D3
:10A1A0000F46032E3FF67CAFA7E7A7F10307032E68
:10A1B0003FF676AFA1E700BFF0B49DF81040ECB1D8
:10A1C0004FEA41079F421CD2DD1B1DD056194FF0AC
:10A1D00030046FEA0203F31803F0010302F8014BA5
:10A1E000B24240F0928007E0134603F8014B5470EE
:10A1F00003F10102B242F7D13B4607E04FF0000500
:10A2000004E04FF0000501E04FF0000500293CD0CC
:10A2100003F1FF34002B3AD000F101034118284626
:10A22000521B04F1FF3515F0020F10D032E0A4F1FB
:10A23000020603F101031F46012C29D03446B4461F
:10A2400013F8016C4FEA1616092E42D944E01E4657
:10A2500013F8015C4FEA1515092D8CBF37353035E1
:10A26000155414B900F1010012E013F8016C06F066
:10A270000F05092D8CBF373530351618757000F174
:10A28000020528468B42D2D102E0284600E028464B
:10A29000F0BC70471E4613F8015C4FEA1515092DF6
:10A2A00094BF303537351554002CDBD013F8016CD2
:10A2B00006F00F05092D94BF303537351618757027
:10A2C00000F102008B42E3D003F10103A4F1020488
:10A2D000BDE706F1300601E006F137065655BCF140
:10A2E000000FBFD013F8016C06F00F06092E94BFC3
:10A2F000303637361018467005F102008F42C7D04D
:10A3000003F10103A4F10204A1E7002B3FF46CAFB9
:10A3100002F8014BB2427FF467AF6DE7DCF814300E
:10A3200093F8452083F84420DCF8141091F8463067
:10A3300081F84530DCF8141091F8472081F8462068
:10A34000DCF8143083F84700704700BFDCF81430A5
:10A3500093F8470093F8462083F84720DCF8141060
:10A3600091F8453081F84630DCF8141091F844201B
:10A3700081F84520704700BF43F21422C2F2000268
:10A38000136840F20001C0F60101C85CC9184978A1
:10A3900003F10203136041EA00207047DCF8043047
:10A3A000DCF8082002EBD300CCF8080003F007012A
:10A3B0004FF0010303FA01F2CCF80420704700BF0C
:10A3C0002DE9F04F83B004468A4693461E46CDF8E9
:10A3D00004C04FF00007B846B9463DE02546304678
:10A3E000D047034600283DD0B9F1000F0CD12028FA
:10A3F00029D0092829D00A2829D00D2829D0022DB2
:10A400004FF0010988BF0225A3F13002D1B209291A
:10A4100010D9A3F14100C1B2052903D8A3F1370334
:10A42000D9B207E0A3F16102D0B205281AD8A3F18E
:10A430005703D9B24FEA0717FCB241EA040708F103
:10A4400001082C4606E02C4604E02C4602E02C468F
:10A4500000E02C463046D847FF2CBFD004F1FF3532
:10A46000002CBCD1DDF804C03846FFF757FF019B34
:10A470005A69D8F1010838BF4FF0000882F85080BF
:10A4800003B0BDE8F08F00BF43F2E403C2F2000363
:10A490001B684B634BB19A68824209D0DB684B63FF
:10A4A0001BB19A688242F9D102E04FF01E0070475A
:10A4B0004FF00000704700BF884204D8884234BF84
:10A4C0000220002070474FF001007047D0F804319F
:10A4D000D0F80021934214BFC05C0020704700BF39
:10A4E000D0F80431FF2B14BF01330023C0F804312E
:10A4F000704700BF10B4DCF81420D16C0B46044642
:10A5000058B14FEA016343EA116301F47F4043EA23
:10A51000002301F47F0143EA1123DCF8040030B189
:10A5200099B24FEA134060F30F0361F31F435CB924
:10A530004FEA036141EA136103F47F4041EA0021DD
:10A5400003F47F0341EA1323D36410BC704700BFB8
:10A55000DCF80030FA2B05D841F26002C2F20002AA
:10A56000D05C70474FF00000704700BFDCF800304F
:10A5700003F10103CCF80030DCF8140090F851200E
:10A5800002F1010280F85120704700BF70B4044608
:10A590000846A1B199188C4211D22518AA420ED2B0
:10A5A00094423ABFC4EB0206F6B20026A94205D295
:10A5B0000019821AD31AF118C8B200E0304670BCF4
:10A5C000704700BFF0B583B043F2BC03C2F2000392
:10A5D0004FF00C021A7043F26000C2F200000468EF
:10A5E0003CB3154643F2BC07C2F200074FF0000629
:10A5F00021680B6873B10DF107000DF10601984752
:10A600009DF807009DF8061032463B78FFF7BEFF25
:10A610004519EDB26468002CEAD143F2BC02C2F2E3
:10A6200000021078A84204D243F2BC01C2F2000139
:10A630000D7043F2BC03C2F200034FF00A025A70DD
:10A6400043F2D404C2F2000424683CB3154643F23A
:10A65000BC07C2F200074FF000062068036873B120
:10A660000DF107000DF1060198479DF807009DF8D0
:10A67000061032467B78FFF789FF4519EDB2646812
:10A68000002CEAD143F2BC01C2F200014A78AA428E
:10A6900004D243F2BC00C2F20000457043F2BC0396
:10A6A000C2F200034FF00201997043F2B404C2F207
:10A6B000000424683CB30D4643F2BC07C2F2000715
:10A6C0004FF000062268136873B10DF107000DF119
:10A6D000060198479DF807009DF806103246BB78A2
:10A6E000FFF754FF4519EDB26468002CEAD143F23C
:10A6F000BC00C2F200008178A94204D243F2BC023D
:10A70000C2F20002957043F2BC03C2F200034FF0A4
:10A710000100D87043F21824C2F2000424683CB34C
:10A72000054643F2BC07C2F200074FF0000621685D
:10A730000A6872B10DF107000DF1060190479DF80E
:10A7400007009DF806103246FB78FFF71FFF4519FA
:10A75000EDB26468002CEAD143F2BC03C2F20003FC
:10A76000D878A84204D243F2BC01C2F20001CD70F5
:10A7700003B0F0BD43F21023C2F20003196840F2A7
:10A780000000C0F60200401A704700BF034610B137
:10A7900082688A4218D043F2B803C2F200031868F4
:10A7A00060B182688A4203D10BE083688B420AD091
:10A7B00040680028F9D14FF0000305E04FF0000396
:10A7C00002E0034600E003461846704710B540F229
:10A7D000A064C1F200044FF4117303FB0044D4F8E9
:10A7E0000811B1F1FF3F03D0D4F8042191420DD1FB
:10A7F00023689A6A4FF0FF019047002834D0D4F8BC
:10A80000080100F10100C4F8080110BD91422BD8E5
:10A810006318197943F2A802C2F2000213787BB9D7
:10A82000FD290FD923689A6A4FF0FE019047D8B1ED
:10A8300043F2A800C2F200004FF00101017010BD08
:10A840006FEA01012268936AC9B2984760B1D4F8EF
:10A85000080100F10100C4F8080143F2A801C2F2A6
:10A8600000014FF000020A7010BD00BF70B506462F
:10A8700040F2A065C1F200054FF4117404FB00F42E
:10A880002B194FF00101C3F80C112A59936998470D
:10A890002859016A3046884770BD00BF38B540F27C
:10A8A000A061C1F200014FF4117202FB00F28C189A
:10A8B000D4F80831D4F80451AB420DD08958E318CC
:10A8C0008A6A1979904738B1D4F80801FF2814BF73
:10A8D00001300020C4F8080138BD00BF38B540F28F
:10A8E000A064C1F200044FF4117202FB00F2A3183D
:10A8F000D3F80451D3F808118D4206D14FF000016E
:10A90000C3F80C11A2589369984738BD10B440F2AF
:10A91000A063C1F200034FF4117202FB003000F596
:10A920008870D0F80031FF2B14BF5A1C0022D0F8D9
:10A930000441A2421CBFC154C0F8002110BC7047A2
:10A94000F8B543F21024C2F2000424688568C76891
:10A95000466807FB05604518611911D2CE180B48EF
:10A96000864210D8012B04D1635D13704FF00000B4
:10A97000F8BD10461A460FF01BFB4FF00000F8BD63
:10A980004FF01F00F8BD4FF01F00F8BD0100020896
:10A9900010B543F2AA03C2F200031A8840F2A06085
:10A9A000C1F200004FF4117404FB0204F5F79CFFA0
:10A9B0004FF0FF31C4F810124FF00003C4F8183202
:10A9C00004F58874F5F79AFF10BD00BFF8B5064688
:10A9D0004FF00203037044F20000C0F60000C28B87
:10A9E0004FF6FF718A4221D03F4C404BA34222D206
:10A9F00003F110033E4DEF1A4FEA17124FF6FF75A1
:10AA000002F1010002F001071C46D98BA9424FD187
:10AA100015E01C46D98BA94211D002F1010203F1C5
:10AA200010031C46D98BA94257D108E044F2000418
:10AA3000C0F6000403E044F20004C0F600044FF640
:10AA4000FF7021464FF00D02FFF752FA4FF6FF73E9
:10AA5000984208BF0020E28982421BD0A4F1100571
:10AA600044F20000C0F6000085421AD34FF6FF7092
:10AA700029464FF00D02FFF73BFA4FF6FF7188426F
:10AA800008BF002034F8024C84420AD12C464FF013
:10AA9000010201E04FF00002607BFF2806D1327016
:10AAA00004E04FF0020333704FF000042046F8BD7D
:10AAB0004FF0000202F1010203F110038242BED006
:10AAC000002FA6D01C46D98BA942B8D002F10102B2
:10AAD00003F1100382429CD1B1E702F1010203F1BC
:10AAE0001003824295D1AAE70080000800400008C8
:10AAF0000F80000870B5C0B005460E4620F0FF0478
:10AB0000684621464FF04002F8F782FB00AB53FA4B
:10AB100085F031464FF010020FF04AFA68462146A0
:10AB20004FF48072F8F7C8FC40B070BD38B50546E8
:10AB300040F2A064C1F200044FF4117303FB00441F
:10AB4000D4F81C02FDF718FB43F2AA00C2F2000081
:10AB50000188A94206D143F2AA03C2F200034FF6CC
:10AB6000FF721A804FF00000C4F81C0238BD00BF0D
:10AB700010B54FF00000FAF77FFF43F26003C2F216
:10AB800000031C6834B12068016901B1884764681A
:10AB9000002CF8D110BD00BF10B50446072827D8F7
:10ABA000032894BF4FF4FA73322303FB01F140F200
:10ABB000A063C1F2000303EBC000C0F8141969B12F
:10ABC000FDF7BCFE002808BF012040F2A063C1F2DF
:10ABD000000303EBC404C4F8100910BD40F2A061E7
:10ABE000C1F2000101EBC4044FF00002C4F81029C7
:10ABF00010BD00BF38B50446072851D840F2A06305
:10AC0000C1F2000303EBC000D0F8145935B340F291
:10AC1000A061C1F2000101EBC402D2F81039EBB11E
:10AC2000FDF78CFE002808BF012040F2A061C1F2B0
:10AC3000000101EBC402D2F81039C01A85420CD2CF
:10AC400040F2A065C1F2000505EBC4014FF000051C
:10AC5000C1F81459C1F8105900E02D1A05F1040586
:10AC60004CF6CD42CCF6CC42A2FB05234FEA930032
:10AC7000032C0AD800F1630348F21F51C5F2EB110F
:10AC8000A1FB03324FEA521038BD00F109014CF626
:10AC9000CD42CCF6CC42A2FB01304FEAD00038BD09
:10ACA0004FF0000038BD00BF70B506466446DCF8C2
:10ACB00014305D6AFDF742FE6169CA6A0AB9C8626A
:10ACC00008E0801A05EB850506FB05F6B04224BFB7
:10ACD0000020C8626369D96AD1F1010038BF002041
:10ACE00070BD00BF10B540F2A063C1F200034FF485
:10ACF000117404FB003303F58873D3F80841002C6A
:10AD00005FD15AB14FF0FF31C3F8001143F21C2359
:10AD1000C2F200034FF00000187010BDD3F80021FC
:10AD2000B2F1FF3F06D1FF294BD14FF00002C3F82B
:10AD3000002110BDFF291ED143F21C21C2F20001E7
:10AD40004FF000040C70012A10D94FF00102C3F833
:10AD5000082140F2A063C1F200034FF4117101FB1E
:10AD60000030D0F81C02FCF7C5FF10BD4FF000000A
:10AD7000C3F8000110BDFE2907D143F21C23C2F223
:10AD800000034FF00101197010BD43F21C20C2F204
:10AD90000000007848B16FEA0101C9B243F21C20FB
:10ADA000C2F200004FF000040470FF2A05D8995445
:10ADB00002F10102C3F8002110BD4FF0FF32C3F8C9
:10ADC000002110BD08B540F2A063C1F200034FF4AA
:10ADD000117202FB0030D0F80811D0F8043100F1F4
:10ADE000040099420AD94FF00002C0F8002143F252
:10ADF000EC00C2F200004068FCF77CFF08BD00BF19
:10AE0000F8B5654643F2E803C2F200031A7802F08F
:10AE10000804E7B227B1DCF8146096F8516007E047
:10AE200012F0110F06BFDCF8147097F8526000267C
:10AE300001EB800411F8203003F0070302F0200238
:10AE4000D7B23FB111F8202002F00807FAB20AB1D8
:10AE50004FEA430311F820704FEA9712012A08D0F5
:10AE6000022A10D111F82000C0F3011101FB06677E
:10AE70000BE06F6997F8517011F82020C2F30110B0
:10AE800000FB077701E04FF00007042B50D8DFE804
:10AE900013F0C60140003B002200050043F21421DC
:10AEA000C2F200010B6840F20007C0F60107FA1871
:10AEB00092F802E0D0784FEA006040EA0E40527803
:10AEC00040EA0220FF5C03F104030B603843FFF704
:10AED0009FF868602CE043F21422C2F2000213686B
:10AEE00040F20000C0F60100C11891F801C0C05C3A
:10AEF0004FEA004040EA0C208978084303F103033D
:10AF000013603F186F6013E0FFF736FAC2196A60EA
:10AF10000EE043F21423C2F20003186840F200016D
:10AF2000C0F601010A5CBF186F6000F101001860F3
:10AF3000637803F0070343F2E800C2F200000178EF
:10AF400001F02002D7B237B1607800F00801CAB230
:10AF50000AB14FEA430367784FEA9710012807D0F8
:10AF600002280ED16178C1F3011202FB06670AE0E4
:10AF70006F6997F851006178C1F3011202FB000775
:10AF800001E04FF00007042B50D8DFE813F0480130
:10AF900040003B002200050043F21421C2F20001F0
:10AFA0000B6840F20007C0F60107FA1892F802E0B9
:10AFB000D0784FEA006040EA0E40527840EA022022
:10AFC000FF5C03F104030B603843FFF721F8A8602E
:10AFD0002CE043F21422C2F20002136840F2000097
:10AFE000C0F60100C11891F801C0C05C4FEA0040F2
:10AFF00040EA0C208978084303F1030313603F18EB
:10B00000AF6013E0FFF7B8F9C219AA600EE043F28F
:10B010001423C2F20003186840F20001C0F60101D7
:10B020000A5CBF18AF6000F101001860A37803F05C
:10B03000070343F2E800C2F20000017801F02002A9
:10B04000D7B237B1A07800F00801CAB20AB14FEA0E
:10B050004303A7784FEA9710012807D002280ED1A2
:10B06000A178C1F3011202FB06670AE06F6997F845
:10B070005100A178C1F3011202FB000701E04FF07B
:10B080000007042B50D8DFE813F0CA0040003B0053
:10B090002200050043F21421C2F200010B6840F2C5
:10B0A0000007C0F60107FA1892F802E0D0784FEADC
:10B0B000006040EA0E40527840EA0220FA5C03F158
:10B0C00004030B601043FEF7A3FFE8602CE043F29B
:10B0D0001422C2F20002136840F20000C0F6010020
:10B0E000C11891F801C0C05C4FEA004040EA0C2052
:10B0F0008978084303F1030313603F18EF6013E0FE
:10B10000FFF73AF9C219EA600EE043F21423C2F2E3
:10B110000003186840F20001C0F601010A5CBF1884
:10B12000EF6000F101001860E37803F0070343F2D9
:10B13000E800C2F20000017801F02002D0B230B184
:10B14000E17801F00802D0B208B14FEA4303E17898
:10B150004FEA9112012A02D0022A0FD108E06E694B
:10B1600096F85100E278C2F3011101FB000607E0F6
:10B17000E078C0F3011101FB066601E04FF0000624
:10B18000042B4CD8DFE803F04B031318300043F2D4
:10B190001423C2F20003186840F20001C0F6010156
:10B1A0000A5CB6182E6100F101001860F8BDFFF7C7
:10B1B000E3F882192A61F8BD43F21422C2F20002B8
:10B1C000136840F20000C0F60100C1184C78C05C62
:10B1D0004FEA004040EA04208978084303F1030362
:10B1E000136036182E61F8BD43F21421C2F200013B
:10B1F0000B6840F20004C0F60104E2189678D0789B
:10B200004FEA006040EA0640527840EA0220E25CE1
:10B2100003F104030B601043FEF7FAFE2861F8BD4A
:10B2200010B58AB0044601A8F6F788FD039B237089
:10B23000029860700199A170079A1AB102F1FF306B
:10B24000C3B201E04FF00603E3704FF0010101FAD1
:10B2500003F222710AB010BD70B582B00546124CDF
:10B2600004EB80066846FFF7DBFF9DF8002014F82A
:10B2700025309A4212D19DF80100717888420DD193
:10B28000B2789DF804301A4208D0F078D0F101006D
:10B2900038BF00204FF00101F17002E04FF00000D4
:10B2A000F07002B070BD00BFF00F001008B50328A9
:10B2B0001ED8DFE800F0020910174EF64C10C0F659
:10B2C000030010F065FC08BD4EF65010C0F60300F8
:10B2D00010F05EFC08BD4EF66410C0F6030010F0DE
:10B2E00057FC08BD4EF67C10C0F6030010F050FC71
:10B2F00008BD00BF2DE9F8430546884616461F469F
:10B3000043F2AA03C2F20003B3F8009043F2545090
:10B31000C2F20000016843F2A402C2F20002136804
:10B32000994201D0FFF734FB072D6ED81F2E6CD841
:10B3300040F2A064C1F200044FF4117000FB094414
:10B3400043F2EC00C2F200004FF00001FCF722FAD9
:10B35000217965F34711072D14BF00250125AA198E
:10B3600062F304012171CBB22DB184F8058043440E
:10B370004FF0020001E04FF0010006F1FF3E5FFADE
:10B380008EFE46B302463F1A0EF0010C3D5C04F1FE
:10B39000040635545B1902F101020EF1FF31C9B206
:10B3A000FF2934D114E0BD5C04F10406B5545B19E7
:10B3B00002F1010201F1FF3101F0FF01BD5CB55462
:10B3C0005B1902F1010201F1FF31C9B2FF29EAD193
:10B3D00000F1010070442218137100F10100C4F85B
:10B3E00004014FF0FF33C4F8083121680B6A43F2BF
:10B3F000AA00C2F2000000789847FCF749FC43F22B
:10B40000EC00C2F20000FCF7D3FABDE8F8834FFA73
:10B410008CF5002DC7D0BD5C04F10406B5545B1952
:10B4200002F1010201F1FF31C9B2FF29BBD1CFE71F
:10B4300010B586B00DF10700FFF7C8FA044618B141
:10B440009DF8073023B90FE044F20004C0F6000471
:10B45000E2894FF6FF7082422BD048F20001C0F61D
:10B4600000018C4209D32AE0304821464FF00D02FA
:10B470000EF048F9002848D0EAE74FF6FF7248F28C
:10B480000000C0F600006FEA0403C118C1F3001108
:10B4900004F11004E389934239D10AE004F1100366
:10B4A0001C46D989914204D003F11004E3899342E8
:10B4B00039D148F20002C0F60002944207D344F2A8
:10B4C0000004C0F6000420462146F7F789FF02A8D1
:10B4D00016494FF00D020EF06BFD4FF0FF008DF896
:10B4E00015004FF6FF7002A94FF00D02FEF700FDA8
:10B4F0004FF6FF71884212BFADF816000021ADF87B
:10B500001610204602A9FFF7F5FA06B010BD8442D6
:10B51000D5D20029C2D004F11004E1899142C8D0EB
:10B520008442BBD3CBE78442B8D3C8E7661000207F
:10B530002DE9F04F85B0884691461D46E2464FF012
:10B54000000426464FF0020B2DE007462846C04770
:10B55000034670B324B9202822D0092802D11FE065
:10B56000012C05D12B2B0DD02D2B0DD05C4601E0ED
:10B57000022C01D12E2B09D0A3F13002D0B2092820
:10B5800017D805E05C4603E05C4601E04FF0030499
:10B590000E2E05D804A98A1902F8103C06F10106FE
:10B5A0002846C8473846FF28CFD000F1FF3700288B
:10B5B000CCD1012C12D98EB104ACA6194FF00004E5
:10B5C00006F8104C684621460EF0F6F8DAF814102A
:10B5D000C864DAF8142082F8504005E0DAF8143034
:10B5E0004FF0010083F8500005B0BDE8F08F00BFB8
:10B5F00010B5044643F26400C2F20000FCF7D8F92B
:10B60000F6F772FEFAF7DEFA08B1FBF701FF204603
:10B61000FCF706FD43F26400C2F200004FF00001A7
:10B62000FCF7B8F810BD00BF10B586B040F20000BE
:10B63000C0F601003449F7F7D3FE00284BD1334B55
:10B64000334A9A421DD240F20001C0F601010B6854
:10B65000B3F1FF3F42D102F104032E4AD01A20F089
:10B660000302991812F0040F3FD118468B420CD0F8
:10B6700003F104021B68B3F1FF3F3ED04FF000001E
:10B6800031E040F20000C0F6010040F20003C0F6D5
:10B690000203984225D10DF10700FFF797F9044600
:10B6A000B0B19DF80710022912D002A821464FF030
:10B6B00010020EF07DFC9DF815006FF307008DF869
:10B6C0001500204602A9FFF715FA4FF001000AE025
:10B6D0004FF0010007E04FF0000004E04FF00000E1
:10B6E00001E04FF0000006B010BD184603F104035E
:10B6F0000268B2F1FF3FB8D0C0E702F1040310685E
:10B70000B0F1FF3FB1D0B9E7FFFF01080000020828
:10B7100000000108030002082DE9F0070346002895
:10B720004ED040F20022C0F6000292F8469092F805
:10B73000470043F2BC04C2F2000494F8018092F87E
:10B7400048C0257843F2D802C2F200021468177A82
:10B75000567AD2F804A04FF000021A7083F80190D4
:10B760009870DA704FF0FB0018714FF0060983F8FB
:10B7700005909D7183F807804FF0040883F80880D6
:10B7800083F8098083F80AC0DD721A734FEA142522
:10B790005D739C73DF731E745A744FF01D029A74AC
:10B7A0004FF00202DA744FF0FE021A755A754FEA32
:10B7B0001A229A7583F817A018764FF01F00587652
:10B7C00029B143F2BC03C2F200031A680A60BDE863
:10B7D000F0077047034628B143F2D802C2F20002D4
:10B7E0001068186043F2D801C2F20001087A70476D
:10B7F00070B505460E4614464FF000002946FEF788
:10B80000C5FF08B1F5F71AF843F2B803C2F2000316
:10B810001A686260A56026601C6070BD08B539B109
:10B8200043F26003C2F200031A68426018601EE02F
:10B8300043F26003C2F200031B6883420FD15868D1
:10B8400043F26001C2F20001086010E042685A60F1
:10B8500041605A688242F9D013461BB907E033B100
:10B860004FF000015A688242F0D01346F5E7FEF728
:10B87000A9FE08BD08B539B143F2D403C2F20003F2
:10B880001A68426018601EE043F2D403C2F200035B
:10B890001B6883420FD1586843F2D401C2F2000101
:10B8A000086010E042685A6041605A688242F9D0EC
:10B8B00013461BB907E033B14FF000015A688242CA
:10B8C000F0D01346F5E7FEF77DFE08BD08B539B1A7
:10B8D00043F2B403C2F200031A68426018601EE02B
:10B8E00043F2B403C2F200031B6883420FD15868CD
:10B8F00043F2B401C2F20001086010E042685A60ED
:10B9000041605A688242F9D013461BB907E033B14F
:10B910004FF000015A688242F0D01346F5E7FEF777
:10B9200051FE08BD08B539B143F21823C2F2000335
:10B930001A68426018601EE043F21823C2F2000346
:10B940001B6883420FD1586843F21821C2F20001EC
:10B95000086010E042685A6041605A688242F9D03B
:10B9600013461BB907E033B14FF000015A68824219
:10B97000F0D01346F5E7FEF725FE08BD01604360F1
:10B98000826043F2E403C2F200031A68C2601860E6
:10B99000704700BF70B582B006464FF000038DF8C7
:10B9A00007300D4601B10B7043F26000C2F2000097
:10B9B000046874B121684B6843B130460DF107014A
:10B9C0002A46984710B19DF8070013E06468002CE0
:10B9D000F0D10B2E05DC0C2E03D83046FAF790F888
:10B9E00008E02DB14FF005022A704FF0000001E091
:10B9F0004FF0000002B070BD70B582B006464FF047
:10BA000000038DF807300D4601B10B7043F2600062
:10BA1000C2F20000046874B121688B6843B13046FB
:10BA20000DF107012A46984710B19DF807001BE069
:10BA30006468002CF0D10B2E0DDC0C2E0BD8304698
:10BA4000FAF774F88DF8070010B13046FAF7B4F839
:10BA50009DF8070008E02DB14FF005022A704FF065
:10BA6000000001E04FF0000002B070BD70B582B080
:10BA700006464FF000038DF807300D4601B10B70FC
:10BA800043F26000C2F20000046874B12168CB6820
:10BA900043B130460DF107012A46984710B19DF891
:10BAA000070013E06468002CF0D10B2E05DC0C2E8F
:10BAB00003D83046FAF70AF808E02DB14FF0050236
:10BAC0002A704FF0000001E04FF0000002B070BD9E
:10BAD00070B582B006464FF000038DF807300D4672
:10BAE00001B10B7043F2D400C2F2000004685CB1F3
:10BAF00021688B682BB130460DF107012A46984723
:10BB000058B96468002CF3D1092E0CDC0A2E0AD82F
:10BB10003046F5F7C9FC8DF807009DF807000030A6
:10BB200018BF012008E02DB14FF006022A704FF037
:10BB3000000001E04FF0000002B070BDF0B583B02E
:10BB400005460E464FF000038DF8073043F2D4004F
:10BB5000C2F200000468E4B14FF000072168CA682F
:10BB60001AB1284631469047F0B923689B6833B133
:10BB700028460DF106010DF10702984700E038460E
:10BB80009DF8071099B9646814B10028E6D004E064
:10BB900018B9092D0DDC0A2D0ED82846314607F0BC
:10BBA00059F94FF0000009E04FF0000006E00846A8
:10BBB00004E04FF0060001E04FF0060003B0F0BDD6
:10BBC00070B582B005460E464FF000038DF8073081
:10BBD00012B11946FFF7B2FF43F2D400C2F20000DF
:10BBE00004686CB121684B68284631460DF10702A4
:10BBF000984710B19DF8070012E06468002CF1D15D
:10BC0000092D08DC0A2D09D828463146F5F76EFCC7
:10BC10004FF0000004E04FF0060001E04FF0060096
:10BC200002B070BD08B54FF0000001464FF00102B0
:10BC3000FFF7C6FF08BD00BF70B582B005460E46CF
:10BC40004FF000038DF8073043F2B400C2F2000059
:10BC500004689CB121684B68284669460DF10702CB
:10BC6000984728B10EB1009830609DF8070014E0A5
:10BC700064681CB19DF80720002AEBD0012D07D87D
:10BC80004EB12846F6F7B6FD30604FF0000004E0F4
:10BC90004FF00F0001E04FF0000002B070BD00BF98
:10BCA00070B582B005460E464FF000038DF80730A0
:10BCB00043F21820C2F20000046884B121684B6886
:10BCC000284631460DF10702984710B19DF807004C
:10BCD00010E064681CB19DF80720002AEED03DB941
:10BCE0004FF000003146F6F767FC4FF0000001E02E
:10BCF0004FF00E0002B070BD70B582B005460E4622
:10BD00004FF000038DF8073043F21820C2F2000014
:10BD10000468A4B121688B685BB1284669460DF1BF
:10BD20000702984728B10EB1009830609DF80700CF
:10BD300014E064681CB19DF80720002AEAD045B9D8
:10BD400056B14FF00000F6F779FD30604FF000007B
:10BD500004E04FF0060001E04FF0000002B070BDBB
:10BD60002DE9F04F2DED048B8BB00746154691421F
:10BD700059D289464FF0000B4FF000089FED908B91
:10BD80009FED919B6FEA0106B01800F00106CDF817
:10BD900004B0022F4CD150E0CDF804B0022F05D1F1
:10BDA0005FFA89F001A9FFF7A7FF04E05FFA89F0C5
:10BDB00001A9FFF741FF04EB44060AA88119A1F18C
:10BDC000200601F8209C01F81F8C01980CF008FA5D
:10BDD00053EC182B0CF0A2FB53EC192B0CF05AFA75
:10BDE0000CF0C4F983B2FF2B28BFFF23B37004F11A
:10BDF00001040A2C04D005F1FF324A450AD14CB1A6
:10BE000004EB44044FF007003946E2B202ABFFF7FF
:10BE100071FA444609F101094E46CDF804B0022FEB
:10BE200040F089808DE00BB0BDEC048BBDE8F08F55
:10BE3000C8B201A9FFF700FF03E0C8B201A9FFF7EC
:10BE40005BFF0AAC04F8209D84F8018001980CF097
:10BE5000C7F953EC182B0CF061FB53EC192B0CF0C9
:10BE600019FA0CF083F981B2FF2934BF0B46FF2386
:10BE7000A3704FF0000404F1010405F1FF324A45BC
:10BE80000DD10AE004EB44044FF007003946E2B25A
:10BE900002ABFFF72FFA444601E0002CF2D109F182
:10BEA00001094D45BFD9002E3FF476AFCDF804B05F
:10BEB000022F05D05FFA89F001A9FFF7BDFE04E06B
:10BEC0005FFA89F001A9FFF717FF04EB44060AA8FF
:10BED000861906F8209D86F8018001980CF080F9FB
:10BEE00053EC182B0CF01AFB53EC192B0CF0D2F975
:10BEF0000CF03CF981B2FF2934BF0B46FF23B3702D
:10BF000004F101040A2C0AD104EB44044FF00700A9
:10BF10003946E2B202ABFFF7EDF9444605E005F120
:10BF2000FF324A4501D1002CEED109F101094D45FE
:10BF30003FF632AF77E75FFA89F001A9FFF77CFEA1
:10BF400004E05FFA89F001A9FFF7D6FE04EB440094
:10BF50000AA90B18A3F1200A03F8206C03F81F8C20
:10BF600001980CF03DF953EC182B0CF0D7FA53EC78
:10BF7000192B0CF08FF90CF0F9F882B2FF2A28BFC8
:10BF8000FF228AF8022004F101040A2C0AD104EBF2
:10BF900044044FF007003946E2B202ABFFF7AAF9BA
:10BFA000444605E005F1FF30B04201D1002CEED14E
:10BFB00009F101094D453FF6EFAE34E7AFF30080DC
:10BFC0000000000000E06F40000000000000E03FC3
:10BFD0002DE9F04F9FB040F6C410FCF721F84FF068
:10BFE00002004FF0000143F2BC03C2F20003DA7812
:10BFF000FFF7B6FE4FF0010002904FF0000BDA465B
:10C00000D94607464CF6CD41CCF6CC4103914FF0D2
:10C010007D00FCF705F88DF83790C8464E464C4633
:10C0200013E045F0800504F10804E4B216A9725C3F
:10C03000AA4202D016ABF554B84606F101069DF8A7
:10C040003750002D50D1202E4ED020460DF1370113
:10C05000FFF7A0FC051C18BF012504F10102D0B2B6
:10C060000DF13701FFF796FC10B145F00205EDB276
:10C0700004F10203D8B20DF13701FFF78BFC08B1D0
:10C0800045F0040504F10300C0B20DF13701FFF7DC
:10C0900081FC08B145F0080504F10401C8B20DF1B6
:10C0A0003701FFF777FC08B145F0100504F10502F0
:10C0B000D0B20DF13701FFF76DFC08B145F0200556
:10C0C00004F10603D8B20DF13701FFF763FC08B1A4
:10C0D00045F0400504F10700C0B20DF13701FFF74C
:10C0E00059FC00289DD19EE7B8F1000F02D1BAF1AA
:10C0F000000F0CD14FF002004946F2B216ABFFF729
:10C10000F9F84FF03200FBF78BFF019701E0CDF813
:10C1100004908DF83790C8464E464C4613E045F0E3
:10C12000800504F10804E4B20EA8315CA94202D0F3
:10C130000EAAB554B84606F101069DF83750002DF9
:10C1400050D1202E4ED020460DF13701FFF7C0FC14
:10C15000051C18BF012504F10100C0B20DF1370123
:10C16000FFF7B6FC10B145F00201CDB204F10202B6
:10C17000D0B20DF13701FFF7ABFC08B145F0040573
:10C1800004F10303D8B20DF13701FFF7A1FC08B1A8
:10C1900045F0080504F10400C0B20DF13701FFF7C6
:10C1A00097FC08B145F0100504F10501C8B20DF186
:10C1B0003701FFF78DFC08B145F0200504F10602B8
:10C1C000D0B20DF13701FFF783FC08B145F040050F
:10C1D00004F10703D8B20DF13701FFF779FC00280D
:10C1E0009DD19EE7B8F1000F02D1BAF1010F0AD13B
:10C1F00048464946F2B20EABFFF77CF84FF03200EA
:10C20000FBF70EFF019743F2BC03C2F200039A78DA
:10C21000B2B1039EA6FB0A044FEA141000EB8001A2
:10C22000BAEB810F0CD138464946FFF799FD4FF024
:10C230003200FBF7F5FEBBF1000F40F0B88003E0E1
:10C24000BBF1000F40F09C8005A849464FF020024A
:10C250000DF0D2FE43F2BC06C2F20006B478ACB3D5
:10C260004D466FEA0900011901F0010209F00703C8
:10C2700007FA03F69DF8140046EA00018DF8141041
:10C2800005F10105A542C0F2B3801FE01EAB03EB30
:10C29000D50605F0070007FA00F216F8641C42EA1A
:10C2A000010306F8643C05F101051EA800EBD50268
:10C2B00005F0070107FA01F312F8646C43EA06007F
:10C2C00002F8640C05F10105A542DFDB4FF0070021
:10C2D0004FF011014FF01E0205ABFFF70BF84FF0C6
:10C2E0003200FBF79DFE05A849464FF020020DF0F5
:10C2F00083FE43F2BC04C2F20004E578A5B34B46CA
:10C300006FEA0902511901F0010609F0070007FA66
:10C3100000F49DF8142044EA02018DF8141003F192
:10C3200001039D4250DC1FE01EAC04EBD30203F07E
:10C33000070007FA00F612F8641C46EA010402F846
:10C34000644C03F101031EAA02EBD30403F00700BF
:10C3500007FA00F614F8641C46EA010204F8642C9B
:10C3600003F101039D42DFDC4FF007004FF01201A3
:10C370004FF01E0205ABFEF7BDFF4FF0060B16E0B7
:10C38000019AA2B9BBF1020F11D1029D7DB943F20E
:10C39000BC03C2F20003DA784AB14FF0020049460A
:10C3A000FFF7DEFC4FF03200FBF73AFE0297BAF1DE
:10C3B000000F06D10BF1FF3BCDF808904FF0280A93
:10C3C00025E60AF1FF3A22E6002EADD01EAE06EBBE
:10C3D000D30403F0070007FA00F214F8641C42EAE1
:10C3E000010604F8646C03F101039D429CDCBBE789
:10C3F000002A3FF44BAF1EAA02EBD50305F0070657
:10C4000007FA06F013F8641C40EA010203F8642CF2
:10C4100005F10105A542FFF639AF57E72DE9F04FC9
:10C420002DED028B87B008EE100A0C461746994690
:10C43000129E1399B5EEC08AF1EE10FA54BF002592
:10C440000125A84604F1FF33D8B2082807D8092AE5
:10C4500005D8A24601F1FF32944205D808E001F167
:10C46000FF339C4240F2CD8001F1FF34E4B2C8E0DA
:10C4700018EE100A0CF0A4FA48B930464FF03F010C
:10C4800022460DF0B9FD4FF000013155C4E018EE21
:10C49000100A0CF099FF06EE900AF2EE047AF4EE20
:10C4A000E76AF1EE10FA0DDB4FF00100B0EE677AAB
:10C4B00000F1010067EE877AF4EEE76AF1EE10FA18
:10C4C000F6DA03E04FF00100F2EE047A2146431958
:10C4D000A34200F39680C0EB040EC5EB0E0202F1FE
:10C4E000FF3E4DF2D87AC0F6030ADFED9C4AF6EE25
:10C4F000003AB2EE044AC0EB040CC5EB0C0303F0A7
:10C50000010BBEF1000F00F38F808AE0BEF1000F37
:10C5100004DDBE45B4BF72463A4601E04FF000026A
:10C520005AF8223003EE103AB8EE430A20EE027AAF
:10C53000B4EEE47AF1EE10FA48BF37EE237ABDEE9E
:10C54000C73A13EE10CABCFBF3FB06EE10BAB8EE06
:10C55000C65AB4EEE75AF1EE10FA0DDB00F1010C09
:10C5600087EE006A67EE847A0EF1FF3E6046BEF108
:10C57000000200F3C380BEE013EE105AB5FBF3F4E3
:10C5800003FB14542CB916EE107A002F08BF4FF09D
:10C590000008B9F1000F07D0C8EB0103181A002AF0
:10C5A00018BF0138831A01E04FF0000301F10101C7
:10C5B000B8F1000F04D04EF6A017C0F6030703E051
:10C5C0004BF61857C0F6030722B14EF6A410C0F67A
:10C5D000030003E04BF61850C0F603004EF6B81502
:10C5E000C0F60305009501978DED026A0390049251
:10C5F000059430464EF6A812C0F603020DF0C6F8B8
:10C600000AE03046002D0CBF2B212D2122460DF0D3
:10C61000F3FC4FF00000305507B0BDEC028BBDE8D5
:10C62000F08F4FF0000203E0BE45B4BF72463A46B9
:10C630005AF8223000EE103AB8EE405A65EE260A5B
:10C64000F4EEE40AF1EE10FA48BF70EEA30ABDEE74
:10C65000E03A13EE10CABCFBF3FC06EE10CAF8EE8B
:10C66000C65AF4EEE75AF1EE10FA85DB00F101004C
:10C6700080EE852A67EE847A0EF1FF3E42199142E0
:10C68000BFDBBBF1000F3FF441AFBEF1000F02DC96
:10C690004FF0000203E0BE45B4BF72463A465AF876
:10C6A000223001EE103AF8EE411A21EE822AB4EE61
:10C6B000E42AF1EE10FA48BF32EE232ABDEEC23A68
:10C6C00013EE10BABBFBF3FB06EE10BAF8EEC62A67
:10C6D000F4EEE72AF1EE10FAFFF64EAF00F101009A
:10C6E00082EE212A67EE847A0EF1FF3E43199942C9
:10C6F000BFF60CAF85E74FF0000202E0BA42A8BFD8
:10C700003A465AF8223006EE903AF8EE660A20EEE3
:10C71000861AB4EEE41AF1EE10FA48BF31EE231A8D
:10C72000BDEEC13A13EE10BABBFBF3FB06EE10BA36
:10C73000F8EEC65AF4EEE75AF1EE10FAFFF61CAF27
:10C740000CF1010081EE202A67EE847A0EF1FF3EA3
:10C7500042199142BFF6DAAE53E700BF0000004B2A
:10C76000F8B505460F46F4F7BFF8064640F2A0625A
:10C77000C1F200024FF4117303FB05F014181158B5
:10C7800011B18A682846904784F820724FF000055E
:10C79000C4F81052C4F81452C4F80451C4F8085133
:10C7A0003046F4F7ABF804F5097029464FF008025B
:10C7B000F4F754F8F8BD00BF70B588B0054640F2F4
:10C7C000A064C1F200044FF4117303FB004494F819
:10C7D000200200284AD043F2AA01C2F200010A88CE
:10C7E0004FF6FF76B24204D0D0B24FF00401FFF70B
:10C7F000B7FF28464FF00001FFF7B2FF43F2AA0649
:10C80000C2F2000635804EF6C410C0F603004FF0A9
:10C81000070142F26122C0F60302FBF7C3FBC4F832
:10C820001C02246830784FF0010300934FF000029F
:10C8300001924AF2CD71C0F6020102914AF6C55347
:10C84000C0F6020303934AF6E541C0F602010491E3
:10C850004AF62D33C0F602030593069264684FF43E
:10C8600016514FF00803A047FEF792F808B070BDCC
:10C87000704700BF08B5B0F1FF3F04D040B9024691
:10C88000F6F70AF808BD4FF000000246F6F704F884
:10C8900008BD00BF38B506F0D1FA43F2C003C2F2BA
:10C8A00000034FF001021A704FF000042546E0B279
:10C8B00029462A46FFF784F940B904F10104E0B2A1
:10C8C00029462A46FFF77CF9002867D04FF0FF3051
:10C8D0004FF00001FFF7CEFF4FF000004FF00001D6
:10C8E000FFF7DEF943F21821C2F200010C6834B1FF
:10C8F0002368DA6802B190476468002CF8D143F2EB
:10C90000B800C2F2000004683CB121680B680BB1AA
:10C91000A06898476468002CF7D1F9F719FEFEF774
:10C9200027F940F2A062C1F2000292F82002042826
:10C9300006D028B14FF000004FF00401FFF710FFC0
:10C9400040F2A061C1F2000191F86434042B06D0DA
:10C950002BB14FF001004FF00401FFF701FF40F24F
:10C96000A062C1F2000292F8A806042806D028B1FD
:10C970004FF002004FF00401FFF7F2FE40F2A06119
:10C98000C1F2000191F8EC38042B06D02BB14FF026
:10C9900003004FF00401FFF7E3FE38BD04F101048A
:10C9A000B4F5807F83D191E738B5054643F2A404FE
:10C9B000C2F200042068FBF7DFFB4FF000032360A6
:10C9C0008DB14EF6D410C0F603004FF007014CF6BF
:10C9D000E122C0F60202FBF7E5FA43F2AC01C2F233
:10C9E0000001086038BD43F2AC04C2F200042068C4
:10C9F000FBF7C2FB4FF000002060FAF755FAFFF793
:10CA000049FF0AF05FFD43F2AA01C2F200010A8861
:10CA10004FF6FF739A4204D0D0B24FF00401FFF7F3
:10CA20009FFE38BD70B543F2EC00C2F200004EF636
:10CA3000E411C0F60301FAF795FE43F2AA03C2F22D
:10CA400000034FF6FF721A8040F2A064C1F20004A6
:10CA50004FF0040684F820624FF00005C4F81C5221
:10CA60002846FBF7B9F8206084F86464C4F8605481
:10CA70004FF00100FBF7B0F8C4F8440284F8A86650
:10CA8000C4F8A4564FF00200FBF7A6F8C4F88804D7
:10CA900084F8EC68C4F8E8584FF00300FBF79CF802
:10CAA000C4F8CC0643F26400C2F200004EF6F01166
:10CAB000C0F60301FAF756FE43F2C400C2F20000CA
:10CAC0004EF27051C0F603012A462B46FEF756FF80
:10CAD000FDF778FD4FF00100FFF766FF70BD00BF66
:10CAE0002DE9F04F2DED048BABB01CAF26AC4DF211
:10CAF000B475C0F6030595E80F0084E80F00A76041
:10CB00004AF25153C0F60203E36020462AA9F7F720
:10CB1000C3FA22AE95E80F0086E80F00B7604AF22C
:10CB20006D50C0F60200F06030462146F7F7B4FAC7
:10CB30004FF000041B9443F26400C2F2000021464F
:10CB4000FAF728FE43F2D801C2F200010C72FFF797
:10CB5000A1FE0AF0B7FC4FF00200FFF72DFE43F2F2
:10CB60001422C2F2000215680DBB0FF001F8F0B9F3
:10CB7000F5F77AF810F0C20F19D14FF00300FEF765
:10CB800095FB4FF47A754FF032063046FBF748FAC2
:10CB9000F5F7AAFB05F1FF343046FBF741FAF5F74C
:10CBA000A3FB651EF1D14FF00000FEF77FFB43F2BF
:10CBB000E803C2F200034FF000041C604FF00100D4
:10CBC000187040F2A066C1F2000606F51965284605
:10CBD000214642F654220DF00FFA41F26000C2F2F3
:10CBE000000021464FF400520DF006FA06F51160E0
:10CBF00021464FF040020DF0FFF943F21410C2F24B
:10CC0000000021464FF0FC020DF0F6F921954FF09F
:10CC10000A01C6F8B41920462946FDF735FC43F24F
:10CC20009C02C2F20002146043F2B003C2F200039D
:10CC30001C6043F21425C2F200054FF030042C6052
:10CC400040F20004C0F6010494F82F0000F1010046
:10CC500094F82E1000EB0122101943F21023C2F2B7
:10CC600000031860FBF76AFE0A902B68E15CFF295D
:10CC700030D143F2D800C2F200004FF0010101723E
:10CC80000360219A106A18B100F1010052F82030B7
:10CC900043F2D801C2F200014B604FF0FF024A722A
:10CCA00043F2AC00C2F200004FF00003036043F215
:10CCB000AA01C2F20001088840F2A062C1F200029B
:10CCC0004FF4117303FB0021D1F81C02FBF712F89B
:10CCD00005F08DBA06F090F84FF000070997BA46B4
:10CCE0003C4601E04FF000042CB94FF00000FEF785
:10CCF0007FFC4FF0640404F1FF3443F2E806C2F213
:10CD00000006357805F0E7026FF34512327043F202
:10CD10001420C2F200000368089343F21426C2F202
:10CD2000000640F20007C0F6010743F2E808C2F22D
:10CD300000084DF69C29C0F6030931687D5C01F1BD
:10CD40000101316098F8002012F0010F0ED10AF1B4
:10CD5000010A40F2FF30824508D943F2D803C2F2FB
:10CD600000034FF03601197205F0F9B90DF1700C9E
:10CD700028464946FEF744F84EF22C13C0F603034A
:10CD800053F825004DF69C6BC0F6030B40F00101F3
:10CD9000084730683A5C0B9200F1010030600F2ABE
:10CDA00005F2D5810DF1700C10465946FEF728F8B2
:10CDB0004DF63413C0F603030B9953F82100E5E751
:10CDC00030683A5C0B9200F101003060102A02D901
:10CDD000154605F0BDB90DF1700C0B984EF22C51B3
:10CDE000C0F60301FEF70CF84DF60003C0F603038E
:10CDF0000B9953F82100C9E73268B85C0B9002F137
:10CE0000010232600F2802D9054605F0A1B90DF1E3
:10CE1000700C0B984EF24C71C0F60301FDF7F0FF59
:10CE20004DF6DC73C0F603030B9953F82100ADE710
:10CE300030683A5C0B9200F1010030602F2A02D971
:10CE4000154605F085B90DF1700C0B984EF28C71FA
:10CE5000C0F60301FDF7D4FF4EF28C63C0F6030366
:10CE60000B9953F8210091E730683A5C0B9200F17E
:10CE7000010030603B2A02D9154605F069B90DF171
:10CE8000700C0B984DF67411C0F60301FDF7B8FF56
:10CE90004DF64403C0F603030B9953F8210075E7E0
:10CEA0003268B85C0B9002F1010232603F2802D96F
:10CEB000054605F04DB90DF1700C0B984EF64C017E
:10CEC000C0F60301FDF79CFF4DF6DC63C0F60303DB
:10CED0000B9953F8210059E730683A5C0B9200F146
:10CEE00001003060432A02D9154605F031B90DF131
:10CEF000700C0B984EF21C01C0F60301FDF780FF89
:10CF00004EF27C53C0F603030B9953F821003DE722
:10CF1000219F97F846600DF1700CFDF717FA219DDF
:10CF2000331895F8502002F0010158181C9085F82C
:10CF30004700FF2894BF0020012085F85000D3E669
:10CF4000219F97F846600DF1700CFDF7FFF9351839
:10CF50001C95219B83F84750FF2D94BF0025012588
:10CF600083F85050C0E60DF1700CFDF7EFF930B1C9
:10CF7000219A92F84700011C18BF012101E04FF0EF
:10CF80000001219F87F84710AEE60DF1700CFDF708
:10CF9000DDF9219E96F84750284086F84700A3E621
:10CFA0001D9BA3F1FB031C9319E11D99A1F1FB014A
:10CFB0001C91A1E11D9AA2F1FB021C92D2E11D98E5
:10CFC000A0F1FB001C906EE21D9EA6F1FB061C96D4
:10CFD0004FF002031B9306E21D99A1F1FB011C9186
:10CFE0001E9A1B9230E21D98A0F1FB001C902AE1D2
:10CFF0001D9EA6F1FB061C96ACE21D9BA3F1FB0354
:10D000001C93E8E21D9FA7F1FB071C971E991B913B
:10D0100025E31D9AA2F1FB021C921E981B904FF073
:10D0200000068DF86A60D3E31D9BA3F1FB031C93FC
:10D030001E991B914FF001028DF86A20C8E31D98DC
:10D04000A0F1FB001C9000F060BC1D9DA5F1FB054C
:10D050001C9500F0B5BC9DF874004FF00101FEF77F
:10D060006DFD8DF86B0000283FF43EAE43F2D8040E
:10D07000C2F20004207205F072B81D9E1C964FF09B
:10D0800001038DF86A301E46219991F8472013421A
:10D0900005D09DF870003146FEF750FD68B99DF847
:10D0A0006A304FEA43008DF86A001C9901F10101D2
:10D0B0001C9110F0FE03E7D10CE09DF86A60012E90
:10D0C00008D19DF86B4043F2D802C2F200021472FC
:10D0D00005F045B80DF1700CFDF738F904E69DF840
:10D0E000740005F07BFEFFE50DF1700CFDF72EF9E5
:10D0F0001C9043F21423C2F200031E681C9906EB35
:10D1000041021A60FDF738F91C9001F0DDBE43F2D0
:10D11000E800C2F20000017811F0280F06D01D9B34
:10D12000B3F5005F34BF0023012304E01D9BFA2BFD
:10D1300094BF0023012343B143F2D804C2F2000498
:10D140004FF01301217205F00AB841F26006C2F2F5
:10D1500000061D9AB05C1C90CBE7219B93F85260AF
:10D160001C96C6E7219A92F850001C90C1E74FF038
:10D17000000AB9E50DF1700CFDF7E8F81C90219F4D
:10D1800097F847101B91FDF797F987F84700ABE533
:10D19000219D95F8470095F84610FDF78DF985F823
:10D1A0005000A1E50DF1700CFDF7F8F81E9B41F25F
:10D1B0006006C2F20006F05C1D9920EA0102F254FA
:10D1C00092E543F21410C2F200004FF000014FF05C
:10D1D000FB020CF011FF87E54FF000031C930DF1EB
:10D1E000A80C1CF8386DFDF7B1F80146304608F080
:10D1F0005DFC8DF86B0000283FF476AD43F2D80457
:10D20000C2F20004207204F0AABF07F055F86BE5E3
:10D2100007F05AF88DF86B0000283FF465AD43F233
:10D22000D801C2F20001087204F099BF43F210273E
:10D23000C2F200073D681D98281807F031F853E541
:10D240004FF000021C921C9B40F2A066C1F2000647
:10D250004FF4117101FB036090F82022032A3FD1A3
:10D2600040F2A067C1F2000701FB03F303F58876E3
:10D27000B919FB1803F104034FF00000D1F80021A5
:10D28000FE2A94BF551C0025D1F80471BD4214BF7D
:10D290000025012565F30000BA4214BF00220122D7
:10D2A00062F34100D3F80051FE2D94BF01350025F3
:10D2B0000DF1A80C4CF8385DD3F80461B54214BFE9
:10D2C0000025012565F38200D3F80811D1F101038F
:10D2D00038BF002363F3C300C0B2FDF71FF803E5B6
:10D2E00043F2D804C2F200044FF04803237204F062
:10D2F00036BF4FF000001C901C9E40F2A062C1F2AD
:10D3000000024FF4117101FB062393F82002032859
:10D310001CD140F2A067C1F2000701FB0675D5F8E9
:10D320001022D5F81412531AB3F5807F88BF03F585
:10D3300080731C931C98FF2884BFFF201C900DF164
:10D34000A80C1CF8380DFCF7E9FFCDE443F2D80433
:10D35000C2F200044FF04806267204F000BF4FF0FE
:10D3600000061C961C9B40F2A062C1F200024FF422
:10D37000117101FB032090F82062032E24D140F2AA
:10D38000A067C1F2000701FB037505F58876D6F8A2
:10D390000021D6F80411501AB0F5807F88BF00F53F
:10D3A00080701C900DF1700CFCF7D0FF8DF86A00B6
:10D3B0001C9B984238BF1C90D6F804711C9DEA193A
:10D3C000D1B2C6F804118FE443F2D804C2F20004CB
:10D3D0004FF04803237204F0C2BE4FF000061C96C3
:10D3E0004FF002001B901C9B40F2A062C1F20002B1
:10D3F0004FF4117101FB032696F82002032815D182
:10D4000040F2A067C1F2000701FB03750DF1700C3B
:10D410001B984AF2CD41C0F602014AF2E142C0F641
:10D42000020205F58873FCF7CBFF5DE443F2D804F4
:10D43000C2F200044FF04803237204F090BE4FF094
:10D4400000021C921D991B911C9E40F2A060C1F22B
:10D4500000004FF4117303FB060292F82012032917
:10D4600015D140F2A067C1F2000703FB06750DF16C
:10D47000700C1B984AF2CD41C0F602014AF2E1421B
:10D48000C0F6020205F58873FEF752F82CE443F269
:10D49000D804C2F200044FF04806267204F05FBEC2
:10D4A0004FF000001C901C9B40F2A062C1F20002F1
:10D4B0004FF4117101FB032696F8200203283DD199
:10D4C00040F2A067C1F2000701FB037505F58875FE
:10D4D0000DF1700CFCF73AFF8DF86A00D5F80421C5
:10D4E0001C924FF000011B91D5F800711346974232
:10D4F00007D0AE5C864219D04FF001024FF0000E0B
:10D500000CE04FF0FF001B9010E002F10101EE5C17
:10D51000864202D11C931B9208E00A46FF2B14BFDF
:10D52000013373469F42F0D11C93EAE70DF1700C72
:10D530009DF86C00FCF7F2FEFFF7D6BB43F2D8046F
:10D54000C2F200044FF04803237204F008BE4FF00B
:10D5500000031C931C9E40F2A062C1F200024FF433
:10D56000117101FB062090F82032032B27D140F2E5
:10D57000A065C1F2000501FB065707F58875D7F8CD
:10D580001462D7F81022964212D00DF1700CFCF7FD
:10D59000DDFE8319DFB21C970DF1700CE85DFCF71E
:10D5A000BDFE4FF00005219E86F85050FFF79CBB52
:10D5B0004FF00101219880F85010FFF795BB43F21E
:10D5C000D804C2F200044FF04806267204F0C7BD2A
:10D5D0004FF000021C921C9840F2A063C1F20003BD
:10D5E0004FF4117101FB003696F82022032A28D14E
:10D5F00040F2A067C1F2000701FB007505F58876CF
:10D60000D6F80431D6F800118B4213D00DF1700C0E
:10D61000F05CFCF783FED6F80471FF2F14BF0137CE
:10D620000027C6F804714FF00005219E86F850507F
:10D63000FFF75ABB4FF00102219880F85020FFF706
:10D6400053BB43F2D804C2F200044FF048002072EA
:10D6500004F085BD4FF000031C931D991B9143F20C
:10D660001022C2F20002D2F800801B9F08EB0706CE
:10D6700040F20000C0F60200864208D943F2D80604
:10D68000C2F200064FF01F02327204F068BD1C9B0C
:10D69000032B08D943F2D801C2F200014FF0370042
:10D6A000087204F05CBDF1780D2908D943F2D80462
:10D6B000C2F200044FF03703237204F050BD40F271
:10D6C000A065C1F200054FF4117202FB035090F8FF
:10D6D00020323BB118F8071021B10FE04846FDF7A2
:10D6E00087FF05E04CF24F354FF09609DDF828B082
:10D6F000FBF724F9CBEB0002AA42EFD918F8077028
:10D70000032F3FF6F1AADFE807F002080F169DF895
:10D710007000FFF751F8FFF7E7BA9DF87000314647
:10D7200008F0E6F9FFF7E0BA9DF87000314606F020
:10D730001FFDFFF7D9BA9DF870504DF2C479C0F6BD
:10D74000030996F8028008EB480809EB0807284609
:10D750004FF00301FFF704F84FF4117000FB05F3DD
:10D7600040F2A061C1F20001C85800283FF4BCAAF1
:10D77000F6784DF66422C0F6030252F8261019F826
:10D7800008207B78BF7800974FF0000601964AF694
:10D790009D07C0F6020702974AF6DD07C0F60207AA
:10D7A00003974AF60D17C0F6020704974AF62D377D
:10D7B000C0F602070597069646682846B047FFF769
:10D7C00093BA4FF000031C931D991B918DF86A309A
:10D7D0001C9B40F2A060C1F200004FF4117101FBEC
:10D7E000030696F82022032A79D140F2A065C1F2FF
:10D7F000000501FB035707F5887943F21020C2F2B8
:10D8000000000168219EB26B01EB020B885CFF28CF
:10D810005CD0D8464FF001074FF0000B0894CDF8CC
:10D820002CA0BA4698F8014004EB002343F21020E4
:10D83000C2F200000668F218D9F804111C919DF894
:10D840006A501DB1F75C02F1010200E05F4602F18F
:10D85000FF349DF86A302BB177B9089C5546DDF846
:10D860002CA005E0607838B9089C5546DDF82CA05E
:10D870001C99C9F804112BE01C99D9F800618E425B
:10D8800018D014F8016F19F801501B9A3AB93046B4
:10D890000BF020FFC6B228460BF01CFFC5B2AE420B
:10D8A00008D11C9BFF2B14BF01335B461C9307F16F
:10D8B000FF37CEE70AF1010A18F8020FFF28B1D1AD
:10D8C000089CDDF82CA04FF0000501E04FF00005AA
:10D8D0000DF1700CE8B2FCF721FDFFF705BA43F239
:10D8E000D804C2F200044FF04803237204F037BC9E
:10D8F0004FF000001C901E9E1B964FF001028DF809
:10D900006A2065E74FF000021C921C9E40F2A06363
:10D91000C1F200034FF4117000FB063191F8202290
:10D92000032A31D140F2A065C1F2000500FB065781
:10D9300007F588750DF1700CFCF708FD8DF86A008D
:10D940004FF000031C93D5F80471D5F800118F42F5
:10D9500012D0EA5D82420FD14FF00006FF2F14BFB4
:10D96000013737468F4202D1C5F8047104E0EB5D00
:10D970008342F3D0C5F804710DF1700C4FF0000034
:10D98000FCF7CCFCFFF7B0B943F2D804C2F20004B4
:10D990004FF04806267204F0E2BBFAF7CFFF0A9D6B
:10D9A000401B0DF1700C4CF24F37B8428CBF002079
:10D9B0000120FCF7B3FCFFF797B94FF000001C9073
:10D9C0001C9E40F2A062C1F200024FF4117101FBF3
:10D9D000062393F82052032D7FF486A940F2A06716
:10D9E000C1F2000701FB067000F10406D0F808112F
:10D9F000D6F8002102F10102914238BF01F5807191
:10DA00008B1AFF2B34BF1D46FF250DF1700CE8B2B9
:10DA1000FCF784FCFFF768B91D9F41F26000C2F279
:10DA20000000C65D06F1FF31C155FFF75DB943F255
:10DA3000E802C2F20002137813F0280F06D01D98F6
:10DA4000B0F5005F34BF0020012004E01D98FA28E3
:10DA500094BF0020012040B143F2D804C2F2000478
:10DA60004FF01301217204F07ABB1D9E41F2600158
:10DA7000C2F200018A5D02F1FF33D8B28855002856
:10DA80003FF432A91E9E1C9601F01EBA43F2E80232
:10DA9000C2F20002137813F0280F06D01D98B0F5DB
:10DAA000005F34BF0020012004E01D98FA2894BFD5
:10DAB0000020012040B143F2D804C2F200044FF02C
:10DAC0001306267204F04BBB1D9E41F26001C2F2A8
:10DAD00000018A5D02F1FF33D8B28855002842F078
:10DAE0002087FFF701B943F2E801C2F200010A788A
:10DAF00012F0280F06D01D9BB3F5005F34BF002342
:10DB0000012304E01D9BFA2B94BF0023012343B1A2
:10DB100043F2D804C2F200044FF01300207204F064
:10DB20001EBB1D9841F26006C2F20006315C01F195
:10DB3000FF32D3B23354002B02F0F386FFF7D4B890
:10DB4000219D95F8517007F1FF3685F85160FFF778
:10DB5000CBB8219991F8472002F1FF3381F8473083
:10DB6000FFF7C2B82198C06C0BF02EFC219DE86431
:10DB7000FFF7BAB8219F97ED137AD7ED127A37EEF7
:10DB8000270A87ED130A2199C86C0AF0F9FE30B113
:10DB90004FF00200219981F85000FFF7A5B8219EAF
:10DBA000F06C0AF0FDFE30B14FF00102219B83F8CA
:10DBB0005020FFF799B84FF00007219D85F850706D
:10DBC000FFF792B89DF87400219901F14C01FEF71E
:10DBD00033F88DF86B0000283FF486A843F2D80490
:10DBE000C2F20004207204F0BABA9DF87400219EBB
:10DBF000F16CFEF755F88DF86B0000283FF474A81F
:10DC000043F2D801C2F20001087204F0A8BA219AC6
:10DC1000D06C0AF0C5FE20B9219B986C0AF0C0FEBA
:10DC200030B14FF00302219B83F85020FFF75CB81E
:10DC30002198D0ED138A90ED128A78EEC80A10EE82
:10DC4000900A0BF0C1FB09EE100A18EE900A18EECC
:10DC5000101A0BF037F801464FF07E500BF032F8F7
:10DC60009FEDCF1A01EE900A21EE812AB4EEC29AFE
:10DC7000F1EE10FA06D84FF00006219981F85060B5
:10DC8000FFF732B8219DD5ED132A95ED123AF4EE47
:10DC9000C32AF1EE10FA05DD4FF0010785F8507048
:10DCA000FFF722B8F4EEC32AF1EE10FA4CBF0222BD
:10DCB000032285F85020FFF717B82198D0ED133ACA
:10DCC000B7EE004A73EEC44AC0ED134A219EF06CD1
:10DCD0000AF066FE30B14FF00305219B83F85050E7
:10DCE000FFF702B82199D1ED138A9FEDAE8A38EE85
:10DCF000C89A19EE100A0BF067FB09EE100A18EE2D
:10DD0000900A18EE101A0AF0DDFF01464FF07E501F
:10DD10000AF0D8FFDFEDA23A04EE100A64EE234ABF
:10DD2000B4EEE49AF1EE10FA22D9219F97ED138A0E
:10DD3000DFED9C8A38EE285A15EE100A0BF044FBF2
:10DD400008EE900A18EE100A6FF052510AF0BAFF6E
:10DD500001464FF07E500AF0B5FFDFED915A06EE16
:10DD6000100A66EE256AF4EEE68AF1EE10FA06D89D
:10DD70004FF00407219A82F85070FEF7B5BF219A40
:10DD8000D56C28460BF020FB08EE100A28464FF011
:10DD900000010AF097FF01464FF07E500AF092FF13
:10DDA000DFED7F7A07EE100A27EE270AB4EEC08A6D
:10DDB000F1EE10FA06D84FF00006219981F8506074
:10DDC000FEF792BF219BD3ED130AF5EEC00AF1EEE8
:10DDD00010FA05DD4FF0010083F85000FEF784BF14
:10DDE000F5EEC00AF1EE10FA4CBF0222032283F8CE
:10DDF0005020FEF779BF219D95ED125AD5ED135AAB
:10DE000085EE256A85ED136ABDE6219EF06C0AF069
:10DE1000B3FD002841F05680FEF766BF2199CE6C15
:10DE200030460BF0D1FA08EE100A30464FF00001F0
:10DE30000AF048FF01464FF07E500AF043FFDFED45
:10DE4000586A07EE100A67EE267AB4EEE78AF1EE1A
:10DE500010FA01F33780FEF747BF219AD06C0AF021
:10DE60008BFD002801F02E80FEF73EBF219B93ED35
:10DE7000130AD3ED120AB4EEE00AF1EE10FA81F2C1
:10DE80002180FEF731BF219890ED131AD0ED121AC0
:10DE9000B4EEE11AF1EE10FA01F31480FEF724BF9C
:10DEA000219991ED132AD1ED122AB4EEE22AF1EE76
:10DEB00010FA41F20780FEF717BF219E96ED133A44
:10DEC000D6ED123AB4EEE33AF1EE10FA00F1FA8729
:10DED000FEF70ABF219AD66C30460BF075FA08EEB1
:10DEE000100A30464FF000010AF0ECFE01464FF0F8
:10DEF0007E500AF0E7FE9FED2A4A04EE900A24EED7
:10DF0000845AB4EEC58AF1EE10FA40F2DB87FEF7D0
:10DF1000EBBE219FF86CFCF751F8F8640DF1700C22
:10DF20004FF00000FCF7E6FAFEF7DEBE1D9BF62B75
:10DF300008D943F2D804C2F200044FF0120323724E
:10DF400004F00DB9219DE86C0AF016FD38B921994D
:10DF500091ED136AF6EE006A36EE268A06E0219805
:10DF600090ED138AF6EE005A38EE658A18EE100A24
:10DF70000AF002FD00BB9FED0C7AB4EEC78AF1EE09
:10DF800010FA04DC18EE100A0AF0FAFCA0B14FF007
:10DF90000106219F87F850606FF000463BE000BF0C
:10DFA00000000034FFFF7F4BFEFFFF4AFEFFFFCA69
:10DFB00000008043000080C318EE100A0AF0DCFC69
:10DFC00098B15FED067AB4EEE78AF1EE10FA04D468
:10DFD00018EE100A0AF0D4FC38B14FF00100219974
:10DFE00081F850004FF0004615E018EE100A0AF0D4
:10DFF000D7FC38B14FF00205219B83F850504FF009
:10E00000000608E0BDEEC88A18EE106A4FF000075F
:10E01000219A82F850704FEA066242EA166506F4C9
:10E020007F4345EA032006F47F0140EA112643F2CC
:10E030001417C2F200071D9ABE50FEF755BE1D9878
:10E04000F62808D943F2D804C2F200044FF01202B5
:10E05000227204F084B843F21415C2F200052E585F
:10E060004FEA066141EA166706F47F4247EA022357
:10E0700006F47F0043EA102500EE105AF8EEC00ABD
:10E08000219EC6ED130A1FED381AF4EEC10AF1EE17
:10E0900010FA06DC5FED3B1AF4EEE10AF1EE10FA3D
:10E0A00005D54FF0010786F85070FEF71DBE4FF002
:10E0B000000186F85010FEF717BE0DF1700C4FF0FE
:10E0C0000100FCF717FA219BD86CFBF7A1FF219DFB
:10E0D000E864FEF709BE219890ED132AF7EE002AB6
:10E0E00032EE223A80ED133AF0E52198C06C0AF046
:10E0F00057FC50B1219D4FF0000385F847304FF099
:10E10000040085F85000FEF7EFBD219E96ED131A2E
:10E11000B5EEC01AF1EE10FA23DB1FED5B3AB4EE58
:10E12000C31AF1EE10FA0FD5FCEEC13A13EE901AB5
:10E130000DF1700CC8B2FCF7F1F84FF00007219A0E
:10E1400082F85070FEF7D0BD0DF1700C4FF0FF005B
:10E15000FCF7E4F84FF00200219E86F85000FEF72D
:10E16000C3BDB5EEC01AF1EE10FA7EF5BDAD5FEDA0
:10E170006F1AB4EEE11AF1EE10FA11DDB1EE412A98
:10E18000FCEEC22A12EE902A0DF1700CD0B2FCF710
:10E19000C5F84FF00105219B83F85050FEF7A4BD50
:10E1A0000DF1700C4FF0FF00FCF7B8F84FF00301D1
:10E1B000219F87F85010FEF797BD43F2E806C2F2A0
:10E1C0000006317811F0280F08D01D9A02F10102E3
:10E1D000B2F5005F34BF0022012206E01D9A02F171
:10E1E0000102FA2A94BF0022012242B143F2D8046C
:10E1F000C2F200044FF01303237203F0B0BF219F5B
:10E2000097ED134AFDEEC44A14EE905A2BB21C93BC
:10E2100098B2C5F3072646EA002141F26002C2F235
:10E2200000021D9FD153FEF75FBD43F2E800C2F22A
:10E230000000067816F0280F08D01D9901F10101A1
:10E24000B1F5005F34BF0021012106E01D9901F105
:10E250000101FA2994BF0021012141B143F2D80400
:10E26000C2F200044FF01302227203F078BF219D26
:10E2700095ED135AFCEEC55A15EE902A97B21C97ED
:10E280004FEA172343EA072041F26006C2F2000674
:10E290001D997052FEF728BD1D9D219FBD64FEF79C
:10E2A00023BD1D98219BD864FEF71EBD0DF1700C97
:10E2B000FCF74CF806EE100AF8EE466A219EC6ED11
:10E2C000136AFEF711BD43F2E801C2F200010A78B9
:10E2D00012F0280F08D01D9800F10100B0F5005F82
:10E2E00034BF0020012006E01D9800F10100FA284B
:10E2F00094BF0020012040B143F2D804C2F20004D0
:10E300004FF01303237203F02ABF41F26005C2F2FB
:10E3100000051D9FEB5B4FEA132646EA03218AB2F4
:10E3200007EE902AB8EE670A219880ED130A9FED58
:10E33000C97AB4EEC70AF1EE10FAFEF6D5ACDFEDFD
:10E34000C60A30EE601A80ED131AFEF7CDBC43F218
:10E35000E806C2F20006317811F0280F08D01D9AA5
:10E3600002F10102B2F5005F34BF0022012206E093
:10E370001D9A02F10102FA2A94BF0022012242B141
:10E3800043F2D804C2F200044FF01300207203F0ED
:10E39000E6BE41F26005C2F200051D9FE85B4FEA50
:10E3A000102343EA0026B1B201EE901AB8EE612ABA
:10E3B000219A82ED132AFEF797BC1D98072808D9E9
:10E3C00043F2D803C2F200034FF008061E7203F0B6
:10E3D000C6BEFCF70FFC02EE900AB8EE623A219D31
:10E3E00085ED133AFEF780BC219FD7ED133A97EDE8
:10E3F000124A63EE844AC7ED134AFFF7C4BB219962
:10E4000091ED135AF1EE455AC1ED135AFEF76CBC6B
:10E410004FF000004FF001010A46FDF7D1FB219AB1
:10E4200092ED136AF1EE046A66EE267A4FF0000070
:10E430000090019043F22020C2F20000BCEEE70AF7
:10E4400010EE101A4FF0FF024BF62543C0F6020300
:10E45000FAF73EFAFEF748BC43F2E803C2F20003C3
:10E460001E7816F0280F08D01D9901F10301B1F5AF
:10E47000005F34BF0021012106E01D9901F1030175
:10E48000FA2994BF0021012141B143F2D804C2F21C
:10E4900000044FF01300207203F061BE41F26005EA
:10E4A000C2F200051D9FE859FBF7B2FD219A906466
:10E4B000FEF71ABC43F2E803C2F200031E7816F01E
:10E4C000280F08D01D9901F10301B1F5005F34BF99
:10E4D0000021012106E01D9901F10301FA2994BFF1
:10E4E0000021012141B143F2D804C2F200044FF0EF
:10E4F0001300207203F033BE41F26005C2F2000542
:10E500001D9FE859FBF784FD219AD064FEF7ECBB10
:10E510001D9B072B08D943F2D804C2F200044FF028
:10E520000806267203F01BBE219ED6ED130AF5EEF7
:10E53000C00AF1EE10FA0FDB9FED487AF4EEC70A3D
:10E54000F1EE10FA08D8FCEEE01ACDED1C1A4FF0EF
:10E55000000586F8505021E09FED401AF4EEC10A04
:10E56000F1EE10FA07DD6FF07F431C934FF00101CD
:10E5700086F8501012E04FF000011C9110EE900A46
:10E580000AF0FAF928B14FF00202219880F85020E1
:10E5900004E04FF00305219F87F850501D981C9907
:10E5A000FCF7FAFAFEF7A0BB219FF86C0AF0F8F925
:10E5B00000287EF499AB219890ED132AB5EEC02A7D
:10E5C000F1EE10FA04DD4FF07E53C364FEF78CBB0E
:10E5D000B5EEC02AF1EE10FA7EF586AB4FF00002E0
:10E5E000CBF68072C264FEF77FBB21998D6ACDB1F4
:10E5F000FAF7A4F9219FBA6AC2F1040318184CF67D
:10E60000CD41CCF6CC41A1FB00154FEA95067A6AC4
:10E61000B6FBF2F302EE903AB8EE623A87ED133AA7
:10E62000FEF762BB4FF6FF76C7F67F76CE64FEF745
:10E630005BBB43F2E800C2F20000017811F0280F42
:10E6400010D01D9E06F10306B6F5005F34BF00260C
:10E6500001260EE00000004700008047FFFF7F4BCF
:10E66000000000341D9E06F10306FA2E94BF00261A
:10E67000012646B143F2D804C2F200044FF013035E
:10E68000237203F06CBD1D9F219DE86CFBF796FC87
:10E6900041F26002C2F20002D051FEF725BB219880
:10E6A000D0ED123A90ED134A73EEC44AC0ED134A0E
:10E6B000FFF769BA219EF76C1C97B56CF564B764D7
:10E6C000FEF712BB219AD06C0AF06AF930B14FF014
:10E6D0000306219981F85060FEF706BB219BD86C98
:10E6E0000AF04EF930B14FF00400219B83F850003E
:10E6F000FEF7FABA2198C66C30460AF065FE08EEBD
:10E70000100A30464FF000010AF0DCFA01464FF0E3
:10E710007E500AF0D7FA1FED2E5A05EE900A25EE2C
:10E72000856AB4EEC68AF1EE10FA06D84FF00005FD
:10E73000219A82F85050FEF7D7BA2199D1ED136A89
:10E74000F5EEC06AF1EE10FA05DD4FF0010781F831
:10E750005070FEF7C9BAF5EEC06AF1EE10FA4CBF80
:10E760000222032281F85020FEF7BEBA219FD7ED86
:10E77000138A97ED128A38EEC89A19EE100A0AF039
:10E7800023FE09EE100A18EE900A18EE101A0AF08D
:10E7900099FA01464FF07E500AF094FA5FED507AF4
:10E7A00000EE100A60EE270AB4EEE09AF1EE10FADD
:10E7B0000DF1700C8CBF00200120FBF7AFFDFEF7C0
:10E7C00093BA219DEE6C30460AF0FEFD08EE100A69
:10E7D00030464FF000010AF075FA01464FF07E50C6
:10E7E0000AF070FA1FED621A07EE100A67EE011ABE
:10E7F000B4EEE18AF1EE10FA0DF1700C8CBF00203E
:10E800000120FBF78BFDFEF76FBA219A92ED132AD8
:10E81000D2ED122AB4EEE22AF1EE10FA0DF1700CEC
:10E82000B4BF00200120FBF779FDFEF75DBA219807
:10E8300090ED133AB5EEC03AF1EE10FA0DF1700C0E
:10E84000B4BF00200120FBF769FDFEF74DBA219B04
:10E85000D3ED133A93ED124AF4EEC43AF1EE10FA06
:10E860000DF1700CD4BF00200120FBF757FDFEF71F
:10E870003BBA2199D1ED134A91ED125AF4EEC54AF3
:10E88000F1EE10FA0DF1700C8CBF00200120FBF7A7
:10E8900045FDFEF729BA219FD7ED135A97ED126A6D
:10E8A000F4EEC65AF1EE10FA0DF1700C54BF0020D0
:10E8B0000120FBF733FDFEF717BA219DD5ED136A52
:10E8C000F5EEC06AF1EE10FA0DF1700C54BF0020A5
:10E8D0000120FBF723FDFEF707BA219ED6ED138A30
:10E8E00096ED128A38EEC89A19EE100A0AF06CFDFD
:10E8F00009EE100A18EE900A18EE101A0AF0E2F962
:10E9000001464FF07E500AF0DDF95FEDAB7A00EE84
:10E91000100A60EE270AB4EEE09AF1EE10FA0DF15B
:10E92000700CD4BF00200120FBF7F8FCFEF7DCB927
:10E93000219AD76C38460AF047FD08EE100A38468F
:10E940004FF000010AF0BEF901464FF07E500AF088
:10E95000B9F91FEDBD1A07EE100A67EE011AB4EE01
:10E96000E18AF1EE10FA0DF1700CD4BF0020012005
:10E97000FBF7D4FCFEF7B8B943F2E800C2F200009E
:10E98000037813F0280F08D01D9901F10201B1F5A9
:10E99000005F34BF0021012106E01D9901F1020151
:10E9A000FA2994BF0021012141B143F2D804C2F2F7
:10E9B00000044FF01300207203F0D1BBF9F7BEFF43
:10E9C000219F00F104004CF6CD45CCF6CC45A5FBCB
:10E9D00000164FEA96007A6AB0FBF2F31D9D41F2F1
:10E9E0006000C2F2000041194E78425D4FEA0245D4
:10E9F00045EA0620897840EA01061B969B1B23F016
:10EA00007F421C9202EE102AF8EE422AC7ED132A2A
:10EA1000FEF76AB9219FFD6CBD64FEF765B92199C7
:10EA200091F85160002E40F04D82FEF75DB9219BB8
:10EA300093F85120002A00F04582FEF755B943F2C1
:10EA4000E800C2F20000017811F0280F06D01D9EE8
:10EA5000B6F5005F34BF0026012604E01D9EFA2EA5
:10EA600094BF0026012646B143F2D804C2F2000446
:10EA70004FF01306267203F072BB41F26002C2F23D
:10EA800000021D9BD05C00287EF42EA91E991C91CB
:10EA90001AE243F2E802C2F20002137813F0280FE0
:10EAA00006D01D98B0F5005F34BF0020012004E0BF
:10EAB0001D98FA2894BF0020012040B143F2D804E9
:10EAC000C2F200044FF01300207203F048BB41F281
:10EAD0006001C2F200011D9E8A5D002A3EF404A975
:10EAE0001E9B1C93F0E11D990F2908D943F2D8030E
:10EAF000C2F200034FF027021A7203F030BBC8B213
:10EB0000FCF7AAFB00283EF4EFA81E9E1C96DBE152
:10EB10001D98F92808D943F2D804C2F200044FF036
:10EB20001200207203F01BBB43F21411C2F2000169
:10EB30000E5C1E9B1E427EF4D7A81F9A1C92C3E156
:10EB40001D99F92908D943F2D804C2F200044FF004
:10EB50001201217203F003BB43F21416C2F2000645
:10EB6000725C1E9B1A423EF4BFA81F981C90ABE13A
:10EB700043F2E806C2F20006327812F0280F06D0FF
:10EB80001D9BB3F5005F34BF0023012304E01D9BF0
:10EB9000FA2B94BF0023012343B143F2D804C2F2FD
:10EBA00000044FF01303237203F0D9BA41F260005E
:10EBB000C2F200001D99465C002E7EF495A81E9AB4
:10EBC0001C92B2E143F2E800C2F20000017811F0B9
:10EBD000280F06D01D9EB6F5005F34BF0026012623
:10EBE00004E01D9EFA2E94BF0026012646B143F292
:10EBF000D804C2F200044FF01306267203F0AFBA35
:10EC000041F26002C2F200021D9BD05C00283EF47B
:10EC10006BA81E991C9188E143F2E802C2F200023F
:10EC2000137813F0280F06D01D98B0F5005F34BF9D
:10EC30000020012004E01D98FA2894BF0020012044
:10EC400040B143F2D804C2F200044FF01301217224
:10EC500003F085BA41F26001C2F200011D9E8A5D97
:10EC60001E9B9A427EF640A81F981C902CE143F20E
:10EC7000E806C2F20006327812F0280F06D01D9B7B
:10EC8000B3F5005F34BF0023012304E01D9BFA2B82
:10EC900094BF0023012343B143F2D804C2F200041D
:10ECA0004FF01300207203F05ABA41F26000C2F232
:10ECB00000001D99465C1E9A9642FEF415A81F9B03
:10ECC0001C9301E143F2E801C2F200010E7816F054
:10ECD000280F06D01D9AB2F5005F34BF0022012232
:10ECE00004E01D9AFA2A94BF0022012242B143F2A5
:10ECF000D804C2F200044FF01300207203F02FBAC0
:10ED000041F26000C2F200001D9BC15C1E9EB14238
:10ED10007DF4EAAF1F9A1C92D6E043F2E803C2F2F8
:10ED20000003197811F0280F06D01D9EB6F5005F7C
:10ED300034BF0026012604E01D9EFA2E94BF002653
:10ED4000012646B143F2D804C2F200044FF0130288
:10ED5000227203F004BA41F26002C2F200021D986E
:10ED6000115C1E9B99423DF4BFAF1F9E1C96ABE009
:10ED700043F2E800C2F20000017811F0280F06D03B
:10ED80001D9BB3F5005F34BF0023012304E01D9BEE
:10ED9000FA2B94BF0023012343B143F2D804C2F2FB
:10EDA00000044FF01306267203F0D9B941F2600651
:10EDB000C2F200061D9AB05C1E9988423DF694AFDF
:10EDC0001F9B1C9380E043F2E802C2F2000210781D
:10EDD00010F0280F06D01D99B1F5005F34BF002157
:10EDE000012104E01D99FA2994BF0021012141B1BC
:10EDF00043F2D804C2F200044FF01306267203F067
:10EE0000AEB941F26006C2F200061D9BF25C1E988C
:10EE10008242BDF469AF1F991C9155E0219B93F884
:10EE200047201D9882427DF45FAF1E991C917CE0C3
:10EE3000219E96F847201D9B9A423DF455AF1E989F
:10EE40001C9072E0219991F847601D9A96427DF6D8
:10EE50004BAF1E9B1C9368E0219890F847101D9EB5
:10EE6000B142FDF441AF1E9A1C925EE0219B93F8E3
:10EE700047001D998842BDF437AF1E9E1C9654E092
:10EE8000219A92F847001D9B98423DF62DAF1E999E
:10EE90001C914AE09DF874000DF16B01FCF7ACFD8C
:10EEA0008DF86A009DF86B6036B143F2D804C2F267
:10EEB0000004267203F053B900283DF415AF1E9AE2
:10EEC0001C9201E01D981C901C9E40F20000C0F6B0
:10EED000010090F82E1090F82F3043EA0122B24240
:10EEE00008D243F2D804C2F200044FF00906267299
:10EEF00003F035B943F21427C2F200073E60FDF774
:10EF0000F3BE0DF1700CFBF721FA1C900028D9D04C
:10EF1000FDF7EABE0DF1700CFBF718FA1C90002803
:10EF2000D0D1FDF7E1BE1D9B1C93219A136A052BDE
:10EF300008D943F2D804C2F200044FF00A03237246
:10EF400003F00DB903F1020043F21421C2F20001F3
:10EF50000E6842F8206003F10103219A1362B3E7BF
:10EF60000DF1700CFBF7F2F91C900028DBD0FDF7D7
:10EF7000BBBE0DF1700CFBF7E9F91C900028D2D153
:10EF8000FDF7B2BE0DF1700CFBF7E0F91C901D9976
:10EF900088427DF4A9AE1E9E1C9695E70DF1700C7B
:10EFA000FBF7D4F91C901D9A90423DF49DAE1E983B
:10EFB0001C9089E70DF1700CFBF7C8F91C901D9BA4
:10EFC00098427DF691AE1E991C917DE70DF1700C73
:10EFD000FBF7BCF91C901D9EB042FDF485AE1E9A55
:10EFE0001C9271E70DF1700CFBF7B0F91C901D9BA2
:10EFF0009842BDF479AE1E981C9065E70DF1700C37
:10F00000FBF7A4F91C901D9988423DF66DAE1E9E3B
:10F010001C9659E79DF874000DF16B01FCF7BAFCE2
:10F020008DF86A009DF86B3033B143F2D804C2F218
:10F030000004237203F093B800283DF455AE1E9AE5
:10F040001C9241E79DF874000DF16B01FCF7A2FCE6
:10F050008DF86A009DF86B1031B143F2D806C2F208
:10F060000006317203F07BB800287DF43DAE1E9897
:10F070001C9029E70DF1700CFBF790F941F260024A
:10F08000C2F200021E9BD15C1D9801423DF42CAEE1
:10F090001F9E1C9618E70DF1700CFBF77FF941F2EB
:10F0A0006002C2F200021E9BD15C1D9801427DF4F9
:10F0B0001BAE1F9E1C9607E70DF1700CFBF76EF957
:10F0C00041F26002C2F200021E9BD15C1D98014217
:10F0D0007DF40AAE1F9E1C9627E70DF1700CFBF71E
:10F0E0005DF941F26002C2F200021E9BD15C1D98E4
:10F0F00001423DF4F9AD1F9E1C9616E798F80050AA
:10F1000045F0080088F80000FDF717BE0DF1700CFF
:10F11000FBF71CF98DF86A00219991F851601D9A4E
:10F12000B3181C9343F2E801C2F200010E7816F006
:10F13000280F09D01E9E06F1FF32D318B3F5005FE9
:10F1400034BF0023012307E01E9A02F1FF31CB18E0
:10F15000FA2B94BF0023012343B143F2D804C2F237
:10F1600000044FF01303237202F0F9BF4FF00007C1
:10F170001B971E9DE5B11C9941F26003C2F200038A
:10F180005E5C864235D005F1FF3241F26007C2F283
:10F1900000077B1841F26005C2F20005C5F10106C7
:10F1A000C1F101014F1B12F0010F1AD003F042B858
:10F1B0004FF0FF001B901CE013F8019F02F1FF3895
:10F1C000484504D11C91CDF86CE01E9211E04246F6
:10F1D000F11807EB030E13F8015FA84243F03780E4
:10F1E000F0E7F11807EB030E002AE5D11C911E92FF
:10F1F000DEE70DF1700C9DF86C00FBF78FF8FDF762
:10F2000073BD0DF1700CFBF7A1F843F28C0BC2F249
:10F21000000B8BF800004FF001061C96CDF830B0C3
:10F22000BBE0219991F851201D9813181C9343F2CB
:10F23000E806C2F20006317811F0280F07D003F17A
:10F240000103B3F5005F34BF0023012305E003F1A0
:10F250000103FA2B94BF0023012343B143F2D804E6
:10F26000C2F200044FF01302227202F078BF1E981F
:10F270001B900DF1700C26AF47F0010122AD45F057
:10F2800001024FF00003FBF79BF8FDF72DBD21981D
:10F2900090F851601D9BF1181C9143F2E802C2F2F4
:10F2A0000002107810F0280F05D0B1F5005F34BFD0
:10F2B0000021012103E0FA2994BF0021012141B17D
:10F2C00043F2D804C2F200044FF01303237202F099
:10F2D00046BF1F9F1E98B84228BF38461B900DF1AD
:10F2E000700C26AD45F0010122AE46F001024FF050
:10F2F0000003FCF71DF9FDF7F7BC0DF1700CFBF7EF
:10F3000025F8034643F28C0BC2F2000B58464FF02F
:10F3100010014EF6F812C0F603020AF037FA1C90FC
:10F32000CDF830B039E01E991C911F9A1B924FF016
:10F3300000000C9031E04FF0FF361C960C962CE04C
:10F34000219BD86C9DF878109DF87C2043F28C06A8
:10F35000C2F2000600964FF0100301934FF0010334
:10F36000FDF75CF84FF0FF311C910C9615E0219AE7
:10F37000D06C9DF878109DF87C2043F28C06C2F288
:10F38000000600964FF0100301934FF00003FDF7C5
:10F3900045F84FF0FF301C900C961D99A1F1FB0031
:10F3A00086B20B96A1F1FB03032B23D840F2A06099
:10F3B000C1F200004FF411760B9906FB010393F89C
:10F3C0002022032A08D043F2D806C2F200064FF0EA
:10F3D0004803337202F0C3BE40F2A067C1F20007D7
:10F3E0004FF411700B9E00FB067707F104074FF0F6
:10F3F000000605E0219F97F8512056184FF00007AE
:10F40000DDF870B0BBF1FF3F11D14FF0FF0B4FF0B3
:10F410000009C84643F2E801C2F200010D9141F231
:10F420006003C2F200030E930F950C9D05E0BBF143
:10F43000000FECD14FF000096FE01D9AA2F1FB0222
:10F44000032A10D8D7F80061FF2E14BF01364646B4
:10F45000D7F80401864206D14046FCF7C9F8D7F830
:10F4600004118E42F8D0B5F1FF3F15D1219850F824
:10F47000341F0B68D3F800C0494610AA4FF00103AF
:10F48000E0478DF86B0080B10F9D43F2D804C2F2C3
:10F490000004207202F063BE25B115F809208DF832
:10F4A000402002E01B9B8DF840301C98B0F1FF3FDC
:10F4B00002D19DF8402082B31D99A1F1FB010329DF
:10F4C00007D8D7F800319DF84000F854C7F800611C
:10F4D0001FE00D9B187810F0280F05D0B6F5005FDF
:10F4E00034BF0020012003E0FA2E94BF0020012049
:10F4F00048B10F9D43F2D804C2F200044FF0130646
:10F50000267202F02CBE9DF840200E998A5506F115
:10F51000010609F10109D9458FD31D9FA7F1FB070A
:10F52000032F05D80B99C8B2FBF7A0F9FDF7DCBB98
:10F53000219D95F8512009EB020E85F851E0FDF769
:10F54000D3BB1D9AA2F1FB01032958D88FB240F218
:10F55000A060C1F200004FF4117101FB070292F8A4
:10F560002032032B08D043F2D804C2F200044FF03B
:10F570004803237202F0F3BD40F2A066C1F2000618
:10F580004FF4117505FB076505F104051E9800F1A0
:10F59000FF311E9170B34FF0000843F21429C2F2FC
:10F5A000000940F200029346C0F6010BD5F8006155
:10F5B000FF2E14BF01364646D5F804319E4206D1CF
:10F5C0004046FCF715F8D5F804018642F8D0D9F882
:10F5D0000030D5F800211BF80310A95403F10103F2
:10F5E000C9F80030C5F800611E9E06F1FF301E907C
:10F5F000002EDBD1F8B2FBF739F9FDF775BB1E9B86
:10F600001C93219991F8510082181B9243F2E8064D
:10F61000C2F20006367816F0280F08D003F1FF3644
:10F62000B218B2F5005F34BF0022012206E003F1F8
:10F63000FF36B218FA2A94BF0022012242B143F2E7
:10F64000D804C2F200044FF01306267202F087BD00
:10F65000C71881F851701C9A02F1FF351C95002AD9
:10F660003DF442AB43F21423C2F200031E681B9F19
:10F6700041F26001C2F20001C91940F20000C0F677
:10F68000010030184FF0000305F0010910F803C025
:10F6900001F803C003F10103934242F0BC850DE081
:10F6A00010F803E001F803E003F1010310F8039000
:10F6B00001F8039003F101039342F1D1E819A9196C
:10F6C00001F1010143F21422C2F2000211604FF075
:10F6D000FF331C9300F101001B90FDF705BB4FF0B9
:10F6E00000028DF86A20219E96F851001D9BC118DA
:10F6F0001C911E9A1B9243F2E800C2F200000378AC
:10F7000013F0280F08D002F1FF335818B0F5005F4E
:10F7100034BF0020012006E002F1FF325018FA2821
:10F7200094BF0020012040B143F2D804C2F200048B
:10F730004FF01302227202F012BD41F26007C2F2D2
:10F74000000707EB01099DF87CB043F21025C2F2D7
:10F7500000052A68B66B9119905DFF2859D088463C
:10F760004FF001070894CDF82CA0BA4698F8014054
:10F7700004EB002343F21025C2F200052A68D618D4
:10F780004FF000011C919DF86A00002802F01985D5
:10F79000D75C06F1010602F016BD9DF86A402CB157
:10F7A0008FB9089C5046DDF82CA005E0727852B95C
:10F7B000089C5046DDF82CA0219F97F851609B19BA
:10F7C00087F8513027E016F8014F19F803B045B912
:10F7D000204609F07FFFC4B2584609F07BFF5FFA6C
:10F7E00080FB5C4508D11C9B03F101031C9307F1CE
:10F7F000FF371B999942D0D2AB460AF1010A18F89B
:10F80000020FFF28B2D1089CDDF82CA04FF00000B9
:10F8100001E04FF000000DF1700CC0B2FAF77EFD70
:10F82000FDF762BA4FF001018DF86A105BE70DF148
:10F83000700CFAF78BFD034643F28C0BC2F2000BFF
:10F8400058464FF010014EF60022C0F6030209F0B0
:10F850009DFF1C90CDF830B09FE50DF1700CFAF7CC
:10F8600075FD034643F28C0BC2F2000B58464FF075
:10F8700010014EF60822C0F6030209F087FF1C9023
:10F88000CDF830B089E50DF1700CFAF75FFD034655
:10F8900043F28C0BC2F2000B58464FF010014EF6AB
:10F8A0000C22C0F6030209F071FF1C90CDF830B0B5
:10F8B00073E50DF1700CFAF749FD034643F28C0B2A
:10F8C000C2F2000B58464FF010014EF61422C0F65B
:10F8D000030209F05BFF1C90CDF830B05DE5219884
:10F8E00090F8517007F1010780F85170FDF7FCB9ED
:10F8F0001D9D41F26002C2F20002515D01F1010161
:10F900005155FDF7F1B9219E96F8473003F10103F7
:10F9100086F84730FDF7E8B99DF874000DF16B01EA
:10F92000FCF738F80DF1700CFAF7F8FC9DF86B0055
:10F9300000283DF4D9A943F2D804C2F20004207291
:10F9400002F00DBC9DF874000DF16B01FCF78EF810
:10F950000DF1700CFAF7E2FC9DF86B1000293DF4F4
:10F96000C3A943F2D802C2F20002117202F0F7BB3F
:10F970001D9E1C964FF000031B934FF001008DF865
:10F980006A009DF870000DF16B01FCF703F89DF81B
:10F990006B1099B920B19DF86A201B9E16431B96E7
:10F9A0009DF86A304FEA43008DF86A001C9901F116
:10F9B00001011C9110F0FE0FE3D10AE09DF86A20CE
:10F9C000012A06D143F2D804C2F20004217202F0E7
:10F9D000C6BB0DF1700C9DF86C00FAF79FFCFDF7AB
:10F9E00083B91D9E1C964FF000031B934FF001003E
:10F9F0008DF86A009DF870000DF16B01FCF736F888
:10FA00009DF86B1099B920B19DF86A201B9E164392
:10FA10001B969DF86A304FEA43008DF86A001C99E6
:10FA200001F101011C9110F0FE0FE3D10AE09DF8F5
:10FA30006A20012A06D143F2D804C2F200042172DE
:10FA400002F08DBB0DF1700C9DF86C00FAF766FCAE
:10FA5000FDF74AB99DF874000DF16B01FBF7CCFF7F
:10FA60008DF86A009DF86B6036B143F2D803C2F29C
:10FA700000031E7202F073BB0DF1700CFAF74EFC1E
:10FA8000FDF732B91D981C904FF000011B914FF00B
:10FA900001008DF86A00219A92F8476030420ED03A
:10FAA0009DF870000DF16B01FBF7A6FF9DF86B3020
:10FAB0009BB920B19DF86A001B9901431B919DF8E9
:10FAC0006A204FEA42068DF86A601C9B03F101032D
:10FAD0001C9316F0FE00DED10AE09DF86A100129A1
:10FAE00006D143F2D804C2F20004237202F037BBFD
:10FAF0001B9F219D85F84770FDF7F6B89DF87400AF
:10FB00000DF16B01FBF7E4FF0DF1700CFAF706FC49
:10FB10009DF86B60002E3DF4E7A843F2D802C2F2D4
:10FB20000002167202F01BBB1D9B1C93D8B20DF194
:10FB30006B01FBF7CDFF1B909DF86B0030B143F2DA
:10FB4000D804C2F20004207202F009BB4FF0010198
:10FB50008DF86A101C9F7A181C92D0B20DF16B01BF
:10FB6000FBF7B6FF9DF86A5000FA05F01B9E0643AE
:10FB70001B9605F101058DF86A501C9A02F10102ED
:10FB80001C92EBB2072BE8D90DF1700C9DF86C00BC
:10FB9000FAF7C4FBFDF7A8B80DF1700C219890F8A6
:10FBA0005100FAF7BBFBFDF79FB8FDF79DB843F294
:10FBB000C001C2F200014FF001070F70FDF794B8C9
:10FBC00043F2C005C2F200054FF000062E70FDF7AB
:10FBD0008BB821984FF000014FF054020AF00CFA54
:10FBE0004FF00002219243F29C03C2F200031C6812
:10FBF00004F1FF30186002F01EBA43F29C02C2F218
:10FC0000000213687F2B08D943F2D804C2F2000423
:10FC10004FF03000207202F0A2BA4FF001071C979B
:10FC200040F2A065C1F20005D5F8E809002842F0CD
:10FC3000D58205E0D6F8AC20002A4ED11C9301E015
:10FC40004FF001031D9840F2A066C1F200064FF08C
:10FC5000540505FB03F3F218C2F89009C2F89409A1
:10FC60001E9982F8E2194FF00A07C2F8B47906F536
:10FC70001967F81800F13400219901F134014FF0AF
:10FC800010020AF095F91C9B05FB037000F144007B
:10FC9000219901F144014FF004020AF089F91C98FE
:10FCA00005FB007000F14800219901F148014FF077
:10FCB00008020AF07DF9219A92F851101C9F05FB69
:10FCC000076686F8E11943F29C05C2F200052B682D
:10FCD00003F101032B60FDF707B803F101073B4671
:10FCE00006F15406D6F8AC50002D42F08B82A5E701
:10FCF0001C93FCF7F9BF219991F852601E967CE79E
:10FD00000DF1700CFAF722FB1E9076E71D9A2199EF
:10FD100081F85120FCF7E8BF0DF1700C9DF87400DC
:10FD2000FAF7FCFAFCF7E0BF219EB36A002B3CF423
:10FD3000DBAFF8F703FE219B9A6A861A586A1D9B6F
:10FD400003FB00F008F07EF94FF000024FF00003D3
:10FD5000C4F2040308F0E2FB08F008FA8642BCF49F
:10FD6000C3AF1E981C90FFF7AFB8F8F7E7FD219FCF
:10FD7000B862FCF7B9BF43F21412C2F2000292F863
:10FD8000FB201E9E9119FB2908D943F2D800C2F22C
:10FD900000004FF01201017202F0E1B943F2E803F2
:10FDA000C2F20003187810F0280F09D01D995318DB
:10FDB00003F1FF30B0F5005FB4BF0020012007E081
:10FDC0001D99531803F1FF30FA28D4BF00200120F9
:10FDD00040B143F2D804C2F200044FF01302227281
:10FDE00002F0BDB943F21415C2F20005A81941F2A0
:10FDF0006007C2F200071D9EB9190AF0D9F8FCF796
:10FE000073BF98F8003043F0100588F80050FCF7F5
:10FE100094BF219F97F84760002E0CBFFF2200225D
:10FE200087F84720FCF760BF219890F847106FEAE9
:10FE3000010380F84730FCF757BF0DF1700CFAF75B
:10FE4000ADFA1E9D41F26007C2F200077E5D1D9A69
:10FE500072407A55FCF748BF2198816B1D9B5E1854
:10FE60001C96BDE12198C26B816B53181C93B7E1BE
:10FE7000219E306C40B943F2D804C2F200044FF026
:10FE80002002227202F06BB900F1FF353564FCF7F5
:10FE90002BBF21990B6C03F101030B64002B7CF445
:10FEA00023AF43F2D806C2F200064FF020003072B2
:10FEB00002F055B9219A516B0B685E6846B943F25E
:10FEC000D800C2F200004FF01E03037202F047B9DF
:10FED0000DF1700CFAF73AFA1C90219850F8342F73
:10FEE00011684E681D991CAA4FF00103B0478DF8A8
:10FEF0006B0000283CF4F8AE43F2D804C2F20004D0
:10FF0000207202F02CB90DF1700CFAF71FFA1C9058
:10FF100054E10DF1700CFAF719FA219FF863FCF720
:10FF2000E3BE0DF1700CFAF711FA219D2864FCF77D
:10FF3000DBBE219850F8342F11680E681D991CAA59
:10FF40004FF00103B0478DF86B0030B143F2D80495
:10FF5000C2F20004207202F002B90DF1A80C1CF8E4
:10FF6000380DFAF7DBF9FCF7BFBE2198436B0DF1B2
:10FF7000700C187AFAF7D2F9FCF7B6BE0DF1700CD6
:10FF8000219F97F83C00FAF7C9F9FCF7ADBE219A1A
:10FF9000116CFF2908D943F2D806C2F200064FF0CF
:10FFA0002004347202F0DBB80DF1700CC8B2FAF71D
:10FFB000B5F9FCF799BE219850F8345F2B689F681B
:10FFC000B84703EE100AF8EE433A2198C0ED133A11
:10FFD000FCF78ABE219A92ED0E4AF8EE444AC2ED31
:10FFE000134AFCF781BE219991ED105AF8EE455A5B
:10FFF000C1ED135AFCF778BE219E96ED136AFCEE14
:020000040803EF
:10000000C66ACDED1C6AEBE0219BD3ED137A9FED20
:10001000B40AF4EEC07AF1EE10FA08DB43F2D80429
:10002000C2F200044FF02000207202F098B8FCEEFB
:10003000E70AC3ED100AFCF757BE219850F8342F99
:1000400011680E681D991CAA4FF00403B0478DF883
:100050006B0030B143F2D803C2F20003187202F011
:100060007EB81C98F9F7D4FF219DA864FCF73CBE2C
:10007000219850F8342F11680E681D991CAA4FF072
:100080000403B0478DF86B0030B143F2D804C2F2DC
:100090000004207202F063B81C98F9F7B9FF219FA1
:1000A000F864FCF721BE2198436B1A68516841B986
:1000B00043F2D800C2F200004FF01E02027202F0BA
:1000C0004EB8C06CF9F77AFF1C90219850F8346F45
:1000D00033685E681D991CAA4FF00403B0478DF881
:1000E0006B0000283CF400AE43F2D804C2F20004D6
:1000F000207202F034B843F2E801C2F200010B783A
:1001000013F0280F0BD0219EF06B1D9A111801F1EE
:10011000FF33B3F5005F34BF0023012309E0219EC4
:10012000F06B1D9A111801F1FF33FA2B94BF0023D5
:10013000012343B143F2D800C2F200004FF0130193
:10014000017202F00CB8219B184650F8347F3E68CB
:1001500036684FF0000141F26007C2F200071D9AB5
:10016000BA18DB6BB0478DF86B0000283CF4BCADCF
:1001700043F2D804C2F20004207201F0F0BF2198CB
:1001800050F8343F1E6836681D991BAA4FF00403CF
:10019000B0478DF86B0030B143F2D804C2F20004CE
:1001A000207201F0DCBF1B9882B2C0F3072141EA44
:1001B00002239EB21C9613E01D981C901C98219956
:1001C000FAF762F98DF86B0000283CF48DAD43F22C
:1001D000D802C2F20002107201F0C1BF1D991C9139
:1001E0001C9BB3F5803F08D343F2D804C2F200044D
:1001F0004FF01F00207201F0B2BF219DAB63FCF7EE
:1002000073BD1D9D219FFD63FCF76EBD1D9E219B4F
:100210001E64FCF769BD2198826B1D99561A1C96C5
:10022000DEE71E9A219BD96B8E18FB2E08D943F26C
:10023000D800C2F200004FF01202027201F08FBF2C
:1002400043F21417C2F2000787F8FB10184650F863
:10025000341F0E6836681D99BA18DB6BB0478DF8ED
:100260006B0000283CF440AD43F2D804C2F2000415
:10027000207201F074BF219B596B0E68766846B9F5
:1002800043F2D801C2F200014FF01E00087201F0E3
:1002900066BF43F2E800C2F20000027812F0280FB5
:1002A0000AD0DA6B1D99881800F1FF30B0F5005FB5
:1002B00034BF0020012008E0D86B1D990A1802F114
:1002C000FF30FA2894BF0020012058B143F2D80330
:1002D000C2F200034FF013061E7201F040BF00BFD0
:1002E0000000804703F134004FF0000141F2600745
:1002F000C2F200071D9ABA18DB6BB0478DF86B008D
:1003000000283CF4F1AC43F2D804C2F2000420729D
:1003100001F025BFF6F72AFA00287CF4E5AC1D9A17
:100320001C92FEF7D1BDF6F721FA00283CF4DCACB4
:100330001D9B1C93FEF7C8BD1D9E0C2E08D943F2D1
:10034000D804C2F200044FF00501217201F007BF8A
:10035000F0B24FF00001F6F7C7F901EE100AB8EE5F
:10036000417A219F87ED137AFCF7BEBC1D980C28BB
:1003700008D943F2D803C2F200034FF005021A7203
:1003800001F0EDBEC0B24FF00101F6F7ADF901EE9C
:10039000900AB8EE612A219D85ED132AFCF7A4BCD2
:1003A0001D9E0C2E08D943F2D804C2F200044FF06F
:1003B0000501217201F0D3BEF0B24FF00001F6F753
:1003C00003F9FCF791BC1D980C2808D943F2D80317
:1003D000C2F200034FF005021A7201F0C0BEC0B2B3
:1003E0004FF00101F6F7F0F8FCF77EBC1D9E0C2ED5
:1003F00008D943F2D804C2F200044FF0050121727B
:1004000001F0ADBEF0B24FF00001F6F72DF9FCF7A8
:100410006BBC1D980C2808D943F2D803C2F2000324
:100420004FF005021A7201F09ABEC0B24FF00101FE
:10043000F6F71AF9FCF758BC9DF87400F1F72EFB9B
:1004400000287CF451AC43F2D806C2F200064FF00B
:100450002804347201F083BE9DF87400219901F1E3
:100460004C01F1F73BFB00287CF43EAC43F2D80191
:10047000C2F200014FF02800087201F070BE219B0B
:10048000D3ED132A9DF87400BCEEE23A13EE101A75
:10049000F1F756FB00287CF427AC43F2D806C2F2F1
:1004A00000064FF02802327201F059BEFCF71CBC66
:1004B0000DF1700CF9F74AFF30B9219F97F84750BA
:1004C000291C18BF012101E04FF00101219880F89B
:1004D0004710FCF709BC9DF874600DF1700CF9F73A
:1004E00035FF014630464FF00102FBF769FB8DF8FE
:1004F0006B0000283CF4F8AB43F2D804C2F20004CD
:10050000207201F02CBE0DF1700CF9F71FFF0146AF
:100510008DF86A009DF87400FBF710FB8DF86B00F6
:1005200000283CF4E1AB43F2D803C2F20003187296
:1005300001F015BE1D9A1C924FF001038DF86A3030
:100540001E46219890F847100B420AD090F84610AA
:100550009DF8700019403246FBF732FB8DF86B00B6
:1005600068B99DF86A304FEA43008DF86A001C9A1A
:1005700002F101021C9210F0FE03E2D10AE09DF8A4
:100580006A60012E06D143F2D804C2F20004207240
:1005900001F0E5BD4FF000078DF86B700DF1700CA8
:1005A000F9F7D4FE0DF1700CF9F7D0FEFCF79CBB07
:1005B0009DF874004FF001010A46FBF701FB8DF82E
:1005C0006B0000283CF490AB43F2D801C2F200016A
:1005D000087201F0C4BD9DF874004FF000014FF0A7
:1005E0000102FBF7EDFA8DF86B0000283CF47CABC0
:1005F00043F2D802C2F20002107201F0B0BD0DF158
:10060000700CF9F7A3FE219D95F84730184385F843
:100610004700FCF769BB1D980DF1A80C4CF8380D8C
:10062000FAF742FB00287CF45FAB43F21426C2F2D7
:1006300000060898306001F015BD10A8FAF7C6F959
:10064000014640B19DF84070022F04D0C2484FF0DF
:100650000D0209F0ADFC0DF1700C9DF84000F9F7AA
:100660005DFEFCF741BBFAF7E3FEFCF73DBB0DF185
:10067000700CF9F76BFEFCF737BB1D9EFA2E08D9FC
:1006800043F2D804C2F200044FF01202227201F0C9
:1006900066BD0DF1700CF9F759FE43F21411C2F268
:1006A00000018855FCF720BB0DF1700CF9F74EFEE8
:1006B00043F21415C2F2000585F8FB00FCF714BBE9
:1006C0000DF1700C219B93F84700F9F727FEFCF71A
:1006D0000BBB1D98FA2808D943F2D806C2F20006CF
:1006E0004FF01201317201F03ABD0DF1700C43F27E
:1006F0001417C2F20007385CF9F710FEFCF7F4BAE1
:100700000DF1700C43F21412C2F2000292F8FB00D9
:10071000F9F704FEFCF7E8BA1D9EF62E08D943F25D
:10072000D804C2F200044FF01200207201F017BD8D
:10073000219DA86CF9F742FC43F21413C2F20003A6
:100740009851FCF7D1BA43F2E801C2F200010A78ED
:1007500012F0280F06D01D9EB6F5005F34BF0026AC
:10076000012604E01D9EFA2E94BF0026012646B104
:1007700043F2D803C2F200034FF013041C7201F0DD
:10078000EEBC0DF1700C41F26007C2F200071D9D36
:10079000785DF9F7C3FDFCF7A7BA0DF1700CF9F716
:1007A000FDFD41F26000C2F200001E99425C1D9EF8
:1007B00032420DF1700C0CBF0020FF20F9F7AEFDA6
:1007C000FCF792BA43F2E803C2F20003187810F083
:1007D000280F08D01D9901F10101B1F5005F34BF68
:1007E0000021012106E01D9901F10101FA2994BFC0
:1007F0000021012141B143F2D800C2F200004FF0C4
:100800001301017201F0ABBC1D9A41F26006C2F205
:100810000006B05CB318597841EA00221C92002A05
:100820003CF462AAFEF750BB43F2E803C2F20003B5
:100830001A7812F0280F06D01D9EB6F5005F34BF5F
:100840000026012604E01D9EFA2E94BF00260126F4
:1008500046B143F2D804C2F200044FF013022272F0
:1008600001F07DBC41F26000C2F200001D99435CC2
:10087000002B56D1FCF738BA43F2E806C2F2000664
:10088000307810F0280F06D01D99B1F5005F34BF05
:100890000021012104E01D99FA2994BF00210121C2
:1008A00041B143F2D804C2F200044FF013002072A9
:1008B00001F055BC41F26002C2F200021D9BD65C01
:1008C0007EB3FCF711BA0DF1700CF9F73FFD1C90E7
:1008D00038BBFCF709BA0DF1700CF9F75FFD41F276
:1008E0006001C2F200011E9A8E5C1D9B1E4218D050
:1008F000FCF7FAB90DF1700CF9F750FD41F2600008
:10090000C2F200001E99425C1D9E324209D1FCF7E2
:10091000EBB90DF1700CF9F719FD1C9000287CF46F
:10092000E3A9219B1E6A46B943F2D804C2F200042F
:100930004FF00300207201F012BC06F1FF351D627A
:1009400006F1010653F8267043F21421C2F20001A9
:100950000F60FCF7C9B900BF6610002098F800507E
:1009600045F0200388F80030FCF7E7B9219F97F89D
:1009700047004FEAD01141EA400287F84720FCF7D0
:10098000B3B9219E96F847504FEA550343EAC5177D
:1009900086F84770FCF7A8B9FAF7EAF8FCF7A4B9AB
:1009A00041F25800C2F20000C2784FF0010101FA92
:1009B00002F1067926EA01060671FCF795B943F2C1
:1009C0001415C2F2000541F25807C2F200073B7845
:1009D00078780090BA78019228464FF0FB014EF6E5
:1009E0001822C0F6030208F0D1FE85F8FB00FCF7E0
:1009F0007BB941F25803C2F20003D97841B941F200
:100A00005807C2F200074FF00600F870FCF76CB907
:100A100001F1FF3641F25805C2F20005EE70FCF715
:100A200063B941F25802C2F20002137803F1FF31B8
:100A3000CEB216701579FF2D0BD1632E7CF654A91A
:100A400041F25803C2F200034FF063021A70FCF740
:100A50004BB9172E7CF648A941F25807C2F200079D
:100A60004FF017003870FCF73FB941F25801C2F25D
:100A700000014E7806F1FF35EFB24F700879FF287C
:100A80000BD1002F7CF430A941F25801C2F20001D1
:100A90004FF00C064E70FCF727B93B2F7CF624A9CB
:100AA00041F25803C2F200034FF03B025A70FCF7C8
:100AB0001BB941F25805C2F20005AF7807F1FF30CB
:100AC000C2B2AA702B79FF2B17D141F25805C2F29E
:100AD00000052F78687807F5FA61F7F72DF88DF89B
:100AE0006A00AA7812B19042BCF4FEA841F2580301
:100AF000C2F200039870FCF7F7B83B2A7CF6F4A822
:100B000041F25801C2F200014FF03B068E70FCF733
:100B1000EBB843F21410C2F200004FF0000180F86D
:100B2000FB1041F25806C2F20006F578457037799D
:100B30000770FCF7D9B843F21416C2F2000641F26E
:100B40005802C2F200021378507800909178019117
:100B500030464FF0FB014EF62822C0F6030208F0A3
:100B600015FE86F8FB00FCF7BFB843F21415C2F27D
:100B7000000541F25807C2F200073B787E780096E4
:100B800028464FF0FB014EF63822C0F6030208F06B
:100B9000FDFD85F8FB00FCF7A7B841F25803C2F24F
:100BA0000003D878052808D941F25801C2F20001A3
:100BB0004FF00005CD70FCF797B800F1010041F24D
:100BC0005802C2F20002D070FCF78EB841F258070A
:100BD000C2F200073E7806F10106F3B23B703879A5
:100BE000FF280BD1632B7CF67FA841F25805C2F297
:100BF00000054FF000072F70FCF776B8172B7CF636
:100C000073A841F25801C2F200014FF000020A70CD
:100C1000FCF76AB841F25806C2F20006737803F195
:100C20000103D8B270703179FF290BD10C287CF602
:100C30005BA841F25807C2F200074FF001067E7030
:100C4000FCF752B83B287CF64FA841F25805C2F297
:100C500000054FF000026A70FCF746B841F25803F5
:100C6000C2F20003987800F10100C5B29D701979B5
:100C7000FF291DD15DB141F25802C2F2000217787E
:100C8000507807F5FA61F6F757FF854208D941F227
:100C90005807C2F200074FF00106BE70FCF724B8F7
:100CA00041F25806C2F200063379FF2B3CF41CA82F
:100CB00041F25800C2F2000085783B2D7CF614A862
:100CC00041F25801C2F200014FF000028A70FCF7B5
:100CD0000BB841F25803C2F20003D8784FF0010577
:100CE00005FA00F5197985EA01021A71FBF7FCBFD4
:100CF0000DF1700CF9F72AFB41F25807C2F2000718
:100D00003871FBF7F1BF0DF1700CF9F71FFB0628E6
:100D100041F25806C2F2000692BFF0700023F37051
:100D2000FBF7E2BF0DF1700CF9F710FB41F258052B
:100D3000C2F200052870FBF7D7BF0DF1700CF9F770
:100D400005FB41F25801C2F200014870FBF7CCBF2D
:100D50000DF1700CF9F7FAFA41F25802C2F20002F2
:100D60009070FBF7C1BF0DF1700C41F25800C2F258
:100D700000000079F9F7D2FAFBF7B6BF0DF1700C5D
:100D800041F25807C2F20007F878F9F7C7FAFBF703
:100D9000ABBF0DF1700C41F25806C2F2000630787C
:100DA000F9F7BCFAFBF7A0BF0DF1700C41F2580344
:100DB000C2F200035878F9F7B1FAFBF795BF0DF1CD
:100DC000700C41F25805C2F20005A878F9F7A6FAAE
:100DD000FBF78ABF11A8F0F7B1FF41F25803C2F246
:100DE0000003169D48F21F50C5F2EB1080FB050270
:100DF0004FEAE577C7EB62164FF0640101FB165529
:100E00001D70159800F101005870149A9A70179B84
:100E10001BB103F1FF36F7B201E04FF0060741F2D4
:100E20005801C2F20001CF704FF0FF050D71FBF7C2
:100E30005BBF1D9A0F2A08D943F2D804C2F20004FE
:100E40004FF02700207201F08AB9C64800EB8201FA
:100E500041F25807C2F2000710F822603E704B784A
:100E60007B704FF00005BD70FD708A783A71FBF71A
:100E70003BBF41F25800C2F20000FAF7D1F9FBF78C
:100E800033BF41F25807C2F20007FE784FF001016C
:100E900001FA06F13B7941EA03053D71FBF724BFF6
:100EA00011A8F0F74BFF41F25800C2F2000002789F
:100EB00002F164021692477807F1FF3615968178A1
:100EC000149111A8F0F7A0FF84E71D980F2808D906
:100ED00043F2D804C2F200044FF02702227201F05C
:100EE0003EB9C0B2FAF7B8F90DF1700CF9F716FA7D
:100EF000FBF7FABE4FF0000313931293119319936B
:100F000041F25807C2F200073E7806F164061696D1
:100F1000797801F1FF351595B878149011A808F08B
:100F20006DFE179A1AB102F1FF37FBB201E04FF0E4
:100F3000060341F25806C2F20006F370FBF7D4BE76
:100F40001D9A0F2A08D943F2D804C2F200044FF0C8
:100F50002702227201F003B9824800EB820141F2BC
:100F60005803C2F200031D7800F822505F784F70DA
:100F70001E798E70FBF7B8BE11A8F0F7DFFE41F2C4
:100F80005800C2F2000001781391437812938578DB
:100F9000119511A8F0F738FFFBF7A6BE0DF1700C04
:100FA000219F97F85000F9F7B9F9FBF79DBE43F27E
:100FB000E806C2F20006347814F0010F08D143F2BB
:100FC000D806C2F200064FF03004347201F0C7B800
:100FD00043F29C02C2F20002106840B943F2D80109
:100FE000C2F200014FF031030B7201F0B8B843F2C6
:100FF000E801C2F200010B7803F0FE0646F004049B
:101000000C7043F2B000C2F200004FF00002026028
:1010100001F011B843F2E800C2F20000027812F0C9
:10102000010F08D143F2D800C2F200004FF03002A5
:10103000027201F094B843F29C01C2F200010B6805
:1010400043B943F2D806C2F200064FF034043472BA
:1010500001F085B843F2E806C2F20006347804F0E5
:10106000FE0040F00202327043F2B001C2F2000111
:101070004FF000030B6000F0DEBF219D95F8467035
:101080000DF1700CF9F762F921993B1A91F8506053
:1010900006F001001A1A1C9281F84720FF2A94BF1B
:1010A0000022012281F85020FBF71EBE43F2E80126
:1010B000C2F200010B7813F0280F06D01D9EB6F582
:1010C000005F34BF0026012604E01D9EFA2E94BF67
:1010D0000026012646B143F2D804C2F200044FF0C4
:1010E0001302227201F03BB841F26005C2F2000522
:1010F0001E9F1D982F54FBF7F7BD4FF000011C9168
:101100001AE04FF001031C9316E04FF002061C9604
:1011100012E04FF003051C950EE04FF004071C97FA
